 DrawLine

 Timestamp is 5d5f3e77 (Fri Aug 23 04:16:39 2019)

 Preferred load address is 10000000

 Start         Length     Name                   Class
 0001:00000000 00000004H .CRT$XCA                CODE
 0001:00000004 00000004H .CRT$XCZ                CODE
 0001:00000008 00000004H .CRT$XIA                CODE
 0001:0000000c 0000000cH .CRT$XIC                CODE
 0001:00000018 00000004H .CRT$XIZ                CODE
 0001:0000001c 00000004H .CRT$XPA                CODE
 0001:00000020 00000008H .CRT$XPX                CODE
 0001:00000028 00000004H .CRT$XPXA               CODE
 0001:0000002c 00000004H .CRT$XPZ                CODE
 0001:00000030 00000004H .CRT$XTA                CODE
 0001:00000034 0000000cH .CRT$XTZ                CODE
 0001:00000038 00000000H .gfids$y                CODE
 0001:00000040 00004c50H .rdata                  CODE
 0001:00004c90 00000000H .rdata$r                CODE
 0001:00004c90 0000000cH .rdata$sxdata           CODE
 0001:00004c9c 00000278H .rdata$zzzdbg           CODE
 0001:00004f14 00000004H .rtc$IAA                CODE
 0001:00004f18 00000004H .rtc$IZZ                CODE
 0001:00004f1c 00000004H .rtc$TAA                CODE
 0001:00004f20 00000010H .rtc$TZZ                CODE
 0001:00004f30 0000c090H .text$mn                CODE
 0001:00010fb7 00000000H .text$x                 CODE
 0001:00010fc0 00000040H .text$yd                CODE
 0001:00011000 000003e0H .xdata$x                CODE
 0001:000113e0 00000091H .edata                  CODE
 0002:00000000 00000a00H .data                   DATA
 0002:00000a00 00000000H .data$r                 DATA
 0002:00000a00 00000b44H .bss                    DATA
 0003:00000000 00000108H .idata$5                DATA
 0003:00000108 00000004H .00cfg                  DATA
 0003:0000010c 00000014H .idata$2                DATA
 0003:00000120 00000014H .idata$3                DATA
 0003:00000134 00000108H .idata$4                DATA
 0003:0000023c 000004bcH .idata$6                DATA
 0004:00000000 00000060H .rsrc$01                DATA
 0004:00000060 00000370H .rsrc$02                DATA

  Address         Publics by Value              Rva+Base       Lib:Object

 0000:00000000       ___guard_longjmp_count     00000000     <absolute>
 0000:00000000       ___guard_iat_count         00000000     <absolute>
 0000:00000000       __except_list              00000000     <absolute>
 0000:00000000       ___guard_fids_count        00000000     <absolute>
 0000:00000000       ___guard_longjmp_table     00000000     <absolute>
 0000:00000000       ___hybrid_code_map_count   00000000     <absolute>
 0000:00000000       ___hybrid_auxiliary_iat    00000000     <absolute>
 0000:00000000       ___dynamic_value_reloc_table 00000000     <absolute>
 0000:00000000       ___guard_fids_table        00000000     <absolute>
 0000:00000000       ___volatile_metadata       00000000     <absolute>
 0000:00000000       ___guard_iat_table         00000000     <absolute>
 0000:00000000       ___enclave_config          00000000     <absolute>
 0000:00000000       ___hybrid_code_map         00000000     <absolute>
 0000:00000003       ___safe_se_handler_count   00000003     <absolute>
 0000:00000100       ___guard_flags             00000100     <absolute>
 0000:00000000       ___ImageBase               10000000     <linker-defined>
 0001:00000000       ___xc_a                    10001000     LIBCMT:initializers.obj
 0001:00000004       ___xc_z                    10001004     LIBCMT:initializers.obj
 0001:00000008       ___xi_a                    10001008     LIBCMT:initializers.obj
 0001:0000000c       ___acrt_multibyte_initializer 1000100c     libucrt:multibyte_initializer.obj
 0001:00000010       ___acrt_stdio_initializer  10001010     libucrt:stdio_initializer.obj
 0001:00000014       ___acrt_tran_sse2_initializer 10001014     libucrt:sse2_initializer.obj
 0001:00000018       ___xi_z                    10001018     LIBCMT:initializers.obj
 0001:0000001c       ___xp_a                    1000101c     LIBCMT:initializers.obj
 0001:00000020       ___acrt_locale_terminator  10001020     libucrt:locale_initializer.obj
 0001:00000024       ___dcrt_console_output_terminator 10001024     libucrt:console_output_initializer.obj
 0001:00000028       ___acrt_stdio_terminator   10001028     libucrt:stdio_initializer.obj
 0001:0000002c       ___xp_z                    1000102c     LIBCMT:initializers.obj
 0001:00000030       ___xt_a                    10001030     LIBCMT:initializers.obj
 0001:00000034       ___xt_z                    10001034     LIBCMT:initializers.obj
 0001:00000040       _MainGuid                  10001040     DrawLine.obj
 0001:00000050       _MenuGuid                  10001050     DrawLine.obj
 0001:00000060       ??_C@_1BC@EFCDDCCP@?$AAD?$AAr?$AAa?$AAw?$AAL?$AAi?$AAn?$AAe@ 10001060     DrawLine.obj
 0001:00000074       ??_C@_1DG@JDOJGKBC@?$AAD?$AAr?$AAa?$AAw?$AA?5?$AAl?$AAi?$AAn?$AAe?$AAs?$AA?5?$AAf?$AAo?$AAr?$AA?5@ 10001074     DrawLine.obj
 0001:000000ac       ??_C@_1DE@BGKMIKPD@?$AAE?$AAu?$AAg?$AAe?$AAn?$AAe?$AA?5?$AAR?$AAo?$AAs?$AAh?$AAa?$AAl?$AA?5?$AA?$CG@ 100010ac     DrawLine.obj
 0001:000000e0       ??_C@_11LOCGONAA@@         100010e0     DrawLine.obj
 0001:000000f0       __imp__EncodePointer@4     100010f0     vc_crt_fix.obj
 0001:000000f4       __imp__DecodePointer@4     100010f4     vc_crt_fix.obj
 0001:000000f8       __imp__GetModuleHandleExW@12 100010f8     vc_crt_fix.obj
 0001:000000fc       __imp__InitializeSListHead@4 100010fc     vc_crt_fix.obj
 0001:00000100       __imp__InterlockedFlushSList@4 10001100     vc_crt_fix.obj
 0001:00000104       __imp__InterlockedPopEntrySList@4 10001104     vc_crt_fix.obj
 0001:00000108       __imp__InterlockedPushEntrySList@8 10001108     vc_crt_fix.obj
 0001:0000010c       __imp__InterlockedPushListSListEx@16 1000110c     vc_crt_fix.obj
 0001:00000110       __imp__RtlFirstEntrySList@4 10001110     vc_crt_fix.obj
 0001:00000114       __imp__QueryDepthSList@4   10001114     vc_crt_fix.obj
 0001:00000118       __imp__GetNumaHighestNodeNumber@4 10001118     vc_crt_fix.obj
 0001:0000011c       __imp__GetLogicalProcessorInformation@8 1000111c     vc_crt_fix.obj
 0001:00000140       ??_C@_0O@NLDKAIKN@EncodePointer@ 10001140     vc_crt_fix_impl.obj
 0001:00000150       ??_C@_0O@KBPMFGHI@DecodePointer@ 10001150     vc_crt_fix_impl.obj
 0001:00000160       ??_C@_0BD@GIGEJCNH@GetModuleHandleExW@ 10001160     vc_crt_fix_impl.obj
 0001:00000174       ??_C@_0BE@NBEJPEJA@InitializeSListHead@ 10001174     vc_crt_fix_impl.obj
 0001:00000188       ??_C@_0BG@PLLPFLHB@InterlockedFlushSList@ 10001188     vc_crt_fix_impl.obj
 0001:000001a0       ??_C@_0BJ@PNEEKDOK@InterlockedPopEntrySList@ 100011a0     vc_crt_fix_impl.obj
 0001:000001bc       ??_C@_0BK@JFGGAIOA@InterlockedPushEntrySList@ 100011bc     vc_crt_fix_impl.obj
 0001:000001d8       ??_C@_0BL@FOECAEGO@InterlockedPushListSListEx@ 100011d8     vc_crt_fix_impl.obj
 0001:000001f4       ??_C@_0BD@FHMMIGCI@RtlFirstEntrySList@ 100011f4     vc_crt_fix_impl.obj
 0001:00000208       ??_C@_0BA@FGPHPMJB@QueryDepthSList@ 10001208     vc_crt_fix_impl.obj
 0001:00000218       ??_C@_0BJ@NLNFLAMA@GetNumaHighestNodeNumber@ 10001218     vc_crt_fix_impl.obj
 0001:00000234       ??_C@_0BP@KHGALBC@GetLogicalProcessorInformation@ 10001234     vc_crt_fix_impl.obj
 0001:00000254       __pRawDllMain              10001254     LIBCMT:dll_dllmain.obj
 0001:00000254       __pDefaultRawDllMain       10001254     LIBCMT:dll_dllmain.obj
 0001:0000026c       ??_C@_1DM@KHCHBNEB@?$AAa?$AAp?$AAi?$AA?9?$AAm?$AAs?$AA?9?$AAw?$AAi?$AAn?$AA?9?$AAc?$AAo?$AAr?$AAe@ 1000126c     libvcruntime:winapi_downlevel.obj
 0001:000002a8       ??_C@_1DK@LPPGFMPP@?$AAa?$AAp?$AAi?$AA?9?$AAm?$AAs?$AA?9?$AAw?$AAi?$AAn?$AA?9?$AAc?$AAo?$AAr?$AAe@ 100012a8     libvcruntime:winapi_downlevel.obj
 0001:000002e4       ??_C@_1BC@GDMECMAK@?$AAk?$AAe?$AAr?$AAn?$AAe?$AAl?$AA3?$AA2@ 100012e4     libvcruntime:winapi_downlevel.obj
 0001:000002f8       ??_C@_1BA@PFFKHIOG@?$AAa?$AAp?$AAi?$AA?9?$AAm?$AAs?$AA?9@ 100012f8     libvcruntime:winapi_downlevel.obj
 0001:00000308       ??_C@_1BA@IAIFMGEF@?$AAe?$AAx?$AAt?$AA?9?$AAm?$AAs?$AA?9@ 10001308     libvcruntime:winapi_downlevel.obj
 0001:00000320       ??_C@_08KNHFBNJ@FlsAlloc@  10001320     libvcruntime:winapi_downlevel.obj
 0001:00000334       ??_C@_07PEJMOBNF@FlsFree@  10001334     libvcruntime:winapi_downlevel.obj
 0001:00000344       ??_C@_0M@GDNOONDI@FlsGetValue@ 10001344     libvcruntime:winapi_downlevel.obj
 0001:00000358       ??_C@_0M@JCPCPOEF@FlsSetValue@ 10001358     libvcruntime:winapi_downlevel.obj
 0001:0000036c       ??_C@_0BM@HCFOFFN@InitializeCriticalSectionEx@ 1000136c     libvcruntime:winapi_downlevel.obj
 0001:00000524       ??_C@_08EHJDFFNH@__based?$CI@ 10001524     libvcruntime:undname.obj
 0001:00000530       ??_C@_07KOLFKCDI@__cdecl@  10001530     libvcruntime:undname.obj
 0001:00000538       ??_C@_08GHMPAG@__pascal@   10001538     libvcruntime:undname.obj
 0001:00000544       ??_C@_09IFJBGAPI@__stdcall@ 10001544     libvcruntime:undname.obj
 0001:00000550       ??_C@_0L@NPHFGOKO@__thiscall@ 10001550     libvcruntime:undname.obj
 0001:0000055c       ??_C@_0L@JMKHOMEK@__fastcall@ 1000155c     libvcruntime:undname.obj
 0001:00000568       ??_C@_0N@BCKKPABJ@__vectorcall@ 10001568     libvcruntime:undname.obj
 0001:00000578       ??_C@_09HIJEGCPM@__clrcall@ 10001578     libvcruntime:undname.obj
 0001:00000584       ??_C@_06GHPCKEAG@__eabi@   10001584     libvcruntime:undname.obj
 0001:0000058c       ??_C@_09IOPIDJLG@__swift_1@ 1000158c     libvcruntime:undname.obj
 0001:00000598       ??_C@_09KFNFGKHF@__swift_2@ 10001598     libvcruntime:undname.obj
 0001:000005a4       ??_C@_07JOMMBBKO@__ptr64@  100015a4     libvcruntime:undname.obj
 0001:000005ac       ??_C@_0L@PILCLIHE@__restrict@ 100015ac     libvcruntime:undname.obj
 0001:000005b8       ??_C@_0M@GFIIJFMG@__unaligned@ 100015b8     libvcruntime:undname.obj
 0001:000005c4       ??_C@_09DHDLOLLB@restrict?$CI@ 100015c4     libvcruntime:undname.obj
 0001:000005ce       ??_C@_00CNPNBAHC@@         100015ce     libvcruntime:undname.obj
 0001:000005d0       ??_C@_04NIHEBCM@?5new@     100015d0     libvcruntime:undname.obj
 0001:000005d8       ??_C@_07FPCDHGMM@?5delete@ 100015d8     libvcruntime:undname.obj
 0001:000005e0       ??_C@_01NEMOKFLO@?$DN@     100015e0     libvcruntime:undname.obj
 0001:000005e4       ??_C@_02GPIOPFAK@?$DO?$DO@ 100015e4     libvcruntime:undname.obj
 0001:000005e8       ??_C@_02FODMEDOG@?$DM?$DM@ 100015e8     libvcruntime:undname.obj
 0001:000005ec       ??_C@_01DCLJPIOD@?$CB@     100015ec     libvcruntime:undname.obj
 0001:000005f0       ??_C@_02EGOFBIJA@?$DN?$DN@ 100015f0     libvcruntime:undname.obj
 0001:000005f4       ??_C@_02FDNJECIE@?$CB?$DN@ 100015f4     libvcruntime:undname.obj
 0001:000005f8       ??_C@_02GPECMEKF@?$FL?$FN@ 100015f8     libvcruntime:undname.obj
 0001:000005fc       ??_C@_08LHJFAFGD@operator@ 100015fc     libvcruntime:undname.obj
 0001:00000608       ??_C@_02HBOOOICD@?9?$DO@   10001608     libvcruntime:undname.obj
 0001:0000060c       ??_C@_01NBENCBCI@?$CK@     1000160c     libvcruntime:undname.obj
 0001:00000610       ??_C@_02ECNGHCIF@?$CL?$CL@ 10001610     libvcruntime:undname.obj
 0001:00000614       ??_C@_02BAABKJLB@?9?9@     10001614     libvcruntime:undname.obj
 0001:00000618       ??_C@_01JOAMLHOP@?9@       10001618     libvcruntime:undname.obj
 0001:0000061c       ??_C@_01MIFGBAGJ@?$CL@     1000161c     libvcruntime:undname.obj
 0001:00000620       ??_C@_01HNPIGOCE@?$CG@     10001620     libvcruntime:undname.obj
 0001:00000624       ??_C@_03MNHNFDLC@?9?$DO?$CK@ 10001624     libvcruntime:undname.obj
 0001:00000628       ??_C@_01KMDKNFGN@?1@       10001628     libvcruntime:undname.obj
 0001:0000062c       ??_C@_01FGNFDNOH@?$CF@     1000162c     libvcruntime:undname.obj
 0001:00000630       ??_C@_01MNNFJEPP@?$DM@     10001630     libvcruntime:undname.obj
 0001:00000634       ??_C@_02EHCHHCKH@?$DM?$DN@ 10001634     libvcruntime:undname.obj
 0001:00000638       ??_C@_01PPODPGHN@?$DO@     10001638     libvcruntime:undname.obj
 0001:0000063c       ??_C@_02EEKDKGMJ@?$DO?$DN@ 1000163c     libvcruntime:undname.obj
 0001:00000640       ??_C@_01IHBHIGKO@?0@       10001640     libvcruntime:undname.obj
 0001:00000644       ??_C@_02HCKGKOFO@?$CI?$CJ@ 10001644     libvcruntime:undname.obj
 0001:00000648       ??_C@_01PJKLJHI@?$HO@      10001648     libvcruntime:undname.obj
 0001:0000064c       ??_C@_01JKBOJNNK@?$FO@     1000164c     libvcruntime:undname.obj
 0001:00000650       ??_C@_01DNKMNLPK@?$HM@     10001650     libvcruntime:undname.obj
 0001:00000654       ??_C@_02PPKAJPJL@?$CG?$CG@ 10001654     libvcruntime:undname.obj
 0001:00000658       ??_C@_02NONPIBCD@?$HM?$HM@ 10001658     libvcruntime:undname.obj
 0001:0000065c       ??_C@_02FPIMKNGF@?$CK?$DN@ 1000165c     libvcruntime:undname.obj
 0001:00000660       ??_C@_02FOEOMHFC@?$CL?$DN@ 10001660     libvcruntime:undname.obj
 0001:00000664       ??_C@_02FKMDLLOA@?9?$DN@   10001664     libvcruntime:undname.obj
 0001:00000668       ??_C@_02FJEHGPIO@?1?$DN@   10001668     libvcruntime:undname.obj
 0001:0000066c       ??_C@_02FENAOKFI@?$CF?$DN@ 1000166c     libvcruntime:undname.obj
 0001:00000670       ??_C@_03IKFCCPFF@?$DO?$DO?$DN@ 10001670     libvcruntime:undname.obj
 0001:00000674       ??_C@_03CDNPDDLA@?$DM?$DM?$DN@ 10001674     libvcruntime:undname.obj
 0001:00000678       ??_C@_02FGJGFEAB@?$CG?$DN@ 10001678     libvcruntime:undname.obj
 0001:0000067c       ??_C@_02DHLNPPGH@?$HM?$DN@ 1000167c     libvcruntime:undname.obj
 0001:00000680       ??_C@_02MHEGNOJ@?$FO?$DN@  10001680     libvcruntime:undname.obj
 0001:00000684       ??_C@_09IFPLHPGF@?$GAvftable?8@ 10001684     libvcruntime:undname.obj
 0001:00000690       ??_C@_09BLBHBJP@?$GAvbtable?8@ 10001690     libvcruntime:undname.obj
 0001:0000069c       ??_C@_07FEEIOKP@?$GAvcall?8@ 1000169c     libvcruntime:undname.obj
 0001:000006a4       ??_C@_08LLFFHHDJ@?$GAtypeof?8@ 100016a4     libvcruntime:undname.obj
 0001:000006b0       ??_C@_0BF@KDPPACIK@?$GAlocal?5static?5guard?8@ 100016b0     libvcruntime:undname.obj
 0001:000006c8       ??_C@_08OBABFOLI@?$GAstring?8@ 100016c8     libvcruntime:undname.obj
 0001:000006d4       ??_C@_0BD@JDLKDPAB@?$GAvbase?5destructor?8@ 100016d4     libvcruntime:undname.obj
 0001:000006e8       ??_C@_0BN@DEGPLNFK@?$GAvector?5deleting?5destructor?8@ 100016e8     libvcruntime:undname.obj
 0001:00000708       ??_C@_0BO@OBMKPJIG@?$GAdefault?5constructor?5closure?8@ 10001708     libvcruntime:undname.obj
 0001:00000728       ??_C@_0BN@IMDCHIKM@?$GAscalar?5deleting?5destructor?8@ 10001728     libvcruntime:undname.obj
 0001:00000748       ??_C@_0BO@PFGOCPJJ@?$GAvector?5constructor?5iterator?8@ 10001748     libvcruntime:undname.obj
 0001:00000768       ??_C@_0BN@LFPFMEDL@?$GAvector?5destructor?5iterator?8@ 10001768     libvcruntime:undname.obj
 0001:00000788       ??_C@_0CE@IKBNEHA@?$GAvector?5vbase?5constructor?5itera@ 10001788     libvcruntime:undname.obj
 0001:000007ac       ??_C@_0BL@NILFHHPC@?$GAvirtual?5displacement?5map?8@ 100017ac     libvcruntime:undname.obj
 0001:000007c8       ??_C@_0CB@JONCMFFK@?$GAeh?5vector?5constructor?5iterator@ 100017c8     libvcruntime:undname.obj
 0001:000007ec       ??_C@_0CA@GCEOPDGL@?$GAeh?5vector?5destructor?5iterator?8@ 100017ec     libvcruntime:undname.obj
 0001:0000080c       ??_C@_0CH@OOJPLCPH@?$GAeh?5vector?5vbase?5constructor?5it@ 1000180c     libvcruntime:undname.obj
 0001:00000834       ??_C@_0BL@LLKPOHJI@?$GAcopy?5constructor?5closure?8@ 10001834     libvcruntime:undname.obj
 0001:00000850       ??_C@_0BA@KBCDOMBN@?$GAudt?5returning?8@ 10001850     libvcruntime:undname.obj
 0001:00000860       ??_C@_03KLGMFNMG@?$GAEH@   10001860     libvcruntime:undname.obj
 0001:00000864       ??_C@_05KHLCHHI@?$GARTTI@  10001864     libvcruntime:undname.obj
 0001:0000086c       ??_C@_0BA@KKLDJDLB@?$GAlocal?5vftable?8@ 1000186c     libvcruntime:undname.obj
 0001:0000087c       ??_C@_0CE@IIHCMGGL@?$GAlocal?5vftable?5constructor?5clos@ 1000187c     libvcruntime:undname.obj
 0001:000008a0       ??_C@_06FHBGPFGH@?5new?$FL?$FN@ 100018a0     libvcruntime:undname.obj
 0001:000008a8       ??_C@_09LBNFPBCA@?5delete?$FL?$FN@ 100018a8     libvcruntime:undname.obj
 0001:000008b4       ??_C@_0P@HJKNJFNN@?$GAomni?5callsig?8@ 100018b4     libvcruntime:undname.obj
 0001:000008c4       ??_C@_0BL@CNOONJFP@?$GAplacement?5delete?5closure?8@ 100018c4     libvcruntime:undname.obj
 0001:000008e0       ??_C@_0BN@CKNJLHMB@?$GAplacement?5delete?$FL?$FN?5closure?8@ 100018e0     libvcruntime:undname.obj
 0001:00000900       ??_C@_0CG@CFDHKGGD@?$GAmanaged?5vector?5constructor?5ite@ 10001900     libvcruntime:undname.obj
 0001:00000928       ??_C@_0CF@IMGKMJNO@?$GAmanaged?5vector?5destructor?5iter@ 10001928     libvcruntime:undname.obj
 0001:00000950       ??_C@_0CG@HLDDJMAG@?$GAeh?5vector?5copy?5constructor?5ite@ 10001950     libvcruntime:undname.obj
 0001:00000978       ??_C@_0CM@FCBBDIGB@?$GAeh?5vector?5vbase?5copy?5construct@ 10001978     libvcruntime:undname.obj
 0001:000009a4       ??_C@_0BL@CLIPGLGB@?$GAdynamic?5initializer?5for?5?8@ 100019a4     libvcruntime:undname.obj
 0001:000009c0       ??_C@_0CB@PDBIFEP@?$GAdynamic?5atexit?5destructor?5for?5@ 100019c0     libvcruntime:undname.obj
 0001:000009e4       ??_C@_0CD@CGAJBKEJ@?$GAvector?5copy?5constructor?5iterat@ 100019e4     libvcruntime:undname.obj
 0001:00000a08       ??_C@_0CJ@GJELGAMM@?$GAvector?5vbase?5copy?5constructor?5@ 10001a08     libvcruntime:undname.obj
 0001:00000a34       ??_C@_0CL@FGIJHLCE@?$GAmanaged?5vector?5copy?5constructo@ 10001a34     libvcruntime:undname.obj
 0001:00000a60       ??_C@_0BM@PMGGMLDN@?$GAlocal?5static?5thread?5guard?8@ 10001a60     libvcruntime:undname.obj
 0001:00000a7c       ??_C@_0N@BDNMDMOL@operator?5?$CC?$CC?5@ 10001a7c     libvcruntime:undname.obj
 0001:00000a8c       ??_C@_0BC@GGEBGALA@operator?5co_await@ 10001a8c     libvcruntime:undname.obj
 0001:00000aa0       ??_C@_0BC@DAFEJGAK@?5Type?5Descriptor?8@ 10001aa0     libvcruntime:undname.obj
 0001:00000ab4       ??_C@_0BM@LDKODKLH@?5Base?5Class?5Descriptor?5at?5?$CI@ 10001ab4     libvcruntime:undname.obj
 0001:00000ad0       ??_C@_0BD@LGICGFMM@?5Base?5Class?5Array?8@ 10001ad0     libvcruntime:undname.obj
 0001:00000ae4       ??_C@_0BN@MECKDCOJ@?5Class?5Hierarchy?5Descriptor?8@ 10001ae4     libvcruntime:undname.obj
 0001:00000b04       ??_C@_0BK@CFCOFLF@?5Complete?5Object?5Locator?8@ 10001b04     libvcruntime:undname.obj
 0001:00000b20       __pDestructExceptionObject 10001b20     libvcruntime:ehhelpers.obj
 0001:00000b28       ___acrt_exception_action_table 10001b28     libucrt:exception_filter.obj
 0001:00000bb8       ___acrt_signal_action_table_count 10001bb8     libucrt:exception_filter.obj
 0001:00000bbc       ___acrt_signal_action_first_fpe_index 10001bbc     libucrt:exception_filter.obj
 0001:00000bc0       ___acrt_signal_action_fpe_count 10001bc0     libucrt:exception_filter.obj
 0001:00000bc4       ??_C@_1BI@BGOHAHKC@?$AAm?$AAs?$AAc?$AAo?$AAr?$AAe?$AAe?$AA?4?$AAd?$AAl?$AAl?$AA?$AA@ 10001bc4     libucrt:exit.obj
 0001:00000bdc       ??_C@_0P@MIGLKIOC@CorExitProcess?$AA@ 10001bdc     libucrt:exit.obj
 0001:00000de8       ??_C@_1M@HPNHIDJI@?$AAj?$AAa?$AA?9?$AAJ?$AAP?$AA?$AA@ 10001de8     libucrt:mbctype.obj
 0001:00000df4       ??_C@_1M@BIBDDEMK@?$AAz?$AAh?$AA?9?$AAC?$AAN?$AA?$AA@ 10001df4     libucrt:mbctype.obj
 0001:00000e00       ??_C@_1M@JLOOOEGK@?$AAk?$AAo?$AA?9?$AAK?$AAR?$AA?$AA@ 10001e00     libucrt:mbctype.obj
 0001:00000e0c       ??_C@_1M@CLNBBOPM@?$AAz?$AAh?$AA?9?$AAT?$AAW?$AA?$AA@ 10001e0c     libucrt:mbctype.obj
 0001:00000e68       ??_C@_1EA@JGEFHKEI@?$AAa?$AAp?$AAi?$AA?9?$AAm?$AAs?$AA?9?$AAw?$AAi?$AAn?$AA?9?$AAc?$AAo?$AAr?$AAe?$AA?9?$AAd?$AAa?$AAt?$AAe?$AAt?$AAi?$AAm?$AAe?$AA?9?$AAl?$AA1?$AA?9?$AA1?$AA?9?$AA1?$AA?$AA@ 10001e68     libucrt:winapi_thunks.obj
 0001:00000ea8       ??_C@_1DM@KHCHBNEB@?$AAa?$AAp?$AAi?$AA?9?$AAm?$AAs?$AA?9?$AAw?$AAi?$AAn?$AA?9?$AAc?$AAo?$AAr?$AAe?$AA?9?$AAf?$AAi?$AAb?$AAe?$AAr?$AAs?$AA?9?$AAl?$AA1?$AA?9?$AA1?$AA?9?$AA1?$AA?$AA@ 10001ea8     libucrt:winapi_thunks.obj
 0001:00000ee4       ??_C@_1DI@IJCEHOCB@?$AAa?$AAp?$AAi?$AA?9?$AAm?$AAs?$AA?9?$AAw?$AAi?$AAn?$AA?9?$AAc?$AAo?$AAr?$AAe?$AA?9?$AAf?$AAi?$AAl?$AAe?$AA?9?$AAl?$AA1?$AA?9?$AA2?$AA?9?$AA2?$AA?$AA@ 10001ee4     libucrt:winapi_thunks.obj
 0001:00000f20       ??_C@_1EI@MPIAOHOC@?$AAa?$AAp?$AAi?$AA?9?$AAm?$AAs?$AA?9?$AAw?$AAi?$AAn?$AA?9?$AAc?$AAo?$AAr?$AAe?$AA?9?$AAl?$AAo?$AAc?$AAa?$AAl?$AAi?$AAz?$AAa?$AAt?$AAi?$AAo?$AAn?$AA?9?$AAl?$AA1?$AA?9@ 10001f20     libucrt:winapi_thunks.obj
 0001:00000f68       ??_C@_1FK@FPHCKFIE@?$AAa?$AAp?$AAi?$AA?9?$AAm?$AAs?$AA?9?$AAw?$AAi?$AAn?$AA?9?$AAc?$AAo?$AAr?$AAe?$AA?9?$AAl?$AAo?$AAc?$AAa?$AAl?$AAi?$AAz?$AAa?$AAt?$AAi?$AAo?$AAn?$AA?9?$AAo?$AAb?$AAs@ 10001f68     libucrt:winapi_thunks.obj
 0001:00000fc8       ??_C@_1EM@DILCGIIO@?$AAa?$AAp?$AAi?$AA?9?$AAm?$AAs?$AA?9?$AAw?$AAi?$AAn?$AA?9?$AAc?$AAo?$AAr?$AAe?$AA?9?$AAp?$AAr?$AAo?$AAc?$AAe?$AAs?$AAs?$AAt?$AAh?$AAr?$AAe?$AAa?$AAd?$AAs?$AA?9?$AAl@ 10001fc8     libucrt:winapi_thunks.obj
 0001:00001014       ??_C@_1DM@LNCGDDPN@?$AAa?$AAp?$AAi?$AA?9?$AAm?$AAs?$AA?9?$AAw?$AAi?$AAn?$AA?9?$AAc?$AAo?$AAr?$AAe?$AA?9?$AAs?$AAt?$AAr?$AAi?$AAn?$AAg?$AA?9?$AAl?$AA1?$AA?9?$AA1?$AA?9?$AA0?$AA?$AA@ 10002014     libucrt:winapi_thunks.obj
 0001:00001050       ??_C@_1DK@LPPGFMPP@?$AAa?$AAp?$AAi?$AA?9?$AAm?$AAs?$AA?9?$AAw?$AAi?$AAn?$AA?9?$AAc?$AAo?$AAr?$AAe?$AA?9?$AAs?$AAy?$AAn?$AAc?$AAh?$AA?9?$AAl?$AA1?$AA?9?$AA2?$AA?9?$AA0?$AA?$AA@ 10002050     libucrt:winapi_thunks.obj
 0001:0000108c       ??_C@_1DO@FPAPJEMD@?$AAa?$AAp?$AAi?$AA?9?$AAm?$AAs?$AA?9?$AAw?$AAi?$AAn?$AA?9?$AAc?$AAo?$AAr?$AAe?$AA?9?$AAs?$AAy?$AAs?$AAi?$AAn?$AAf?$AAo?$AA?9?$AAl?$AA1?$AA?9?$AA2?$AA?9?$AA1?$AA?$AA@ 1000208c     libucrt:winapi_thunks.obj
 0001:000010cc       ??_C@_1DK@NDHNAHIO@?$AAa?$AAp?$AAi?$AA?9?$AAm?$AAs?$AA?9?$AAw?$AAi?$AAn?$AA?9?$AAc?$AAo?$AAr?$AAe?$AA?9?$AAw?$AAi?$AAn?$AAr?$AAt?$AA?9?$AAl?$AA1?$AA?9?$AA1?$AA?9?$AA0?$AA?$AA@ 100020cc     libucrt:winapi_thunks.obj
 0001:00001108       ??_C@_1DM@KGHDGBCM@?$AAa?$AAp?$AAi?$AA?9?$AAm?$AAs?$AA?9?$AAw?$AAi?$AAn?$AA?9?$AAc?$AAo?$AAr?$AAe?$AA?9?$AAx?$AAs?$AAt?$AAa?$AAt?$AAe?$AA?9?$AAl?$AA2?$AA?9?$AA1?$AA?9?$AA0?$AA?$AA@ 10002108     libucrt:winapi_thunks.obj
 0001:00001148       ??_C@_1EO@IJIOEFOH@?$AAa?$AAp?$AAi?$AA?9?$AAm?$AAs?$AA?9?$AAw?$AAi?$AAn?$AA?9?$AAr?$AAt?$AAc?$AAo?$AAr?$AAe?$AA?9?$AAn?$AAt?$AAu?$AAs?$AAe?$AAr?$AA?9?$AAw?$AAi?$AAn?$AAd?$AAo?$AAw?$AA?9@ 10002148     libucrt:winapi_thunks.obj
 0001:00001198       ??_C@_1FG@HHGEKANL@?$AAa?$AAp?$AAi?$AA?9?$AAm?$AAs?$AA?9?$AAw?$AAi?$AAn?$AA?9?$AAs?$AAe?$AAc?$AAu?$AAr?$AAi?$AAt?$AAy?$AA?9?$AAs?$AAy?$AAs?$AAt?$AAe?$AAm?$AAf?$AAu?$AAn?$AAc?$AAt?$AAi@ 10002198     libucrt:winapi_thunks.obj
 0001:000011f0       ??_C@_1EG@DBIOJECG@?$AAe?$AAx?$AAt?$AA?9?$AAm?$AAs?$AA?9?$AAw?$AAi?$AAn?$AA?9?$AAn?$AAt?$AAu?$AAs?$AAe?$AAr?$AA?9?$AAd?$AAi?$AAa?$AAl?$AAo?$AAg?$AAb?$AAo?$AAx?$AA?9?$AAl?$AA1?$AA?9?$AA1@ 100021f0     libucrt:winapi_thunks.obj
 0001:00001238       ??_C@_1EO@FIHMJCLF@?$AAe?$AAx?$AAt?$AA?9?$AAm?$AAs?$AA?9?$AAw?$AAi?$AAn?$AA?9?$AAn?$AAt?$AAu?$AAs?$AAe?$AAr?$AA?9?$AAw?$AAi?$AAn?$AAd?$AAo?$AAw?$AAs?$AAt?$AAa?$AAt?$AAi?$AAo?$AAn?$AA?9@ 10002238     libucrt:winapi_thunks.obj
 0001:00001288       ??_C@_1BC@DNHGCMLG@?$AAa?$AAd?$AAv?$AAa?$AAp?$AAi?$AA3?$AA2?$AA?$AA@ 10002288     libucrt:winapi_thunks.obj
 0001:0000129c       ??_C@_1BC@GDMECMAK@?$AAk?$AAe?$AAr?$AAn?$AAe?$AAl?$AA3?$AA2?$AA?$AA@ 1000229c     libucrt:winapi_thunks.obj
 0001:000012b0       ??_C@_1M@OAIMIKLP@?$AAn?$AAt?$AAd?$AAl?$AAl?$AA?$AA@ 100022b0     libucrt:winapi_thunks.obj
 0001:000012c0       ??_C@_1EG@DPGNFKGC@?$AAa?$AAp?$AAi?$AA?9?$AAm?$AAs?$AA?9?$AAw?$AAi?$AAn?$AA?9?$AAa?$AAp?$AAp?$AAm?$AAo?$AAd?$AAe?$AAl?$AA?9?$AAr?$AAu?$AAn?$AAt?$AAi?$AAm?$AAe?$AA?9?$AAl?$AA1?$AA?9?$AA1@ 100022c0     libucrt:winapi_thunks.obj
 0001:00001308       ??_C@_1O@BCCLBEOE@?$AAu?$AAs?$AAe?$AAr?$AA3?$AA2?$AA?$AA@ 10002308     libucrt:winapi_thunks.obj
 0001:00001318       ??_C@_1BA@PFFKHIOG@?$AAa?$AAp?$AAi?$AA?9?$AAm?$AAs?$AA?9?$AA?$AA@ 10002318     libucrt:winapi_thunks.obj
 0001:00001328       ??_C@_1BA@IAIFMGEF@?$AAe?$AAx?$AAt?$AA?9?$AAm?$AAs?$AA?9?$AA?$AA@ 10002328     libucrt:winapi_thunks.obj
 0001:0000133c       ??_C@_0BA@FHFNEAED@AreFileApisANSI?$AA@ 1000233c     libucrt:winapi_thunks.obj
 0001:00001354       ??_C@_08KNHFBNJ@FlsAlloc?$AA@ 10002354     libucrt:winapi_thunks.obj
 0001:00001368       ??_C@_07PEJMOBNF@FlsFree?$AA@ 10002368     libucrt:winapi_thunks.obj
 0001:00001378       ??_C@_0M@GDNOONDI@FlsGetValue?$AA@ 10002378     libucrt:winapi_thunks.obj
 0001:0000138c       ??_C@_0M@JCPCPOEF@FlsSetValue?$AA@ 1000238c     libucrt:winapi_thunks.obj
 0001:000013a0       ??_C@_0BM@HCFOFFN@InitializeCriticalSectionEx?$AA@ 100023a0     libucrt:winapi_thunks.obj
 0001:000013c4       ??_C@_0O@KKBNKAPF@LCMapStringEx?$AA@ 100023c4     libucrt:winapi_thunks.obj
 0001:000013dc       ??_C@_0BB@HBDEELFH@LocaleNameToLCID?$AA@ 100023dc     libucrt:winapi_thunks.obj
 0001:000013f4       ??_C@_0CF@OJOFEIGO@AppPolicyGetProcessTerminationMe@ 100023f4     libucrt:winapi_thunks.obj
 0001:00001420       ___lc_time_c               10002420     libucrt:nlsdata.obj
 0001:00001584       ??_C@_03KOEHGMDN@Sun?$AA@  10002584     libucrt:nlsdata.obj
 0001:00001588       ??_C@_03PDAGKDH@Mon?$AA@   10002588     libucrt:nlsdata.obj
 0001:0000158c       ??_C@_03NAGEINEP@Tue?$AA@  1000258c     libucrt:nlsdata.obj
 0001:00001590       ??_C@_03MHOMLAJA@Wed?$AA@  10002590     libucrt:nlsdata.obj
 0001:00001594       ??_C@_03IOFIKPDN@Thu?$AA@  10002594     libucrt:nlsdata.obj
 0001:00001598       ??_C@_03IDIOELNC@Fri?$AA@  10002598     libucrt:nlsdata.obj
 0001:0000159c       ??_C@_03FEFJNEK@Sat?$AA@   1000259c     libucrt:nlsdata.obj
 0001:000015a0       ??_C@_06OOPIFAJ@Sunday?$AA@ 100025a0     libucrt:nlsdata.obj
 0001:000015a8       ??_C@_06JLEDEDGH@Monday?$AA@ 100025a8     libucrt:nlsdata.obj
 0001:000015b0       ??_C@_07BAAGCFCM@Tuesday?$AA@ 100025b0     libucrt:nlsdata.obj
 0001:000015b8       ??_C@_09DLIGFAKA@Wednesday?$AA@ 100025b8     libucrt:nlsdata.obj
 0001:000015c4       ??_C@_08HACCIKIA@Thursday?$AA@ 100025c4     libucrt:nlsdata.obj
 0001:000015d0       ??_C@_06JECMNKMI@Friday?$AA@ 100025d0     libucrt:nlsdata.obj
 0001:000015d8       ??_C@_08INBOOONO@Saturday?$AA@ 100025d8     libucrt:nlsdata.obj
 0001:000015e4       ??_C@_03JIHJHPIE@Jan?$AA@  100025e4     libucrt:nlsdata.obj
 0001:000015e8       ??_C@_03HJBDCHOM@Feb?$AA@  100025e8     libucrt:nlsdata.obj
 0001:000015ec       ??_C@_03ODNJBKGA@Mar?$AA@  100025ec     libucrt:nlsdata.obj
 0001:000015f0       ??_C@_03LEOLGMJP@Apr?$AA@  100025f0     libucrt:nlsdata.obj
 0001:000015f4       ??_C@_03CNMDKL@May?$AA@    100025f4     libucrt:nlsdata.obj
 0001:000015f8       ??_C@_03IDFGHECI@Jun?$AA@  100025f8     libucrt:nlsdata.obj
 0001:000015fc       ??_C@_03LBGABGKK@Jul?$AA@  100025fc     libucrt:nlsdata.obj
 0001:00001600       ??_C@_03IFJFEIGA@Aug?$AA@  10002600     libucrt:nlsdata.obj
 0001:00001604       ??_C@_03GGCAPAJC@Sep?$AA@  10002604     libucrt:nlsdata.obj
 0001:00001608       ??_C@_03BMAOKBAD@Oct?$AA@  10002608     libucrt:nlsdata.obj
 0001:0000160c       ??_C@_03JPJOFNIA@Nov?$AA@  1000260c     libucrt:nlsdata.obj
 0001:00001610       ??_C@_03MKABNOCG@Dec?$AA@  10002610     libucrt:nlsdata.obj
 0001:00001614       ??_C@_07CGJPFGJA@January?$AA@ 10002614     libucrt:nlsdata.obj
 0001:0000161c       ??_C@_08GNJGEPFN@February?$AA@ 1000261c     libucrt:nlsdata.obj
 0001:00001628       ??_C@_05HPCKOFNC@March?$AA@ 10002628     libucrt:nlsdata.obj
 0001:00001630       ??_C@_05DMJDNLEJ@April?$AA@ 10002630     libucrt:nlsdata.obj
 0001:00001638       ??_C@_04CNLMGBGM@June?$AA@ 10002638     libucrt:nlsdata.obj
 0001:00001640       ??_C@_04MIEPOIFP@July?$AA@ 10002640     libucrt:nlsdata.obj
 0001:00001648       ??_C@_06LBBHFDDG@August?$AA@ 10002648     libucrt:nlsdata.obj
 0001:00001650       ??_C@_09BHHEALKD@September?$AA@ 10002650     libucrt:nlsdata.obj
 0001:0000165c       ??_C@_07JJNFCEND@October?$AA@ 1000265c     libucrt:nlsdata.obj
 0001:00001664       ??_C@_08HCHEGEOA@November?$AA@ 10002664     libucrt:nlsdata.obj
 0001:00001670       ??_C@_08EDHMEBNP@December?$AA@ 10002670     libucrt:nlsdata.obj
 0001:0000167c       ??_C@_02DEDBPAFC@AM?$AA@   1000267c     libucrt:nlsdata.obj
 0001:00001680       ??_C@_02CJNFDJBF@PM?$AA@   10002680     libucrt:nlsdata.obj
 0001:00001684       ??_C@_08BPBNCDIB@MM?1dd?1yy?$AA@ 10002684     libucrt:nlsdata.obj
 0001:00001690       ??_C@_0BE@CKGJFCPC@dddd?0?5MMMM?5dd?0?5yyyy?$AA@ 10002690     libucrt:nlsdata.obj
 0001:000016a4       ??_C@_08JCCMCCIL@HH?3mm?3ss?$AA@ 100026a4     libucrt:nlsdata.obj
 0001:000016b0       ??_C@_17MBGCMIPB@?$AAS?$AAu?$AAn?$AA?$AA@ 100026b0     libucrt:nlsdata.obj
 0001:000016b8       ??_C@_17KBOMKBF@?$AAM?$AAo?$AAn?$AA?$AA@ 100026b8     libucrt:nlsdata.obj
 0001:000016c0       ??_C@_17BMKGEGOJ@?$AAT?$AAu?$AAe?$AA?$AA@ 100026c0     libucrt:nlsdata.obj
 0001:000016c8       ??_C@_17CJEDCEPE@?$AAW?$AAe?$AAd?$AA?$AA@ 100026c8     libucrt:nlsdata.obj
 0001:000016d0       ??_C@_17PDPHAADD@?$AAT?$AAh?$AAu?$AA?$AA@ 100026d0     libucrt:nlsdata.obj
 0001:000016d8       ??_C@_17HFOLPPLP@?$AAF?$AAr?$AAi?$AA?$AA@ 100026d8     libucrt:nlsdata.obj
 0001:000016e0       ??_C@_17GGIBDPIH@?$AAS?$AAa?$AAt?$AA?$AA@ 100026e0     libucrt:nlsdata.obj
 0001:000016e8       ??_C@_1O@IHNHDHPB@?$AAS?$AAu?$AAn?$AAd?$AAa?$AAy?$AA?$AA@ 100026e8     libucrt:nlsdata.obj
 0001:000016f8       ??_C@_1O@MMNBFLIA@?$AAM?$AAo?$AAn?$AAd?$AAa?$AAy?$AA?$AA@ 100026f8     libucrt:nlsdata.obj
 0001:00001708       ??_C@_1BA@ENFBFFEK@?$AAT?$AAu?$AAe?$AAs?$AAd?$AAa?$AAy?$AA?$AA@ 10002708     libucrt:nlsdata.obj
 0001:00001718       ??_C@_1BE@EBOGMDOH@?$AAW?$AAe?$AAd?$AAn?$AAe?$AAs?$AAd?$AAa?$AAy?$AA?$AA@ 10002718     libucrt:nlsdata.obj
 0001:0000172c       ??_C@_1BC@HHMNLIHE@?$AAT?$AAh?$AAu?$AAr?$AAs?$AAd?$AAa?$AAy?$AA?$AA@ 1000272c     libucrt:nlsdata.obj
 0001:00001740       ??_C@_1O@PDICJHAG@?$AAF?$AAr?$AAi?$AAd?$AAa?$AAy?$AA?$AA@ 10002740     libucrt:nlsdata.obj
 0001:00001750       ??_C@_1BC@ENMNNPAJ@?$AAS?$AAa?$AAt?$AAu?$AAr?$AAd?$AAa?$AAy?$AA?$AA@ 10002750     libucrt:nlsdata.obj
 0001:00001764       ??_C@_17DKNBKCHM@?$AAJ?$AAa?$AAn?$AA?$AA@ 10002764     libucrt:nlsdata.obj
 0001:0000176c       ??_C@_17LMDJEKJN@?$AAF?$AAe?$AAb?$AA?$AA@ 1000276c     libucrt:nlsdata.obj
 0001:00001774       ??_C@_17CKNLEDEC@?$AAM?$AAa?$AAr?$AA?$AA@ 10002774     libucrt:nlsdata.obj
 0001:0000177c       ??_C@_17LFPOIHDD@?$AAA?$AAp?$AAr?$AA?$AA@ 1000277c     libucrt:nlsdata.obj
 0001:00001784       ??_C@_17PNNKMEED@?$AAM?$AAa?$AAy?$AA?$AA@ 10002784     libucrt:nlsdata.obj
 0001:0000178c       ??_C@_17KCJGOCPB@?$AAJ?$AAu?$AAn?$AA?$AA@ 1000278c     libucrt:nlsdata.obj
 0001:00001794       ??_C@_17IJPCKHK@?$AAJ?$AAu?$AAl?$AA?$AA@ 10002794     libucrt:nlsdata.obj
 0001:0000179c       ??_C@_17ICPELBCN@?$AAA?$AAu?$AAg?$AA?$AA@ 1000279c     libucrt:nlsdata.obj
 0001:000017a4       ??_C@_17HCHCOKMG@?$AAS?$AAe?$AAp?$AA?$AA@ 100027a4     libucrt:nlsdata.obj
 0001:000017ac       ??_C@_17FNLKOI@?$AAO?$AAc?$AAt?$AA?$AA@ 100027ac     libucrt:nlsdata.obj
 0001:000017b4       ??_C@_17BBDMLCIG@?$AAN?$AAo?$AAv?$AA?$AA@ 100027b4     libucrt:nlsdata.obj
 0001:000017bc       ??_C@_17EGKACKIF@?$AAD?$AAe?$AAc?$AA?$AA@ 100027bc     libucrt:nlsdata.obj
 0001:000017c4       ??_C@_1BA@EFMEIEBA@?$AAJ?$AAa?$AAn?$AAu?$AAa?$AAr?$AAy?$AA?$AA@ 100027c4     libucrt:nlsdata.obj
 0001:000017d4       ??_C@_1BC@JGDDFFAM@?$AAF?$AAe?$AAb?$AAr?$AAu?$AAa?$AAr?$AAy?$AA?$AA@ 100027d4     libucrt:nlsdata.obj
 0001:000017e8       ??_C@_1M@IKEENEDF@?$AAM?$AAa?$AAr?$AAc?$AAh?$AA?$AA@ 100027e8     libucrt:nlsdata.obj
 0001:000017f4       ??_C@_1M@GJNLMHFD@?$AAA?$AAp?$AAr?$AAi?$AAl?$AA?$AA@ 100027f4     libucrt:nlsdata.obj
 0001:00001800       ??_C@_19EPFLPGAP@?$AAJ?$AAu?$AAn?$AAe?$AA?$AA@ 10002800     libucrt:nlsdata.obj
 0001:0000180c       ??_C@_19BIFMLPCD@?$AAJ?$AAu?$AAl?$AAy?$AA?$AA@ 1000280c     libucrt:nlsdata.obj
 0001:00001818       ??_C@_1O@PAHLKOAC@?$AAA?$AAu?$AAg?$AAu?$AAs?$AAt?$AA?$AA@ 10002818     libucrt:nlsdata.obj
 0001:00001828       ??_C@_1BE@DKAAMBJL@?$AAS?$AAe?$AAp?$AAt?$AAe?$AAm?$AAb?$AAe?$AAr?$AA?$AA@ 10002828     libucrt:nlsdata.obj
 0001:0000183c       ??_C@_1BA@EPANDLNG@?$AAO?$AAc?$AAt?$AAo?$AAb?$AAe?$AAr?$AA?$AA@ 1000283c     libucrt:nlsdata.obj
 0001:0000184c       ??_C@_1BC@BGLIFPF@?$AAN?$AAo?$AAv?$AAe?$AAm?$AAb?$AAe?$AAr?$AA?$AA@ 1000284c     libucrt:nlsdata.obj
 0001:00001860       ??_C@_1BC@FEMKIFH@?$AAD?$AAe?$AAc?$AAe?$AAm?$AAb?$AAe?$AAr?$AA?$AA@ 10002860     libucrt:nlsdata.obj
 0001:00001874       ??_C@_15ODEHAHHF@?$AAA?$AAM?$AA?$AA@ 10002874     libucrt:nlsdata.obj
 0001:0000187c       ??_C@_15CLMNNGEL@?$AAP?$AAM?$AA?$AA@ 1000287c     libucrt:nlsdata.obj
 0001:00001884       ??_C@_1BC@IEBCMHCM@?$AAM?$AAM?$AA?1?$AAd?$AAd?$AA?1?$AAy?$AAy?$AA?$AA@ 10002884     libucrt:nlsdata.obj
 0001:00001898       ??_C@_1CI@KNAKOEBC@?$AAd?$AAd?$AAd?$AAd?$AA?0?$AA?5?$AAM?$AAM?$AAM?$AAM?$AA?5?$AAd?$AAd?$AA?0?$AA?5?$AAy?$AAy?$AAy?$AAy?$AA?$AA@ 10002898     libucrt:nlsdata.obj
 0001:000018c0       ??_C@_1BC@GDGBMEMK@?$AAH?$AAH?$AA?3?$AAm?$AAm?$AA?3?$AAs?$AAs?$AA?$AA@ 100028c0     libucrt:nlsdata.obj
 0001:000018d4       ??_C@_1M@BMHNFIME@?$AAe?$AAn?$AA?9?$AAU?$AAS?$AA?$AA@ 100028d4     libucrt:nlsdata.obj
 0001:000018e0       ___newctype                100028e0     libucrt:ctype.obj
 0001:00001be0       ___newclmap                10002be0     libucrt:ctype.obj
 0001:00001d60       ___newcumap                10002d60     libucrt:ctype.obj
 0001:00002600       ??_C@_15EMKDOKLE@?$AAa?$AAr?$AA?$AA@ 10003600     libucrt:lcidtoname_downlevel.obj
 0001:00002608       ??_C@_15KNPADPLH@?$AAb?$AAg?$AA?$AA@ 10003608     libucrt:lcidtoname_downlevel.obj
 0001:00002610       ??_C@_15EDMHLDMO@?$AAc?$AAa?$AA?$AA@ 10003610     libucrt:lcidtoname_downlevel.obj
 0001:00002618       ??_C@_1O@BPEAJADD@?$AAz?$AAh?$AA?9?$AAC?$AAH?$AAS?$AA?$AA@ 10003618     libucrt:lcidtoname_downlevel.obj
 0001:00002628       ??_C@_15LJNHCMNK@?$AAc?$AAs?$AA?$AA@ 10003628     libucrt:lcidtoname_downlevel.obj
 0001:00002630       ??_C@_15FOMCIDHG@?$AAd?$AAa?$AA?$AA@ 10003630     libucrt:lcidtoname_downlevel.obj
 0001:00002638       ??_C@_15NBKABECB@?$AAd?$AAe?$AA?$AA@ 10003638     libucrt:lcidtoname_downlevel.obj
 0001:00002640       ??_C@_15GHPEIIAO@?$AAe?$AAl?$AA?$AA@ 10003640     libucrt:lcidtoname_downlevel.obj
 0001:00002648       ??_C@_15MNPNEAIF@?$AAe?$AAn?$AA?$AA@ 10003648     libucrt:lcidtoname_downlevel.obj
 0001:00002650       ??_C@_15GPIOMPMH@?$AAe?$AAs?$AA?$AA@ 10003650     libucrt:lcidtoname_downlevel.obj
 0001:00002658       ??_C@_15NGLOAKJC@?$AAf?$AAi?$AA?$AA@ 10003658     libucrt:lcidtoname_downlevel.obj
 0001:00002660       ??_C@_15FBKGNKAM@?$AAf?$AAr?$AA?$AA@ 10003660     libucrt:lcidtoname_downlevel.obj
 0001:00002668       ??_C@_15KGGCNEFK@?$AAh?$AAe?$AA?$AA@ 10003668     libucrt:lcidtoname_downlevel.obj
 0001:00002670       ??_C@_15PGHLIDMF@?$AAh?$AAu?$AA?$AA@ 10003670     libucrt:lcidtoname_downlevel.obj
 0001:00002678       ??_C@_15BIEMAPLM@?$AAi?$AAs?$AA?$AA@ 10003678     libucrt:lcidtoname_downlevel.obj
 0001:00002680       ??_C@_15IFJLDHAF@?$AAi?$AAt?$AA?$AA@ 10003680     libucrt:lcidtoname_downlevel.obj
 0001:00002688       ??_C@_15GEMIOCAG@?$AAj?$AAa?$AA?$AA@ 10003688     libucrt:lcidtoname_downlevel.obj
 0001:00002690       ??_C@_15EPELEGJA@?$AAk?$AAo?$AA?$AA@ 10003690     libucrt:lcidtoname_downlevel.obj
 0001:00002698       ??_C@_15NDDHIMN@?$AAn?$AAl?$AA?$AA@ 10003698     libucrt:lcidtoname_downlevel.obj
 0001:000026a0       ??_C@_15BPIGNHCD@?$AAn?$AAo?$AA?$AA@ 100036a0     libucrt:lcidtoname_downlevel.obj
 0001:000026a8       ??_C@_15DEOPBLCG@?$AAp?$AAl?$AA?$AA@ 100036a8     libucrt:lcidtoname_downlevel.obj
 0001:000026b0       ??_C@_15KBECGEFG@?$AAp?$AAt?$AA?$AA@ 100036b0     libucrt:lcidtoname_downlevel.obj
 0001:000026b8       ??_C@_15GLJCBFMD@?$AAr?$AAo?$AA?$AA@ 100036b8     libucrt:lcidtoname_downlevel.obj
 0001:000026c0       ??_C@_15FEDGKCDI@?$AAr?$AAu?$AA?$AA@ 100036c0     libucrt:lcidtoname_downlevel.obj
 0001:000026c8       ??_C@_15GLKMLLHM@?$AAh?$AAr?$AA?$AA@ 100036c8     libucrt:lcidtoname_downlevel.obj
 0001:000026d0       ??_C@_15CPKMFBDB@?$AAs?$AAk?$AA?$AA@ 100036d0     libucrt:lcidtoname_downlevel.obj
 0001:000026d8       ??_C@_15BAAIOGMK@?$AAs?$AAq?$AA?$AA@ 100036d8     libucrt:lcidtoname_downlevel.obj
 0001:000026e0       ??_C@_15INNPNOHD@?$AAs?$AAv?$AA?$AA@ 100036e0     libucrt:lcidtoname_downlevel.obj
 0001:000026e8       ??_C@_15CABMMOGH@?$AAt?$AAh?$AA?$AA@ 100036e8     libucrt:lcidtoname_downlevel.obj
 0001:000026f0       ??_C@_15BPLIHJJM@?$AAt?$AAr?$AA?$AA@ 100036f0     libucrt:lcidtoname_downlevel.obj
 0001:000026f8       ??_C@_15NEOEKKDJ@?$AAu?$AAr?$AA?$AA@ 100036f8     libucrt:lcidtoname_downlevel.obj
 0001:00002700       ??_C@_15NFICGAJK@?$AAi?$AAd?$AA?$AA@ 10003700     libucrt:lcidtoname_downlevel.obj
 0001:00002708       ??_C@_15PJPFLCCM@?$AAu?$AAk?$AA?$AA@ 10003708     libucrt:lcidtoname_downlevel.obj
 0001:00002710       ??_C@_15HPJPHDM@?$AAb?$AAe?$AA?$AA@ 10003710     libucrt:lcidtoname_downlevel.obj
 0001:00002718       ??_C@_15LCHLGJII@?$AAs?$AAl?$AA?$AA@ 10003718     libucrt:lcidtoname_downlevel.obj
 0001:00002720       ??_C@_15PCFJPHHO@?$AAe?$AAt?$AA?$AA@ 10003720     libucrt:lcidtoname_downlevel.obj
 0001:00002728       ??_C@_15HPFPGODN@?$AAl?$AAv?$AA?$AA@ 10003728     libucrt:lcidtoname_downlevel.obj
 0001:00002730       ??_C@_15NFFGKGLG@?$AAl?$AAt?$AA?$AA@ 10003730     libucrt:lcidtoname_downlevel.obj
 0001:00002738       ??_C@_15BDAKCCHN@?$AAf?$AAa?$AA?$AA@ 10003738     libucrt:lcidtoname_downlevel.obj
 0001:00002740       ??_C@_15NFGIAIAJ@?$AAv?$AAi?$AA?$AA@ 10003740     libucrt:lcidtoname_downlevel.obj
 0001:00002748       ??_C@_15LMKNDMHN@?$AAh?$AAy?$AA?$AA@ 10003748     libucrt:lcidtoname_downlevel.obj
 0001:00002750       ??_C@_15IJBHMCFL@?$AAa?$AAz?$AA?$AA@ 10003750     libucrt:lcidtoname_downlevel.obj
 0001:00002758       ??_C@_15EKOFJABL@?$AAe?$AAu?$AA?$AA@ 10003758     libucrt:lcidtoname_downlevel.obj
 0001:00002760       ??_C@_15BGHADCNK@?$AAm?$AAk?$AA?$AA@ 10003760     libucrt:lcidtoname_downlevel.obj
 0001:00002768       ??_C@_15JDNICKHM@?$AAa?$AAf?$AA?$AA@ 10003768     libucrt:lcidtoname_downlevel.obj
 0001:00002770       ??_C@_15KPJEDBKD@?$AAk?$AAa?$AA?$AA@ 10003770     libucrt:lcidtoname_downlevel.obj
 0001:00002778       ??_C@_15PDNFFFEO@?$AAf?$AAo?$AA?$AA@ 10003778     libucrt:lcidtoname_downlevel.obj
 0001:00002780       ??_C@_15OMLEGLOC@?$AAh?$AAi?$AA?$AA@ 10003780     libucrt:lcidtoname_downlevel.obj
 0001:00002788       ??_C@_15IDNNENKK@?$AAm?$AAs?$AA?$AA@ 10003788     libucrt:lcidtoname_downlevel.obj
 0001:00002790       ??_C@_15MACJNBMH@?$AAk?$AAk?$AA?$AA@ 10003790     libucrt:lcidtoname_downlevel.obj
 0001:00002798       ??_C@_15DKDJEOND@?$AAk?$AAy?$AA?$AA@ 10003798     libucrt:lcidtoname_downlevel.obj
 0001:000027a0       ??_C@_15DFGDLJBG@?$AAs?$AAw?$AA?$AA@ 100037a0     libucrt:lcidtoname_downlevel.obj
 0001:000027a8       ??_C@_15BBFAICNG@?$AAu?$AAz?$AA?$AA@ 100037a8     libucrt:lcidtoname_downlevel.obj
 0001:000027b0       ??_C@_15DKNDCGEA@?$AAt?$AAt?$AA?$AA@ 100037b0     libucrt:lcidtoname_downlevel.obj
 0001:000027b8       ??_C@_15MGIFMDPL@?$AAp?$AAa?$AA?$AA@ 100037b8     libucrt:lcidtoname_downlevel.obj
 0001:000027c0       ??_C@_15HCNDBBA@?$AAg?$AAu?$AA?$AA@ 100037c0     libucrt:lcidtoname_downlevel.obj
 0001:000027c8       ??_C@_15FNBEIBON@?$AAt?$AAa?$AA?$AA@ 100037c8     libucrt:lcidtoname_downlevel.obj
 0001:000027d0       ??_C@_15NCHGBGLK@?$AAt?$AAe?$AA?$AA@ 100037d0     libucrt:lcidtoname_downlevel.obj
 0001:000027d8       ??_C@_15PHPHCBPF@?$AAk?$AAn?$AA?$AA@ 100037d8     libucrt:lcidtoname_downlevel.obj
 0001:000027e0       ??_C@_15DLGBCKMP@?$AAm?$AAr?$AA?$AA@ 100037e0     libucrt:lcidtoname_downlevel.obj
 0001:000027e8       ??_C@_15EABBLBFF@?$AAs?$AAa?$AA?$AA@ 100037e8     libucrt:lcidtoname_downlevel.obj
 0001:000027f0       ??_C@_15CBKOMCOI@?$AAm?$AAn?$AA?$AA@ 100037f0     libucrt:lcidtoname_downlevel.obj
 0001:000027f8       ??_C@_15CKDMCJAF@?$AAg?$AAl?$AA?$AA@ 100037f8     libucrt:lcidtoname_downlevel.obj
 0001:00002800       ??_C@_17CNJFBPG@?$AAk?$AAo?$AAk?$AA?$AA@ 10003800     libucrt:lcidtoname_downlevel.obj
 0001:00002808       ??_C@_17FFBJICPL@?$AAs?$AAy?$AAr?$AA?$AA@ 10003808     libucrt:lcidtoname_downlevel.obj
 0001:00002810       ??_C@_17KPNDCPAF@?$AAd?$AAi?$AAv?$AA?$AA@ 10003810     libucrt:lcidtoname_downlevel.obj
 0001:00002818       ??_C@_11LOCGONAA@?$AA?$AA@ 10003818     libucrt:lcidtoname_downlevel.obj
 0001:0000281c       ??_C@_1M@OKAHONE@?$AAa?$AAr?$AA?9?$AAS?$AAA?$AA?$AA@ 1000381c     libucrt:lcidtoname_downlevel.obj
 0001:00002828       ??_C@_1M@FFFIGIGK@?$AAb?$AAg?$AA?9?$AAB?$AAG?$AA?$AA@ 10003828     libucrt:lcidtoname_downlevel.obj
 0001:00002834       ??_C@_1M@BJNKEDC@?$AAc?$AAa?$AA?9?$AAE?$AAS?$AA?$AA@ 10003834     libucrt:lcidtoname_downlevel.obj
 0001:00002840       ??_C@_1M@IJJHFJHA@?$AAc?$AAs?$AA?9?$AAC?$AAZ?$AA?$AA@ 10003840     libucrt:lcidtoname_downlevel.obj
 0001:0000284c       ??_C@_1M@CLPEOBGI@?$AAd?$AAa?$AA?9?$AAD?$AAK?$AA?$AA@ 1000384c     libucrt:lcidtoname_downlevel.obj
 0001:00002858       ??_C@_1M@MCMADGCB@?$AAd?$AAe?$AA?9?$AAD?$AAE?$AA?$AA@ 10003858     libucrt:lcidtoname_downlevel.obj
 0001:00002864       ??_C@_1M@OOCKEMAM@?$AAe?$AAl?$AA?9?$AAG?$AAR?$AA?$AA@ 10003864     libucrt:lcidtoname_downlevel.obj
 0001:00002870       ??_C@_1M@DDNJFGID@?$AAf?$AAi?$AA?9?$AAF?$AAI?$AA?$AA@ 10003870     libucrt:lcidtoname_downlevel.obj
 0001:0000287c       ??_C@_1M@GLIPPMAC@?$AAf?$AAr?$AA?9?$AAF?$AAR?$AA?$AA@ 1000387c     libucrt:lcidtoname_downlevel.obj
 0001:00002888       ??_C@_1M@GFMCHPE@?$AAh?$AAe?$AA?9?$AAI?$AAL?$AA?$AA@ 10003888     libucrt:lcidtoname_downlevel.obj
 0001:00002894       ??_C@_1M@MHLPGNKM@?$AAh?$AAu?$AA?9?$AAH?$AAU?$AA?$AA@ 10003894     libucrt:lcidtoname_downlevel.obj
 0001:000028a0       ??_C@_1M@LPDDNNPN@?$AAi?$AAs?$AA?9?$AAI?$AAS?$AA?$AA@ 100038a0     libucrt:lcidtoname_downlevel.obj
 0001:000028ac       ??_C@_1M@MADIPODN@?$AAi?$AAt?$AA?9?$AAI?$AAT?$AA?$AA@ 100038ac     libucrt:lcidtoname_downlevel.obj
 0001:000028b8       ??_C@_1M@IHBJJGG@?$AAn?$AAl?$AA?9?$AAN?$AAL?$AA?$AA@ 100038b8     libucrt:lcidtoname_downlevel.obj
 0001:000028c4       ??_C@_1M@EANAGDL@?$AAn?$AAb?$AA?9?$AAN?$AAO?$AA?$AA@ 100038c4     libucrt:lcidtoname_downlevel.obj
 0001:000028d0       ??_C@_1M@NEIEMEGP@?$AAp?$AAl?$AA?9?$AAP?$AAL?$AA?$AA@ 100038d0     libucrt:lcidtoname_downlevel.obj
 0001:000028dc       ??_C@_1M@BOCFIGEP@?$AAp?$AAt?$AA?9?$AAB?$AAR?$AA?$AA@ 100038dc     libucrt:lcidtoname_downlevel.obj
 0001:000028e8       ??_C@_1M@IMPFOPBG@?$AAr?$AAo?$AA?9?$AAR?$AAO?$AA?$AA@ 100038e8     libucrt:lcidtoname_downlevel.obj
 0001:000028f4       ??_C@_1M@IDNNEJMM@?$AAr?$AAu?$AA?9?$AAR?$AAU?$AA?$AA@ 100038f4     libucrt:lcidtoname_downlevel.obj
 0001:00002900       ??_C@_1M@LILEEOGM@?$AAh?$AAr?$AA?9?$AAH?$AAR?$AA?$AA@ 10003900     libucrt:lcidtoname_downlevel.obj
 0001:0000290c       ??_C@_1M@FKIFEHPB@?$AAs?$AAk?$AA?9?$AAS?$AAK?$AA?$AA@ 1000390c     libucrt:lcidtoname_downlevel.obj
 0001:00002918       ??_C@_1M@LJMAMNPJ@?$AAs?$AAq?$AA?9?$AAA?$AAL?$AA?$AA@ 10003918     libucrt:lcidtoname_downlevel.obj
 0001:00002924       ??_C@_1M@GIAKDKJK@?$AAs?$AAv?$AA?9?$AAS?$AAE?$AA?$AA@ 10003924     libucrt:lcidtoname_downlevel.obj
 0001:00002930       ??_C@_1M@MKJKIKCL@?$AAt?$AAh?$AA?9?$AAT?$AAH?$AA?$AA@ 10003930     libucrt:lcidtoname_downlevel.obj
 0001:0000293c       ??_C@_1M@MFLCCMPB@?$AAt?$AAr?$AA?9?$AAT?$AAR?$AA?$AA@ 1000393c     libucrt:lcidtoname_downlevel.obj
 0001:00002948       ??_C@_1M@OIJHDKJN@?$AAu?$AAr?$AA?9?$AAP?$AAK?$AA?$AA@ 10003948     libucrt:lcidtoname_downlevel.obj
 0001:00002954       ??_C@_1M@LHIPCIEK@?$AAi?$AAd?$AA?9?$AAI?$AAD?$AA?$AA@ 10003954     libucrt:lcidtoname_downlevel.obj
 0001:00002960       ??_C@_1M@MFMOBGI@?$AAu?$AAk?$AA?9?$AAU?$AAA?$AA?$AA@ 10003960     libucrt:lcidtoname_downlevel.obj
 0001:0000296c       ??_C@_1M@OBGLJIPL@?$AAb?$AAe?$AA?9?$AAB?$AAY?$AA?$AA@ 1000396c     libucrt:lcidtoname_downlevel.obj
 0001:00002978       ??_C@_1M@BCFAJEAD@?$AAs?$AAl?$AA?9?$AAS?$AAI?$AA?$AA@ 10003978     libucrt:lcidtoname_downlevel.obj
 0001:00002984       ??_C@_1M@FKFFEDDN@?$AAe?$AAt?$AA?9?$AAE?$AAE?$AA?$AA@ 10003984     libucrt:lcidtoname_downlevel.obj
 0001:00002990       ??_C@_1M@KGKKAACI@?$AAl?$AAv?$AA?9?$AAL?$AAV?$AA?$AA@ 10003990     libucrt:lcidtoname_downlevel.obj
 0001:0000299c       ??_C@_1M@IFGBIJO@?$AAl?$AAt?$AA?9?$AAL?$AAT?$AA?$AA@ 1000399c     libucrt:lcidtoname_downlevel.obj
 0001:000029a8       ??_C@_1M@FGEAHEDM@?$AAf?$AAa?$AA?9?$AAI?$AAR?$AA?$AA@ 100039a8     libucrt:lcidtoname_downlevel.obj
 0001:000029b4       ??_C@_1M@KBMAIBFN@?$AAv?$AAi?$AA?9?$AAV?$AAN?$AA?$AA@ 100039b4     libucrt:lcidtoname_downlevel.obj
 0001:000029c0       ??_C@_1M@GPCBKDJK@?$AAh?$AAy?$AA?9?$AAA?$AAM?$AA?$AA@ 100039c0     libucrt:lcidtoname_downlevel.obj
 0001:000029cc       ??_C@_1BG@BECMDDJB@?$AAa?$AAz?$AA?9?$AAA?$AAZ?$AA?9?$AAL?$AAa?$AAt?$AAn?$AA?$AA@ 100039cc     libucrt:lcidtoname_downlevel.obj
 0001:000029e4       ??_C@_1M@MAOFCAEA@?$AAe?$AAu?$AA?9?$AAE?$AAS?$AA?$AA@ 100039e4     libucrt:lcidtoname_downlevel.obj
 0001:000029f0       ??_C@_1M@IGHABKPI@?$AAm?$AAk?$AA?9?$AAM?$AAK?$AA?$AA@ 100039f0     libucrt:lcidtoname_downlevel.obj
 0001:000029fc       ??_C@_1M@IAIGNEJG@?$AAt?$AAn?$AA?9?$AAZ?$AAA?$AA?$AA@ 100039fc     libucrt:lcidtoname_downlevel.obj
 0001:00002a08       ??_C@_1M@IIJCOJFA@?$AAx?$AAh?$AA?9?$AAZ?$AAA?$AA?$AA@ 10003a08     libucrt:lcidtoname_downlevel.obj
 0001:00002a14       ??_C@_1M@LGPJHNJH@?$AAz?$AAu?$AA?9?$AAZ?$AAA?$AA?$AA@ 10003a14     libucrt:lcidtoname_downlevel.obj
 0001:00002a20       ??_C@_1M@HOKAOIO@?$AAa?$AAf?$AA?9?$AAZ?$AAA?$AA?$AA@ 10003a20     libucrt:lcidtoname_downlevel.obj
 0001:00002a2c       ??_C@_1M@DPCLHLIE@?$AAk?$AAa?$AA?9?$AAG?$AAE?$AA?$AA@ 10003a2c     libucrt:lcidtoname_downlevel.obj
 0001:00002a38       ??_C@_1M@BLKMHJBI@?$AAf?$AAo?$AA?9?$AAF?$AAO?$AA?$AA@ 10003a38     libucrt:lcidtoname_downlevel.obj
 0001:00002a44       ??_C@_1M@LGGJAPPB@?$AAh?$AAi?$AA?9?$AAI?$AAN?$AA?$AA@ 10003a44     libucrt:lcidtoname_downlevel.obj
 0001:00002a50       ??_C@_1M@FIKPIHFE@?$AAm?$AAt?$AA?9?$AAM?$AAT?$AA?$AA@ 10003a50     libucrt:lcidtoname_downlevel.obj
 0001:00002a5c       ??_C@_1M@HEGGPBFA@?$AAs?$AAe?$AA?9?$AAN?$AAO?$AA?$AA@ 10003a5c     libucrt:lcidtoname_downlevel.obj
 0001:00002a68       ??_C@_1M@EIBJEEPA@?$AAm?$AAs?$AA?9?$AAM?$AAY?$AA?$AA@ 10003a68     libucrt:lcidtoname_downlevel.obj
 0001:00002a74       ??_C@_1M@FHLBGMPP@?$AAk?$AAk?$AA?9?$AAK?$AAZ?$AA?$AA@ 10003a74     libucrt:lcidtoname_downlevel.obj
 0001:00002a80       ??_C@_1M@NGJJLCGI@?$AAk?$AAy?$AA?9?$AAK?$AAG?$AA?$AA@ 10003a80     libucrt:lcidtoname_downlevel.obj
 0001:00002a8c       ??_C@_1M@GIENNBFC@?$AAs?$AAw?$AA?9?$AAK?$AAE?$AA?$AA@ 10003a8c     libucrt:lcidtoname_downlevel.obj
 0001:00002a98       ??_C@_1BG@NDGMJIMJ@?$AAu?$AAz?$AA?9?$AAU?$AAZ?$AA?9?$AAL?$AAa?$AAt?$AAn?$AA?$AA@ 10003a98     libucrt:lcidtoname_downlevel.obj
 0001:00002ab0       ??_C@_1M@IDCCIHBC@?$AAt?$AAt?$AA?9?$AAR?$AAU?$AA?$AA@ 10003ab0     libucrt:lcidtoname_downlevel.obj
 0001:00002abc       ??_C@_1M@LOICPMOJ@?$AAb?$AAn?$AA?9?$AAI?$AAN?$AA?$AA@ 10003abc     libucrt:lcidtoname_downlevel.obj
 0001:00002ac8       ??_C@_1M@KPKKNEAH@?$AAp?$AAa?$AA?9?$AAI?$AAN?$AA?$AA@ 10003ac8     libucrt:lcidtoname_downlevel.obj
 0001:00002ad4       ??_C@_1M@PJGPPBOG@?$AAg?$AAu?$AA?9?$AAI?$AAN?$AA?$AA@ 10003ad4     libucrt:lcidtoname_downlevel.obj
 0001:00002ae0       ??_C@_1M@KMKMOPHI@?$AAt?$AAa?$AA?9?$AAI?$AAN?$AA?$AA@ 10003ae0     libucrt:lcidtoname_downlevel.obj
 0001:00002aec       ??_C@_1M@KFEHEPAC@?$AAt?$AAe?$AA?9?$AAI?$AAN?$AA?$AA@ 10003aec     libucrt:lcidtoname_downlevel.obj
 0001:00002af8       ??_C@_1M@CDCLMGHI@?$AAk?$AAn?$AA?9?$AAI?$AAN?$AA?$AA@ 10003af8     libucrt:lcidtoname_downlevel.obj
 0001:00002b04       ??_C@_1M@MIODLDKF@?$AAm?$AAl?$AA?9?$AAI?$AAN?$AA?$AA@ 10003b04     libucrt:lcidtoname_downlevel.obj
 0001:00002b10       ??_C@_1M@PBIEACPO@?$AAm?$AAr?$AA?9?$AAI?$AAN?$AA?$AA@ 10003b10     libucrt:lcidtoname_downlevel.obj
 0001:00002b1c       ??_C@_1M@NIDEAGPH@?$AAs?$AAa?$AA?9?$AAI?$AAN?$AA?$AA@ 10003b1c     libucrt:lcidtoname_downlevel.obj
 0001:00002b28       ??_C@_1M@FHIHCBIO@?$AAm?$AAn?$AA?9?$AAM?$AAN?$AA?$AA@ 10003b28     libucrt:lcidtoname_downlevel.obj
 0001:00002b34       ??_C@_1M@JAIJPENP@?$AAc?$AAy?$AA?9?$AAG?$AAB?$AA?$AA@ 10003b34     libucrt:lcidtoname_downlevel.obj
 0001:00002b40       ??_C@_1M@PHGFBEPN@?$AAg?$AAl?$AA?9?$AAE?$AAS?$AA?$AA@ 10003b40     libucrt:lcidtoname_downlevel.obj
 0001:00002b4c       ??_C@_1O@KPIPDNCP@?$AAk?$AAo?$AAk?$AA?9?$AAI?$AAN?$AA?$AA@ 10003b4c     libucrt:lcidtoname_downlevel.obj
 0001:00002b5c       ??_C@_1O@KNHJLDJA@?$AAs?$AAy?$AAr?$AA?9?$AAS?$AAY?$AA?$AA@ 10003b5c     libucrt:lcidtoname_downlevel.obj
 0001:00002b6c       ??_C@_1O@MKEKBLAH@?$AAd?$AAi?$AAv?$AA?9?$AAM?$AAV?$AA?$AA@ 10003b6c     libucrt:lcidtoname_downlevel.obj
 0001:00002b7c       ??_C@_1O@OHDCKDDF@?$AAq?$AAu?$AAz?$AA?9?$AAB?$AAO?$AA?$AA@ 10003b7c     libucrt:lcidtoname_downlevel.obj
 0001:00002b8c       ??_C@_1M@LEPJNLFD@?$AAn?$AAs?$AA?9?$AAZ?$AAA?$AA?$AA@ 10003b8c     libucrt:lcidtoname_downlevel.obj
 0001:00002b98       ??_C@_1M@OMLEIIJB@?$AAm?$AAi?$AA?9?$AAN?$AAZ?$AA?$AA@ 10003b98     libucrt:lcidtoname_downlevel.obj
 0001:00002ba4       ??_C@_1M@PMPEAILG@?$AAa?$AAr?$AA?9?$AAI?$AAQ?$AA?$AA@ 10003ba4     libucrt:lcidtoname_downlevel.obj
 0001:00002bb0       ??_C@_1M@CNKPNOEE@?$AAd?$AAe?$AA?9?$AAC?$AAH?$AA?$AA@ 10003bb0     libucrt:lcidtoname_downlevel.obj
 0001:00002bbc       ??_C@_1M@LKMGMLKO@?$AAe?$AAn?$AA?9?$AAG?$AAB?$AA?$AA@ 10003bbc     libucrt:lcidtoname_downlevel.obj
 0001:00002bc8       ??_C@_1M@PGKJFFGL@?$AAe?$AAs?$AA?9?$AAM?$AAX?$AA?$AA@ 10003bc8     libucrt:lcidtoname_downlevel.obj
 0001:00002bd4       ??_C@_1M@DNNANBDC@?$AAf?$AAr?$AA?9?$AAB?$AAE?$AA?$AA@ 10003bd4     libucrt:lcidtoname_downlevel.obj
 0001:00002be0       ??_C@_1M@HLGMDFHM@?$AAi?$AAt?$AA?9?$AAC?$AAH?$AA?$AA@ 10003be0     libucrt:lcidtoname_downlevel.obj
 0001:00002bec       ??_C@_1M@CLLBGJH@?$AAn?$AAl?$AA?9?$AAB?$AAE?$AA?$AA@ 10003bec     libucrt:lcidtoname_downlevel.obj
 0001:00002bf8       ??_C@_1M@BODBOGLF@?$AAn?$AAn?$AA?9?$AAN?$AAO?$AA?$AA@ 10003bf8     libucrt:lcidtoname_downlevel.obj
 0001:00002c04       ??_C@_1M@HFFAHKAD@?$AAp?$AAt?$AA?9?$AAP?$AAT?$AA?$AA@ 10003c04     libucrt:lcidtoname_downlevel.obj
 0001:00002c10       ??_C@_1BG@LNOAKHIE@?$AAs?$AAr?$AA?9?$AAS?$AAP?$AA?9?$AAL?$AAa?$AAt?$AAn?$AA?$AA@ 10003c10     libucrt:lcidtoname_downlevel.obj
 0001:00002c28       ??_C@_1M@HBMHBGAK@?$AAs?$AAv?$AA?9?$AAF?$AAI?$AA?$AA@ 10003c28     libucrt:lcidtoname_downlevel.obj
 0001:00002c34       ??_C@_1BG@DGCJGJBE@?$AAa?$AAz?$AA?9?$AAA?$AAZ?$AA?9?$AAC?$AAy?$AAr?$AAl?$AA?$AA@ 10003c34     libucrt:lcidtoname_downlevel.obj
 0001:00002c4c       ??_C@_1M@KEJDAAHB@?$AAs?$AAe?$AA?9?$AAS?$AAE?$AA?$AA@ 10003c4c     libucrt:lcidtoname_downlevel.obj
 0001:00002c58       ??_C@_1M@HEIBJJAD@?$AAm?$AAs?$AA?9?$AAB?$AAN?$AA?$AA@ 10003c58     libucrt:lcidtoname_downlevel.obj
 0001:00002c64       ??_C@_1BG@PBGJMCEM@?$AAu?$AAz?$AA?9?$AAU?$AAZ?$AA?9?$AAC?$AAy?$AAr?$AAl?$AA?$AA@ 10003c64     libucrt:lcidtoname_downlevel.obj
 0001:00002c7c       ??_C@_1O@LAOBCMDF@?$AAq?$AAu?$AAz?$AA?9?$AAE?$AAC?$AA?$AA@ 10003c7c     libucrt:lcidtoname_downlevel.obj
 0001:00002c8c       ??_C@_1M@POEEMAIO@?$AAa?$AAr?$AA?9?$AAE?$AAG?$AA?$AA@ 10003c8c     libucrt:lcidtoname_downlevel.obj
 0001:00002c98       ??_C@_1M@EFAKDEDL@?$AAz?$AAh?$AA?9?$AAH?$AAK?$AA?$AA@ 10003c98     libucrt:lcidtoname_downlevel.obj
 0001:00002ca4       ??_C@_1M@HKKIJHGI@?$AAd?$AAe?$AA?9?$AAA?$AAT?$AA?$AA@ 10003ca4     libucrt:lcidtoname_downlevel.obj
 0001:00002cb0       ??_C@_1M@KBFBEHJF@?$AAe?$AAn?$AA?9?$AAA?$AAU?$AA?$AA@ 10003cb0     libucrt:lcidtoname_downlevel.obj
 0001:00002cbc       ??_C@_1M@MNPLFAAH@?$AAe?$AAs?$AA?9?$AAE?$AAS?$AA?$AA@ 10003cbc     libucrt:lcidtoname_downlevel.obj
 0001:00002cc8       ??_C@_1M@HJOOJFMA@?$AAf?$AAr?$AA?9?$AAC?$AAA?$AA?$AA@ 10003cc8     libucrt:lcidtoname_downlevel.obj
 0001:00002cd4       ??_C@_1BG@JPOFPNAB@?$AAs?$AAr?$AA?9?$AAS?$AAP?$AA?9?$AAC?$AAy?$AAr?$AAl?$AA?$AA@ 10003cd4     libucrt:lcidtoname_downlevel.obj
 0001:00002cec       ??_C@_1M@LNFOCMOB@?$AAs?$AAe?$AA?9?$AAF?$AAI?$AA?$AA@ 10003cec     libucrt:lcidtoname_downlevel.obj
 0001:00002cf8       ??_C@_1O@MGJBOAMB@?$AAq?$AAu?$AAz?$AA?9?$AAP?$AAE?$AA?$AA@ 10003cf8     libucrt:lcidtoname_downlevel.obj
 0001:00002d08       ??_C@_1M@GJINLBOK@?$AAa?$AAr?$AA?9?$AAL?$AAY?$AA?$AA@ 10003d08     libucrt:lcidtoname_downlevel.obj
 0001:00002d14       ??_C@_1M@GGMNHJNL@?$AAz?$AAh?$AA?9?$AAS?$AAG?$AA?$AA@ 10003d14     libucrt:lcidtoname_downlevel.obj
 0001:00002d20       ??_C@_1M@HOIKODND@?$AAd?$AAe?$AA?9?$AAL?$AAU?$AA?$AA@ 10003d20     libucrt:lcidtoname_downlevel.obj
 0001:00002d2c       ??_C@_1M@DDOCCGFG@?$AAe?$AAn?$AA?9?$AAC?$AAA?$AA?$AA@ 10003d2c     libucrt:lcidtoname_downlevel.obj
 0001:00002d38       ??_C@_1M@BNOEMJLF@?$AAe?$AAs?$AA?9?$AAG?$AAT?$AA?$AA@ 10003d38     libucrt:lcidtoname_downlevel.obj
 0001:00002d44       ??_C@_1M@EOGNKEK@?$AAf?$AAr?$AA?9?$AAC?$AAH?$AA?$AA@ 10003d44     libucrt:lcidtoname_downlevel.obj
 0001:00002d50       ??_C@_1M@FLIDJFHL@?$AAh?$AAr?$AA?9?$AAB?$AAA?$AA?$AA@ 10003d50     libucrt:lcidtoname_downlevel.obj
 0001:00002d5c       ??_C@_1O@FMCELNAJ@?$AAs?$AAm?$AAj?$AA?9?$AAN?$AAO?$AA?$AA@ 10003d5c     libucrt:lcidtoname_downlevel.obj
 0001:00002d6c       ??_C@_1M@JHGLJMGJ@?$AAa?$AAr?$AA?9?$AAD?$AAZ?$AA?$AA@ 10003d6c     libucrt:lcidtoname_downlevel.obj
 0001:00002d78       ??_C@_1M@JKKFDCNP@?$AAz?$AAh?$AA?9?$AAM?$AAO?$AA?$AA@ 10003d78     libucrt:lcidtoname_downlevel.obj
 0001:00002d84       ??_C@_1M@GEEFALPE@?$AAd?$AAe?$AA?9?$AAL?$AAI?$AA?$AA@ 10003d84     libucrt:lcidtoname_downlevel.obj
 0001:00002d90       ??_C@_1M@IGEOFBG@?$AAe?$AAn?$AA?9?$AAN?$AAZ?$AA?$AA@ 10003d90     libucrt:lcidtoname_downlevel.obj
 0001:00002d9c       ??_C@_1M@KDBONEHP@?$AAe?$AAs?$AA?9?$AAC?$AAR?$AA?$AA@ 10003d9c     libucrt:lcidtoname_downlevel.obj
 0001:00002da8       ??_C@_1M@FHMDOHNN@?$AAf?$AAr?$AA?9?$AAL?$AAU?$AA?$AA@ 10003da8     libucrt:lcidtoname_downlevel.obj
 0001:00002db4       ??_C@_1BG@NFKKMAFG@?$AAb?$AAs?$AA?9?$AAB?$AAA?$AA?9?$AAL?$AAa?$AAt?$AAn?$AA?$AA@ 10003db4     libucrt:lcidtoname_downlevel.obj
 0001:00002dcc       ??_C@_1O@IMNBEMCI@?$AAs?$AAm?$AAj?$AA?9?$AAS?$AAE?$AA?$AA@ 10003dcc     libucrt:lcidtoname_downlevel.obj
 0001:00002ddc       ??_C@_1M@DHHMBNDP@?$AAa?$AAr?$AA?9?$AAM?$AAA?$AA?$AA@ 10003ddc     libucrt:lcidtoname_downlevel.obj
 0001:00002de8       ??_C@_1M@BNBLJCGH@?$AAe?$AAn?$AA?9?$AAI?$AAE?$AA?$AA@ 10003de8     libucrt:lcidtoname_downlevel.obj
 0001:00002df4       ??_C@_1M@GEPAFMDL@?$AAe?$AAs?$AA?9?$AAP?$AAA?$AA?$AA@ 10003df4     libucrt:lcidtoname_downlevel.obj
 0001:00002e00       ??_C@_1M@OJONDMDL@?$AAf?$AAr?$AA?9?$AAM?$AAC?$AA?$AA@ 10003e00     libucrt:lcidtoname_downlevel.obj
 0001:00002e0c       ??_C@_1BG@OBCNFJB@?$AAs?$AAr?$AA?9?$AAB?$AAA?$AA?9?$AAL?$AAa?$AAt?$AAn?$AA?$AA@ 10003e0c     libucrt:lcidtoname_downlevel.obj
 0001:00002e24       ??_C@_1O@KEMEEGPO@?$AAs?$AAm?$AAa?$AA?9?$AAN?$AAO?$AA?$AA@ 10003e24     libucrt:lcidtoname_downlevel.obj
 0001:00002e34       ??_C@_1M@ELMGFODK@?$AAa?$AAr?$AA?9?$AAT?$AAN?$AA?$AA@ 10003e34     libucrt:lcidtoname_downlevel.obj
 0001:00002e40       ??_C@_1M@BHDLHFAF@?$AAe?$AAn?$AA?9?$AAZ?$AAA?$AA?$AA@ 10003e40     libucrt:lcidtoname_downlevel.obj
 0001:00002e4c       ??_C@_1M@BMGIGLIF@?$AAe?$AAs?$AA?9?$AAD?$AAO?$AA?$AA@ 10003e4c     libucrt:lcidtoname_downlevel.obj
 0001:00002e58       ??_C@_1BG@CMBHIPBE@?$AAs?$AAr?$AA?9?$AAB?$AAA?$AA?9?$AAC?$AAy?$AAr?$AAl?$AA?$AA@ 10003e58     libucrt:lcidtoname_downlevel.obj
 0001:00002e70       ??_C@_1O@HEDBLHNP@?$AAs?$AAm?$AAa?$AA?9?$AAS?$AAE?$AA?$AA@ 10003e70     libucrt:lcidtoname_downlevel.obj
 0001:00002e80       ??_C@_1M@DAGCADIM@?$AAa?$AAr?$AA?9?$AAO?$AAM?$AA?$AA@ 10003e80     libucrt:lcidtoname_downlevel.obj
 0001:00002e8c       ??_C@_1M@FODLMICG@?$AAe?$AAn?$AA?9?$AAJ?$AAM?$AA?$AA@ 10003e8c     libucrt:lcidtoname_downlevel.obj
 0001:00002e98       ??_C@_1M@DNMLCIHB@?$AAe?$AAs?$AA?9?$AAV?$AAE?$AA?$AA@ 10003e98     libucrt:lcidtoname_downlevel.obj
 0001:00002ea4       ??_C@_1O@EOKHMKJK@?$AAs?$AAm?$AAs?$AA?9?$AAF?$AAI?$AA?$AA@ 10003ea4     libucrt:lcidtoname_downlevel.obj
 0001:00002eb4       ??_C@_1M@CAFJMKOF@?$AAa?$AAr?$AA?9?$AAY?$AAE?$AA?$AA@ 10003eb4     libucrt:lcidtoname_downlevel.obj
 0001:00002ec0       ??_C@_1M@CBFHIJLI@?$AAe?$AAn?$AA?9?$AAC?$AAB?$AA?$AA@ 10003ec0     libucrt:lcidtoname_downlevel.obj
 0001:00002ecc       ??_C@_1M@BGNFLDN@?$AAe?$AAs?$AA?9?$AAC?$AAO?$AA?$AA@ 10003ecc     libucrt:lcidtoname_downlevel.obj
 0001:00002ed8       ??_C@_1O@JMPHMAMC@?$AAs?$AAm?$AAn?$AA?9?$AAF?$AAI?$AA?$AA@ 10003ed8     libucrt:lcidtoname_downlevel.obj
 0001:00002ee8       ??_C@_1M@JLANABKE@?$AAa?$AAr?$AA?9?$AAS?$AAY?$AA?$AA@ 10003ee8     libucrt:lcidtoname_downlevel.obj
 0001:00002ef4       ??_C@_1M@HPKGCFGN@?$AAe?$AAn?$AA?9?$AAB?$AAZ?$AA?$AA@ 10003ef4     libucrt:lcidtoname_downlevel.obj
 0001:00002f00       ??_C@_1M@OLJCMLGM@?$AAe?$AAs?$AA?9?$AAP?$AAE?$AA?$AA@ 10003f00     libucrt:lcidtoname_downlevel.obj
 0001:00002f0c       ??_C@_1M@MKKGFKLE@?$AAa?$AAr?$AA?9?$AAJ?$AAO?$AA?$AA@ 10003f0c     libucrt:lcidtoname_downlevel.obj
 0001:00002f18       ??_C@_1M@EKPGLDNI@?$AAe?$AAn?$AA?9?$AAT?$AAT?$AA?$AA@ 10003f18     libucrt:lcidtoname_downlevel.obj
 0001:00002f24       ??_C@_1M@OONGHFHE@?$AAe?$AAs?$AA?9?$AAA?$AAR?$AA?$AA@ 10003f24     libucrt:lcidtoname_downlevel.obj
 0001:00002f30       ??_C@_1M@OOJFGBHE@?$AAa?$AAr?$AA?9?$AAL?$AAB?$AA?$AA@ 10003f30     libucrt:lcidtoname_downlevel.obj
 0001:00002f3c       ??_C@_1M@GCEJHNEG@?$AAe?$AAn?$AA?9?$AAZ?$AAW?$AA?$AA@ 10003f3c     libucrt:lcidtoname_downlevel.obj
 0001:00002f48       ??_C@_1M@JNOCAHJI@?$AAe?$AAs?$AA?9?$AAE?$AAC?$AA?$AA@ 10003f48     libucrt:lcidtoname_downlevel.obj
 0001:00002f54       ??_C@_1M@JEFHPGGB@?$AAa?$AAr?$AA?9?$AAK?$AAW?$AA?$AA@ 10003f54     libucrt:lcidtoname_downlevel.obj
 0001:00002f60       ??_C@_1M@MLKIBJOJ@?$AAe?$AAn?$AA?9?$AAP?$AAH?$AA?$AA@ 10003f60     libucrt:lcidtoname_downlevel.obj
 0001:00002f6c       ??_C@_1M@BDNIPEND@?$AAe?$AAs?$AA?9?$AAC?$AAL?$AA?$AA@ 10003f6c     libucrt:lcidtoname_downlevel.obj
 0001:00002f78       ??_C@_1M@MPNMEKBD@?$AAa?$AAr?$AA?9?$AAA?$AAE?$AA?$AA@ 10003f78     libucrt:lcidtoname_downlevel.obj
 0001:00002f84       ??_C@_1M@KBJALCPI@?$AAe?$AAs?$AA?9?$AAU?$AAY?$AA?$AA@ 10003f84     libucrt:lcidtoname_downlevel.obj
 0001:00002f90       ??_C@_1M@LLCCOAGA@?$AAa?$AAr?$AA?9?$AAB?$AAH?$AA?$AA@ 10003f90     libucrt:lcidtoname_downlevel.obj
 0001:00002f9c       ??_C@_1M@PBFNCDEL@?$AAe?$AAs?$AA?9?$AAP?$AAY?$AA?$AA@ 10003f9c     libucrt:lcidtoname_downlevel.obj
 0001:00002fa8       ??_C@_1M@EDGINPNP@?$AAa?$AAr?$AA?9?$AAQ?$AAA?$AA?$AA@ 10003fa8     libucrt:lcidtoname_downlevel.obj
 0001:00002fb4       ??_C@_1M@MKDBIIJI@?$AAe?$AAs?$AA?9?$AAB?$AAO?$AA?$AA@ 10003fb4     libucrt:lcidtoname_downlevel.obj
 0001:00002fc0       ??_C@_1M@CPKKEBLD@?$AAe?$AAs?$AA?9?$AAS?$AAV?$AA?$AA@ 10003fc0     libucrt:lcidtoname_downlevel.obj
 0001:00002fcc       ??_C@_1M@NDBGMMJL@?$AAe?$AAs?$AA?9?$AAH?$AAN?$AA?$AA@ 10003fcc     libucrt:lcidtoname_downlevel.obj
 0001:00002fd8       ??_C@_1M@JIJIBHDP@?$AAe?$AAs?$AA?9?$AAN?$AAI?$AA?$AA@ 10003fd8     libucrt:lcidtoname_downlevel.obj
 0001:00002fe4       ??_C@_1M@CGFMKEEK@?$AAe?$AAs?$AA?9?$AAP?$AAR?$AA?$AA@ 10003fe4     libucrt:lcidtoname_downlevel.obj
 0001:00002ff0       ??_C@_1O@ICJHKIIK@?$AAz?$AAh?$AA?9?$AAC?$AAH?$AAT?$AA?$AA@ 10003ff0     libucrt:lcidtoname_downlevel.obj
 0001:00003000       ??_C@_15CLNEJCE@?$AAs?$AAr?$AA?$AA@ 10004000     libucrt:lcidtoname_downlevel.obj
 0001:00003728       ??_C@_1M@KAHEKEIG@?$AAa?$AAf?$AA?9?$AAz?$AAa?$AA?$AA@ 10004728     libucrt:lcidtoname_downlevel.obj
 0001:00003734       ??_C@_1M@GIECOABL@?$AAa?$AAr?$AA?9?$AAa?$AAe?$AA?$AA@ 10004734     libucrt:lcidtoname_downlevel.obj
 0001:00003740       ??_C@_1M@BMLMEKGI@?$AAa?$AAr?$AA?9?$AAb?$AAh?$AA?$AA@ 10004740     libucrt:lcidtoname_downlevel.obj
 0001:0000374c       ??_C@_1M@DAPFDGGB@?$AAa?$AAr?$AA?9?$AAd?$AAz?$AA?$AA@ 1000474c     libucrt:lcidtoname_downlevel.obj
 0001:00003758       ??_C@_1M@FJNKGKIG@?$AAa?$AAr?$AA?9?$AAe?$AAg?$AA?$AA@ 10004758     libucrt:lcidtoname_downlevel.obj
 0001:00003764       ??_C@_1M@FLGKKCLO@?$AAa?$AAr?$AA?9?$AAi?$AAq?$AA?$AA@ 10004764     libucrt:lcidtoname_downlevel.obj
 0001:00003770       ??_C@_1M@GNDIPALM@?$AAa?$AAr?$AA?9?$AAj?$AAo?$AA?$AA@ 10004770     libucrt:lcidtoname_downlevel.obj
 0001:0000377c       ??_C@_1M@DDMJFMGJ@?$AAa?$AAr?$AA?9?$AAk?$AAw?$AA?$AA@ 1000477c     libucrt:lcidtoname_downlevel.obj
 0001:00003788       ??_C@_1M@EJALMLHM@?$AAa?$AAr?$AA?9?$AAl?$AAb?$AA?$AA@ 10004788     libucrt:lcidtoname_downlevel.obj
 0001:00003794       ??_C@_1M@MOBDBLOC@?$AAa?$AAr?$AA?9?$AAl?$AAy?$AA?$AA@ 10004794     libucrt:lcidtoname_downlevel.obj
 0001:000037a0       ??_C@_1M@JAOCLHDH@?$AAa?$AAr?$AA?9?$AAm?$AAa?$AA?$AA@ 100047a0     libucrt:lcidtoname_downlevel.obj
 0001:000037ac       ??_C@_1M@JHPMKJIE@?$AAa?$AAr?$AA?9?$AAo?$AAm?$AA?$AA@ 100047ac     libucrt:lcidtoname_downlevel.obj
 0001:000037b8       ??_C@_1M@OEPGHFNH@?$AAa?$AAr?$AA?9?$AAq?$AAa?$AA?$AA@ 100047b8     libucrt:lcidtoname_downlevel.obj
 0001:000037c4       ??_C@_1M@KJDONENM@?$AAa?$AAr?$AA?9?$AAs?$AAa?$AA?$AA@ 100047c4     libucrt:lcidtoname_downlevel.obj
 0001:000037d0       ??_C@_1M@DMJDKLKM@?$AAa?$AAr?$AA?9?$AAs?$AAy?$AA?$AA@ 100047d0     libucrt:lcidtoname_downlevel.obj
 0001:000037dc       ??_C@_1M@OMFIPEDC@?$AAa?$AAr?$AA?9?$AAt?$AAn?$AA?$AA@ 100047dc     libucrt:lcidtoname_downlevel.obj
 0001:000037e8       ??_C@_1M@IHMHGAON@?$AAa?$AAr?$AA?9?$AAy?$AAe?$AA?$AA@ 100047e8     libucrt:lcidtoname_downlevel.obj
 0001:000037f4       ??_C@_1BG@KDCPGJGB@?$AAa?$AAz?$AA?9?$AAa?$AAz?$AA?9?$AAc?$AAy?$AAr?$AAl?$AA?$AA@ 100047f4     libucrt:lcidtoname_downlevel.obj
 0001:0000380c       ??_C@_1BG@IBCKDDOE@?$AAa?$AAz?$AA?9?$AAa?$AAz?$AA?9?$AAl?$AAa?$AAt?$AAn?$AA?$AA@ 1000480c     libucrt:lcidtoname_downlevel.obj
 0001:00003824       ??_C@_1M@EGPFDCPD@?$AAb?$AAe?$AA?9?$AAb?$AAy?$AA?$AA@ 10004824     libucrt:lcidtoname_downlevel.obj
 0001:00003830       ??_C@_1M@PCMGMCGC@?$AAb?$AAg?$AA?9?$AAb?$AAg?$AA?$AA@ 10004830     libucrt:lcidtoname_downlevel.obj
 0001:0000383c       ??_C@_1M@BJBMFGOB@?$AAb?$AAn?$AA?9?$AAi?$AAn?$AA?$AA@ 1000483c     libucrt:lcidtoname_downlevel.obj
 0001:00003848       ??_C@_1BG@EAKMMACD@?$AAb?$AAs?$AA?9?$AAb?$AAa?$AA?9?$AAl?$AAa?$AAt?$AAn?$AA?$AA@ 10004848     libucrt:lcidtoname_downlevel.obj
 0001:00003860       ??_C@_1M@KGADAODK@?$AAc?$AAa?$AA?9?$AAe?$AAs?$AA?$AA@ 10004860     libucrt:lcidtoname_downlevel.obj
 0001:0000386c       ??_C@_1M@COAJPDHI@?$AAc?$AAs?$AA?9?$AAc?$AAz?$AA?$AA@ 1000486c     libucrt:lcidtoname_downlevel.obj
 0001:00003878       ??_C@_1M@DHBHFONH@?$AAc?$AAy?$AA?9?$AAg?$AAb?$AA?$AA@ 10004878     libucrt:lcidtoname_downlevel.obj
 0001:00003884       ??_C@_1M@IMGKELGA@?$AAd?$AAa?$AA?9?$AAd?$AAk?$AA?$AA@ 10004884     libucrt:lcidtoname_downlevel.obj
 0001:00003890       ??_C@_1M@NNDGDNGA@?$AAd?$AAe?$AA?9?$AAa?$AAt?$AA?$AA@ 10004890     libucrt:lcidtoname_downlevel.obj
 0001:0000389c       ??_C@_1M@IKDBHEEM@?$AAd?$AAe?$AA?9?$AAc?$AAh?$AA?$AA@ 1000489c     libucrt:lcidtoname_downlevel.obj
 0001:000038a8       ??_C@_1M@GFFOJMCJ@?$AAd?$AAe?$AA?9?$AAd?$AAe?$AA?$AA@ 100048a8     libucrt:lcidtoname_downlevel.obj
 0001:000038b4       ??_C@_1M@MDNLKBPM@?$AAd?$AAe?$AA?9?$AAl?$AAi?$AA?$AA@ 100048b4     libucrt:lcidtoname_downlevel.obj
 0001:000038c0       ??_C@_1M@NJBEEJNL@?$AAd?$AAe?$AA?9?$AAl?$AAu?$AA?$AA@ 100048c0     libucrt:lcidtoname_downlevel.obj
 0001:000038cc       ??_C@_1O@GNNELBAP@?$AAd?$AAi?$AAv?$AA?9?$AAm?$AAv?$AA?$AA@ 100048cc     libucrt:lcidtoname_downlevel.obj
 0001:000038dc       ??_C@_1M@EJLEOGAE@?$AAe?$AAl?$AA?9?$AAg?$AAr?$AA?$AA@ 100048dc     libucrt:lcidtoname_downlevel.obj
 0001:000038e8       ??_C@_1M@GMPONJN@?$AAe?$AAn?$AA?9?$AAa?$AAu?$AA?$AA@ 100048e8     libucrt:lcidtoname_downlevel.obj
 0001:000038f4       ??_C@_1M@NIDIIPGF@?$AAe?$AAn?$AA?9?$AAb?$AAz?$AA?$AA@ 100048f4     libucrt:lcidtoname_downlevel.obj
 0001:00003900       ??_C@_1M@JEHMIMFO@?$AAe?$AAn?$AA?9?$AAc?$AAa?$AA?$AA@ 10004900     libucrt:lcidtoname_downlevel.obj
 0001:0000390c       ??_C@_1M@IGMJCDLA@?$AAe?$AAn?$AA?9?$AAc?$AAb?$AA?$AA@ 1000490c     libucrt:lcidtoname_downlevel.obj
 0001:00003918       ??_C@_1M@BNFIGBKG@?$AAe?$AAn?$AA?9?$AAg?$AAb?$AA?$AA@ 10004918     libucrt:lcidtoname_downlevel.obj
 0001:00003924       ??_C@_1M@LKIFDIGP@?$AAe?$AAn?$AA?9?$AAi?$AAe?$AA?$AA@ 10004924     libucrt:lcidtoname_downlevel.obj
 0001:00003930       ??_C@_1M@PJKFGCCO@?$AAe?$AAn?$AA?9?$AAj?$AAm?$AA?$AA@ 10004930     libucrt:lcidtoname_downlevel.obj
 0001:0000393c       ??_C@_1M@KPPKEPBO@?$AAe?$AAn?$AA?9?$AAn?$AAz?$AA?$AA@ 1000493c     libucrt:lcidtoname_downlevel.obj
 0001:00003948       ??_C@_1M@GMDGLDOB@?$AAe?$AAn?$AA?9?$AAp?$AAh?$AA?$AA@ 10004948     libucrt:lcidtoname_downlevel.obj
 0001:00003954       ??_C@_1M@ONGIBJNA@?$AAe?$AAn?$AA?9?$AAt?$AAt?$AA?$AA@ 10004954     libucrt:lcidtoname_downlevel.obj
 0001:00003960       ??_C@_1M@LLODPCMM@?$AAe?$AAn?$AA?9?$AAu?$AAs?$AA?$AA@ 10004960     libucrt:lcidtoname_downlevel.obj
 0001:0000396c       ??_C@_1M@LAKFNPAN@?$AAe?$AAn?$AA?9?$AAz?$AAa?$AA?$AA@ 1000496c     libucrt:lcidtoname_downlevel.obj
 0001:00003978       ??_C@_1M@MFNHNHEO@?$AAe?$AAn?$AA?9?$AAz?$AAw?$AA?$AA@ 10004978     libucrt:lcidtoname_downlevel.obj
 0001:00003984       ??_C@_1M@EJEINPHM@?$AAe?$AAs?$AA?9?$AAa?$AAr?$AA?$AA@ 10004984     libucrt:lcidtoname_downlevel.obj
 0001:00003990       ??_C@_1M@GNKPCCJA@?$AAe?$AAs?$AA?9?$AAb?$AAo?$AA?$AA@ 10004990     libucrt:lcidtoname_downlevel.obj
 0001:0000399c       ??_C@_1M@LEEGFONL@?$AAe?$AAs?$AA?9?$AAc?$AAl?$AA?$AA@ 1000499c     libucrt:lcidtoname_downlevel.obj
 0001:000039a8       ??_C@_1M@KGPDPBDF@?$AAe?$AAs?$AA?9?$AAc?$AAo?$AA?$AA@ 100049a8     libucrt:lcidtoname_downlevel.obj
 0001:000039b4       ??_C@_1M@EIAHOHH@?$AAe?$AAs?$AA?9?$AAc?$AAr?$AA?$AA@ 100049b4     libucrt:lcidtoname_downlevel.obj
 0001:000039c0       ??_C@_1M@LLPGMBIN@?$AAe?$AAs?$AA?9?$AAd?$AAo?$AA?$AA@ 100049c0     libucrt:lcidtoname_downlevel.obj
 0001:000039cc       ??_C@_1M@DKHMKNJA@?$AAe?$AAs?$AA?9?$AAe?$AAc?$AA?$AA@ 100049cc     libucrt:lcidtoname_downlevel.obj
 0001:000039d8       ??_C@_1M@GKGFPKAP@?$AAe?$AAs?$AA?9?$AAe?$AAs?$AA?$AA@ 100049d8     libucrt:lcidtoname_downlevel.obj
 0001:000039e4       ??_C@_1M@LKHKGDLN@?$AAe?$AAs?$AA?9?$AAg?$AAt?$AA?$AA@ 100049e4     libucrt:lcidtoname_downlevel.obj
 0001:000039f0       ??_C@_1M@HEIIGGJD@?$AAe?$AAs?$AA?9?$AAh?$AAn?$AA?$AA@ 100049f0     libucrt:lcidtoname_downlevel.obj
 0001:000039fc       ??_C@_1M@FBDHPPGD@?$AAe?$AAs?$AA?9?$AAm?$AAx?$AA?$AA@ 100049fc     libucrt:lcidtoname_downlevel.obj
 0001:00003a08       ??_C@_1M@DPAGLNDH@?$AAe?$AAs?$AA?9?$AAn?$AAi?$AA?$AA@ 10004a08     libucrt:lcidtoname_downlevel.obj
 0001:00003a14       ??_C@_1M@MDGOPGDD@?$AAe?$AAs?$AA?9?$AAp?$AAa?$AA?$AA@ 10004a14     libucrt:lcidtoname_downlevel.obj
 0001:00003a20       ??_C@_1M@EMAMGBGE@?$AAe?$AAs?$AA?9?$AAp?$AAe?$AA?$AA@ 10004a20     libucrt:lcidtoname_downlevel.obj
 0001:00003a2c       ??_C@_1M@IBMCAOEC@?$AAe?$AAs?$AA?9?$AAp?$AAr?$AA?$AA@ 10004a2c     libucrt:lcidtoname_downlevel.obj
 0001:00003a38       ??_C@_1M@FGMDIJED@?$AAe?$AAs?$AA?9?$AAp?$AAy?$AA?$AA@ 10004a38     libucrt:lcidtoname_downlevel.obj
 0001:00003a44       ??_C@_1M@IIDEOLLL@?$AAe?$AAs?$AA?9?$AAs?$AAv?$AA?$AA@ 10004a44     libucrt:lcidtoname_downlevel.obj
 0001:00003a50       ??_C@_1M@GAOBIPA@?$AAe?$AAs?$AA?9?$AAu?$AAy?$AA?$AA@ 10004a50     libucrt:lcidtoname_downlevel.obj
 0001:00003a5c       ??_C@_1M@JKFFICHJ@?$AAe?$AAs?$AA?9?$AAv?$AAe?$AA?$AA@ 10004a5c     libucrt:lcidtoname_downlevel.obj
 0001:00003a68       ??_C@_1M@PNMLOJDF@?$AAe?$AAt?$AA?9?$AAe?$AAe?$AA?$AA@ 10004a68     libucrt:lcidtoname_downlevel.obj
 0001:00003a74       ??_C@_1M@GHHLIKEI@?$AAe?$AAu?$AA?9?$AAe?$AAs?$AA?$AA@ 10004a74     libucrt:lcidtoname_downlevel.obj
 0001:00003a80       ??_C@_1M@PBNONODE@?$AAf?$AAa?$AA?9?$AAi?$AAr?$AA?$AA@ 10004a80     libucrt:lcidtoname_downlevel.obj
 0001:00003a8c       ??_C@_1M@JEEHPMIL@?$AAf?$AAi?$AA?9?$AAf?$AAi?$AA?$AA@ 10004a8c     libucrt:lcidtoname_downlevel.obj
 0001:00003a98       ??_C@_1M@LMDCNDBA@?$AAf?$AAo?$AA?9?$AAf?$AAo?$AA?$AA@ 10004a98     libucrt:lcidtoname_downlevel.obj
 0001:00003aa4       ??_C@_1M@JKEOHLDK@?$AAf?$AAr?$AA?9?$AAb?$AAe?$AA?$AA@ 10004aa4     libucrt:lcidtoname_downlevel.obj
 0001:00003ab0       ??_C@_1M@NOHADPMI@?$AAf?$AAr?$AA?9?$AAc?$AAa?$AA?$AA@ 10004ab0     libucrt:lcidtoname_downlevel.obj
 0001:00003abc       ??_C@_1M@KDHIHAEC@?$AAf?$AAr?$AA?9?$AAc?$AAh?$AA?$AA@ 10004abc     libucrt:lcidtoname_downlevel.obj
 0001:00003ac8       ??_C@_1M@MMBBFGAK@?$AAf?$AAr?$AA?9?$AAf?$AAr?$AA?$AA@ 10004ac8     libucrt:lcidtoname_downlevel.obj
 0001:00003ad4       ??_C@_1M@PAFNENNF@?$AAf?$AAr?$AA?9?$AAl?$AAu?$AA?$AA@ 10004ad4     libucrt:lcidtoname_downlevel.obj
 0001:00003ae0       ??_C@_1M@EOHDJGDD@?$AAf?$AAr?$AA?9?$AAm?$AAc?$AA?$AA@ 10004ae0     libucrt:lcidtoname_downlevel.obj
 0001:00003aec       ??_C@_1M@FAPLLOPF@?$AAg?$AAl?$AA?9?$AAe?$AAs?$AA?$AA@ 10004aec     libucrt:lcidtoname_downlevel.obj
 0001:00003af8       ??_C@_1M@FOPBFLOO@?$AAg?$AAu?$AA?9?$AAi?$AAn?$AA?$AA@ 10004af8     libucrt:lcidtoname_downlevel.obj
 0001:00003b04       ??_C@_1M@KBMCINPM@?$AAh?$AAe?$AA?9?$AAi?$AAl?$AA?$AA@ 10004b04     libucrt:lcidtoname_downlevel.obj
 0001:00003b10       ??_C@_1M@BBPHKFPJ@?$AAh?$AAi?$AA?9?$AAi?$AAn?$AA?$AA@ 10004b10     libucrt:lcidtoname_downlevel.obj
 0001:00003b1c       ??_C@_1M@PMBNDPHD@?$AAh?$AAr?$AA?9?$AAb?$AAa?$AA?$AA@ 10004b1c     libucrt:lcidtoname_downlevel.obj
 0001:00003b28       ??_C@_1M@BPCKOEGE@?$AAh?$AAr?$AA?9?$AAh?$AAr?$AA?$AA@ 10004b28     libucrt:lcidtoname_downlevel.obj
 0001:00003b34       ??_C@_1M@GACBMHKE@?$AAh?$AAu?$AA?9?$AAh?$AAu?$AA?$AA@ 10004b34     libucrt:lcidtoname_downlevel.obj
 0001:00003b40       ??_C@_1M@MILPAJJC@?$AAh?$AAy?$AA?9?$AAa?$AAm?$AA?$AA@ 10004b40     libucrt:lcidtoname_downlevel.obj
 0001:00003b4c       ??_C@_1M@BABBICEC@?$AAi?$AAd?$AA?9?$AAi?$AAd?$AA?$AA@ 10004b4c     libucrt:lcidtoname_downlevel.obj
 0001:00003b58       ??_C@_1M@BIKNHHPF@?$AAi?$AAs?$AA?9?$AAi?$AAs?$AA?$AA@ 10004b58     libucrt:lcidtoname_downlevel.obj
 0001:00003b64       ??_C@_1M@NMPCJPHE@?$AAi?$AAt?$AA?9?$AAc?$AAh?$AA?$AA@ 10004b64     libucrt:lcidtoname_downlevel.obj
 0001:00003b70       ??_C@_1M@GHKGFEDF@?$AAi?$AAt?$AA?9?$AAi?$AAt?$AA?$AA@ 10004b70     libucrt:lcidtoname_downlevel.obj
 0001:00003b7c       ??_C@_1M@NIEJCJJA@?$AAj?$AAa?$AA?9?$AAj?$AAp?$AA?$AA@ 10004b7c     libucrt:lcidtoname_downlevel.obj
 0001:00003b88       ??_C@_1M@JILFNBIM@?$AAk?$AAa?$AA?9?$AAg?$AAe?$AA?$AA@ 10004b88     libucrt:lcidtoname_downlevel.obj
 0001:00003b94       ??_C@_1M@PACPMGPH@?$AAk?$AAk?$AA?9?$AAk?$AAz?$AA?$AA@ 10004b94     libucrt:lcidtoname_downlevel.obj
 0001:00003ba0       ??_C@_1M@IELFGMHA@?$AAk?$AAn?$AA?9?$AAi?$AAn?$AA?$AA@ 10004ba0     libucrt:lcidtoname_downlevel.obj
 0001:00003bac       ??_C@_1O@IBBJHCH@?$AAk?$AAo?$AAk?$AA?9?$AAi?$AAn?$AA?$AA@ 10004bac     libucrt:lcidtoname_downlevel.obj
 0001:00003bbc       ??_C@_1M@DMHAEOGC@?$AAk?$AAo?$AA?9?$AAk?$AAr?$AA?$AA@ 10004bbc     libucrt:lcidtoname_downlevel.obj
 0001:00003bc8       ??_C@_1M@HBAHBIGA@?$AAk?$AAy?$AA?9?$AAk?$AAg?$AA?$AA@ 10004bc8     libucrt:lcidtoname_downlevel.obj
 0001:00003bd4       ??_C@_1M@KPMILCJG@?$AAl?$AAt?$AA?9?$AAl?$AAt?$AA?$AA@ 10004bd4     libucrt:lcidtoname_downlevel.obj
 0001:00003be0       ??_C@_1M@BDEKKCA@?$AAl?$AAv?$AA?9?$AAl?$AAv?$AA?$AA@ 10004be0     libucrt:lcidtoname_downlevel.obj
 0001:00003bec       ??_C@_1M@ELCKCCJJ@?$AAm?$AAi?$AA?9?$AAn?$AAz?$AA?$AA@ 10004bec     libucrt:lcidtoname_downlevel.obj
 0001:00003bf8       ??_C@_1M@CBOOLAPA@?$AAm?$AAk?$AA?9?$AAm?$AAk?$AA?$AA@ 10004bf8     libucrt:lcidtoname_downlevel.obj
 0001:00003c04       ??_C@_1M@GPHNBJKN@?$AAm?$AAl?$AA?9?$AAi?$AAn?$AA?$AA@ 10004c04     libucrt:lcidtoname_downlevel.obj
 0001:00003c10       ??_C@_1M@PABJILIG@?$AAm?$AAn?$AA?9?$AAm?$AAn?$AA?$AA@ 10004c10     libucrt:lcidtoname_downlevel.obj
 0001:00003c1c       ??_C@_1M@FGBKKIPG@?$AAm?$AAr?$AA?9?$AAi?$AAn?$AA?$AA@ 10004c1c     libucrt:lcidtoname_downlevel.obj
 0001:00003c28       ??_C@_1M@NDBPDDAL@?$AAm?$AAs?$AA?9?$AAb?$AAn?$AA?$AA@ 10004c28     libucrt:lcidtoname_downlevel.obj
 0001:00003c34       ??_C@_1M@OPIHOOPI@?$AAm?$AAs?$AA?9?$AAm?$AAy?$AA?$AA@ 10004c34     libucrt:lcidtoname_downlevel.obj
 0001:00003c40       ??_C@_1M@PPDBCNFM@?$AAm?$AAt?$AA?9?$AAm?$AAt?$AA?$AA@ 10004c40     libucrt:lcidtoname_downlevel.obj
 0001:00003c4c       ??_C@_1M@KDJDKMDD@?$AAn?$AAb?$AA?9?$AAn?$AAo?$AA?$AA@ 10004c4c     libucrt:lcidtoname_downlevel.obj
 0001:00003c58       ??_C@_1M@KFCFLMJP@?$AAn?$AAl?$AA?9?$AAb?$AAe?$AA?$AA@ 10004c58     libucrt:lcidtoname_downlevel.obj
 0001:00003c64       ??_C@_1M@KPOPDDGO@?$AAn?$AAl?$AA?9?$AAn?$AAl?$AA?$AA@ 10004c64     libucrt:lcidtoname_downlevel.obj
 0001:00003c70       ??_C@_1M@LJKPEMLN@?$AAn?$AAn?$AA?9?$AAn?$AAo?$AA?$AA@ 10004c70     libucrt:lcidtoname_downlevel.obj
 0001:00003c7c       ??_C@_1M@BDGHHBFL@?$AAn?$AAs?$AA?9?$AAz?$AAa?$AA?$AA@ 10004c7c     libucrt:lcidtoname_downlevel.obj
 0001:00003c88       ??_C@_1M@IDEHOAP@?$AAp?$AAa?$AA?9?$AAi?$AAn?$AA?$AA@ 10004c88     libucrt:lcidtoname_downlevel.obj
 0001:00003c94       ??_C@_1M@HDBKGOGH@?$AAp?$AAl?$AA?9?$AAp?$AAl?$AA?$AA@ 10004c94     libucrt:lcidtoname_downlevel.obj
 0001:00003ca0       ??_C@_1M@LJLLCMEH@?$AAp?$AAt?$AA?9?$AAb?$AAr?$AA?$AA@ 10004ca0     libucrt:lcidtoname_downlevel.obj
 0001:00003cac       ??_C@_1M@NCMONAAL@?$AAp?$AAt?$AA?9?$AAp?$AAt?$AA?$AA@ 10004cac     libucrt:lcidtoname_downlevel.obj
 0001:00003cb8       ??_C@_1O@EAKMAJDN@?$AAq?$AAu?$AAz?$AA?9?$AAb?$AAo?$AA?$AA@ 10004cb8     libucrt:lcidtoname_downlevel.obj
 0001:00003cc8       ??_C@_1O@BHHPIGDN@?$AAq?$AAu?$AAz?$AA?9?$AAe?$AAc?$AA?$AA@ 10004cc8     libucrt:lcidtoname_downlevel.obj
 0001:00003cd8       ??_C@_1O@GBAPEKMJ@?$AAq?$AAu?$AAz?$AA?9?$AAp?$AAe?$AA?$AA@ 10004cd8     libucrt:lcidtoname_downlevel.obj
 0001:00003ce8       ??_C@_1M@CLGLEFBO@?$AAr?$AAo?$AA?9?$AAr?$AAo?$AA?$AA@ 10004ce8     libucrt:lcidtoname_downlevel.obj
 0001:00003cf4       ??_C@_1M@CEEDODME@?$AAr?$AAu?$AA?9?$AAr?$AAu?$AA?$AA@ 10004cf4     libucrt:lcidtoname_downlevel.obj
 0001:00003d00       ??_C@_1M@HPKKKMPP@?$AAs?$AAa?$AA?9?$AAi?$AAn?$AA?$AA@ 10004d00     libucrt:lcidtoname_downlevel.obj
 0001:00003d0c       ??_C@_1M@BKMAIGOJ@?$AAs?$AAe?$AA?9?$AAf?$AAi?$AA?$AA@ 10004d0c     libucrt:lcidtoname_downlevel.obj
 0001:00003d18       ??_C@_1M@NDPIFLFI@?$AAs?$AAe?$AA?9?$AAn?$AAo?$AA?$AA@ 10004d18     libucrt:lcidtoname_downlevel.obj
 0001:00003d24       ??_C@_1M@DANKKHJ@?$AAs?$AAe?$AA?9?$AAs?$AAe?$AA?$AA@ 10004d24     libucrt:lcidtoname_downlevel.obj
 0001:00003d30       ??_C@_1M@PNBLONPJ@?$AAs?$AAk?$AA?9?$AAs?$AAk?$AA?$AA@ 10004d30     libucrt:lcidtoname_downlevel.obj
 0001:00003d3c       ??_C@_1M@LFMODOAL@?$AAs?$AAl?$AA?9?$AAs?$AAi?$AA?$AA@ 10004d3c     libucrt:lcidtoname_downlevel.obj
 0001:00003d48       ??_C@_1O@DFKOMPG@?$AAs?$AAm?$AAa?$AA?9?$AAn?$AAo?$AA?$AA@ 10004d48     libucrt:lcidtoname_downlevel.obj
 0001:00003d58       ??_C@_1O@NDKPBNNH@?$AAs?$AAm?$AAa?$AA?9?$AAs?$AAe?$AA?$AA@ 10004d58     libucrt:lcidtoname_downlevel.obj
 0001:00003d68       ??_C@_1O@PLLKBHAB@?$AAs?$AAm?$AAj?$AA?9?$AAn?$AAo?$AA?$AA@ 10004d68     libucrt:lcidtoname_downlevel.obj
 0001:00003d78       ??_C@_1O@CLEPOGCA@?$AAs?$AAm?$AAj?$AA?9?$AAs?$AAe?$AA?$AA@ 10004d78     libucrt:lcidtoname_downlevel.obj
 0001:00003d88       ??_C@_1O@DLGJGKMK@?$AAs?$AAm?$AAn?$AA?9?$AAf?$AAi?$AA?$AA@ 10004d88     libucrt:lcidtoname_downlevel.obj
 0001:00003d98       ??_C@_1O@OJDJGAJC@?$AAs?$AAm?$AAs?$AA?9?$AAf?$AAi?$AA?$AA@ 10004d98     libucrt:lcidtoname_downlevel.obj
 0001:00003da8       ??_C@_1M@BOFOGHPB@?$AAs?$AAq?$AA?9?$AAa?$AAl?$AA?$AA@ 10004da8     libucrt:lcidtoname_downlevel.obj
 0001:00003db4       ??_C@_1BG@LJBBIPGB@?$AAs?$AAr?$AA?9?$AAb?$AAa?$AA?9?$AAc?$AAy?$AAr?$AAl?$AA?$AA@ 10004db4     libucrt:lcidtoname_downlevel.obj
 0001:00003dcc       ??_C@_1BG@JLBENFOE@?$AAs?$AAr?$AA?9?$AAb?$AAa?$AA?9?$AAl?$AAa?$AAt?$AAn?$AA?$AA@ 10004dcc     libucrt:lcidtoname_downlevel.obj
 0001:00003de4       ??_C@_1BG@KODPNHE@?$AAs?$AAr?$AA?9?$AAs?$AAp?$AA?9?$AAc?$AAy?$AAr?$AAl?$AA?$AA@ 10004de4     libucrt:lcidtoname_downlevel.obj
 0001:00003dfc       ??_C@_1BG@CIOGKHPB@?$AAs?$AAr?$AA?9?$AAs?$AAp?$AA?9?$AAl?$AAa?$AAt?$AAn?$AA?$AA@ 10004dfc     libucrt:lcidtoname_downlevel.obj
 0001:00003e14       ??_C@_1M@NGFJLMAC@?$AAs?$AAv?$AA?9?$AAf?$AAi?$AA?$AA@ 10004e14     libucrt:lcidtoname_downlevel.obj
 0001:00003e20       ??_C@_1M@MPJEJAJC@?$AAs?$AAv?$AA?9?$AAs?$AAe?$AA?$AA@ 10004e20     libucrt:lcidtoname_downlevel.obj
 0001:00003e2c       ??_C@_1M@MPNDHLFK@?$AAs?$AAw?$AA?9?$AAk?$AAe?$AA?$AA@ 10004e2c     libucrt:lcidtoname_downlevel.obj
 0001:00003e38       ??_C@_1O@KOHBJJI@?$AAs?$AAy?$AAr?$AA?9?$AAs?$AAy?$AA?$AA@ 10004e38     libucrt:lcidtoname_downlevel.obj
 0001:00003e48       ??_C@_1M@LDCEFHA@?$AAt?$AAa?$AA?9?$AAi?$AAn?$AA?$AA@ 10004e48     libucrt:lcidtoname_downlevel.obj
 0001:00003e54       ??_C@_1M@CNJOFAK@?$AAt?$AAe?$AA?9?$AAi?$AAn?$AA?$AA@ 10004e54     libucrt:lcidtoname_downlevel.obj
 0001:00003e60       ??_C@_1M@GNAECACD@?$AAt?$AAh?$AA?9?$AAt?$AAh?$AA?$AA@ 10004e60     libucrt:lcidtoname_downlevel.obj
 0001:00003e6c       ??_C@_1M@CHBIHOJO@?$AAt?$AAn?$AA?9?$AAz?$AAa?$AA?$AA@ 10004e6c     libucrt:lcidtoname_downlevel.obj
 0001:00003e78       ??_C@_1M@GCCMIGPJ@?$AAt?$AAr?$AA?9?$AAt?$AAr?$AA?$AA@ 10004e78     libucrt:lcidtoname_downlevel.obj
 0001:00003e84       ??_C@_1M@CELMCNBK@?$AAt?$AAt?$AA?9?$AAr?$AAu?$AA?$AA@ 10004e84     libucrt:lcidtoname_downlevel.obj
 0001:00003e90       ??_C@_1M@KLMCELGA@?$AAu?$AAk?$AA?9?$AAu?$AAa?$AA?$AA@ 10004e90     libucrt:lcidtoname_downlevel.obj
 0001:00003e9c       ??_C@_1M@EPAJJAJF@?$AAu?$AAr?$AA?9?$AAp?$AAk?$AA?$AA@ 10004e9c     libucrt:lcidtoname_downlevel.obj
 0001:00003ea8       ??_C@_1BG@GEGPMCDJ@?$AAu?$AAz?$AA?9?$AAu?$AAz?$AA?9?$AAc?$AAy?$AAr?$AAl?$AA?$AA@ 10004ea8     libucrt:lcidtoname_downlevel.obj
 0001:00003ec0       ??_C@_1BG@EGGKJILM@?$AAu?$AAz?$AA?9?$AAu?$AAz?$AA?9?$AAl?$AAa?$AAt?$AAn?$AA?$AA@ 10004ec0     libucrt:lcidtoname_downlevel.obj
 0001:00003ed8       ??_C@_1M@GFOCLFF@?$AAv?$AAi?$AA?9?$AAv?$AAn?$AA?$AA@ 10004ed8     libucrt:lcidtoname_downlevel.obj
 0001:00003ee4       ??_C@_1M@CPAMEDFI@?$AAx?$AAh?$AA?9?$AAz?$AAa?$AA?$AA@ 10004ee4     libucrt:lcidtoname_downlevel.obj
 0001:00003ef0       ??_C@_1O@EBKIFIGN@?$AAz?$AAh?$AA?9?$AAc?$AAh?$AAs?$AA?$AA@ 10004ef0     libucrt:lcidtoname_downlevel.obj
 0001:00003f00       ??_C@_1O@NMHPGANE@?$AAz?$AAh?$AA?9?$AAc?$AAh?$AAt?$AA?$AA@ 10004f00     libucrt:lcidtoname_downlevel.obj
 0001:00003f10       ??_C@_1M@LPINJOMC@?$AAz?$AAh?$AA?9?$AAc?$AAn?$AA?$AA@ 10004f10     libucrt:lcidtoname_downlevel.obj
 0001:00003f1c       ??_C@_1M@OCJEJODD@?$AAz?$AAh?$AA?9?$AAh?$AAk?$AA?$AA@ 10004f1c     libucrt:lcidtoname_downlevel.obj
 0001:00003f28       ??_C@_1M@DNDLJINH@?$AAz?$AAh?$AA?9?$AAm?$AAo?$AA?$AA@ 10004f28     libucrt:lcidtoname_downlevel.obj
 0001:00003f34       ??_C@_1M@MBFDNDND@?$AAz?$AAh?$AA?9?$AAs?$AAg?$AA?$AA@ 10004f34     libucrt:lcidtoname_downlevel.obj
 0001:00003f40       ??_C@_1M@IMEPLEPE@?$AAz?$AAh?$AA?9?$AAt?$AAw?$AA?$AA@ 10004f40     libucrt:lcidtoname_downlevel.obj
 0001:00003f4c       ??_C@_1M@BBGHNHJP@?$AAz?$AAu?$AA?9?$AAz?$AAa?$AA?$AA@ 10004f4c     libucrt:lcidtoname_downlevel.obj
 0001:00003f58       ??_C@_00CNPNBAHC@?$AA@     10004f58     libucrt:mbrtowc.obj
 0001:00003fb8       ??_C@_1BA@BALFACEM@?$AAC?$AAO?$AAN?$AAO?$AAU?$AAT?$AA$?$AA?$AA@ 10004fb8     libucrt:initcon.obj
 0001:000040d0       __infinity                 100050d0     libucrt:87tran.obj
 0001:000040da       __minfinity                100050da     libucrt:87tran.obj
 0001:000040e4       __logemax                  100050e4     libucrt:87tran.obj
 0001:0000410a       __OP_EXPjmptab             1000510a     libucrt:87tran.obj
 0001:00004130       __indefinite               10005130     libucrt:87disp.obj
 0001:0000413a       __piby2                    1000513a     libucrt:87disp.obj
 0001:00004144       __piby4                    10005144     libucrt:87disp.obj
 0001:00004178       __DEFAULT_CW_in_mem        10005178     libucrt:common.obj
 0001:0000417a       __pi_by_2_to_61            1000517a     libucrt:common.obj
 0001:000041b4       ??_C@_03MGHMBJCF@log?$AA@  100051b4     libucrt:libm_error.obj
 0001:000041b8       ??_C@_05HGHHAHAP@log10?$AA@ 100051b8     libucrt:libm_error.obj
 0001:000041c0       ??_C@_03KHJOGHMM@exp?$AA@  100051c0     libucrt:libm_error.obj
 0001:000041c4       ??_C@_03JGHBODFD@pow?$AA@  100051c4     libucrt:libm_error.obj
 0001:000041c8       ??_C@_04FIHNOPOL@asin?$AA@ 100051c8     libucrt:libm_error.obj
 0001:000041d0       ??_C@_04PDIFKINK@acos?$AA@ 100051d0     libucrt:libm_error.obj
 0001:000041d8       ??_C@_04EIAKFFMI@sqrt?$AA@ 100051d8     libucrt:libm_error.obj
 0001:000041e0       __real@3ff0000000000000    100051e0     libucrt:libm_error.obj
 0001:00004200       ___acrt_log10_table_t      10005200     libucrt:log10_tables.obj
 0001:00004610       ___acrt_log10_table_cb     10005610     libucrt:log10_tables.obj
 0001:00004a20       __real@3fe0000000000000    10005a20     libucrt:powhlp.obj
 0001:00004b10       ??_C@_04COOMCNPB@sinh?$AA@ 10005b10     libucrt:fpexcept.obj
 0001:00004b18       ??_C@_04HPJJNFIM@cosh?$AA@ 10005b18     libucrt:fpexcept.obj
 0001:00004b20       ??_C@_04FJHINJAO@tanh?$AA@ 10005b20     libucrt:fpexcept.obj
 0001:00004b28       ??_C@_04MLLJIGOK@atan?$AA@ 10005b28     libucrt:fpexcept.obj
 0001:00004b30       ??_C@_05KNGEOGJB@atan2?$AA@ 10005b30     libucrt:fpexcept.obj
 0001:00004b38       ??_C@_03BLEJJJBH@sin?$AA@  10005b38     libucrt:fpexcept.obj
 0001:00004b3c       ??_C@_03LALBNOCG@cos?$AA@  10005b3c     libucrt:fpexcept.obj
 0001:00004b40       ??_C@_03IIINPABG@tan?$AA@  10005b40     libucrt:fpexcept.obj
 0001:00004b44       ??_C@_04GFPJNGEK@ceil?$AA@ 10005b44     libucrt:fpexcept.obj
 0001:00004b4c       ??_C@_05PBJFFIGL@floor?$AA@ 10005b4c     libucrt:fpexcept.obj
 0001:00004b54       ??_C@_04ODHECPBC@fabs?$AA@ 10005b54     libucrt:fpexcept.obj
 0001:00004b5c       ??_C@_04EHEDPDJG@modf?$AA@ 10005b5c     libucrt:fpexcept.obj
 0001:00004b64       ??_C@_05CEJMAHNP@ldexp?$AA@ 10005b64     libucrt:fpexcept.obj
 0001:00004b6c       ??_C@_05KBKMEMPO@_cabs?$AA@ 10005b6c     libucrt:fpexcept.obj
 0001:00004b74       ??_C@_06MEIMCGCF@_hypot?$AA@ 10005b74     libucrt:fpexcept.obj
 0001:00004b7c       ??_C@_04KEPJIHGP@fmod?$AA@ 10005b7c     libucrt:fpexcept.obj
 0001:00004b84       ??_C@_05GKKHEGJL@frexp?$AA@ 10005b84     libucrt:fpexcept.obj
 0001:00004b8c       ??_C@_03MJLDFKDL@_y0?$AA@  10005b8c     libucrt:fpexcept.obj
 0001:00004b90       ??_C@_03NAKIGLHK@_y1?$AA@  10005b90     libucrt:fpexcept.obj
 0001:00004b94       ??_C@_03ONILCKOB@_yn?$AA@  10005b94     libucrt:fpexcept.obj
 0001:00004b98       ??_C@_05JGDBENOH@_logb?$AA@ 10005b98     libucrt:fpexcept.obj
 0001:00004ba0       ??_C@_0L@KDOEJCKC@_nextafter?$AA@ 10005ba0     libucrt:fpexcept.obj
 0001:00004bb0       __d_inf                    10005bb0     libucrt:util.obj
 0001:00004bb8       __d_max                    10005bb8     libucrt:util.obj
 0001:00004bc0       __d_mzero                  10005bc0     libucrt:util.obj
 0001:00004bf0       __load_config_used         10005bf0     LIBCMT:loadcfg.obj
 0001:00004c90       ___safe_se_handler_table   10005c90     <linker-defined>
 0001:00004f14       ___rtc_iaa                 10005f14     LIBCMT:initsect.obj
 0001:00004f18       ___rtc_izz                 10005f18     LIBCMT:initsect.obj
 0001:00004f1c       ___rtc_taa                 10005f1c     LIBCMT:initsect.obj
 0001:00004f20       ___rtc_tzz                 10005f20     LIBCMT:initsect.obj
 0001:00004f30       __alloca_probe             10005f30 f   chkstk.obj
 0001:00004f30       __chkstk                   10005f30 f   chkstk.obj
 0001:00004f60       ?ProcessShiftKey@@YAXHH@Z  10005f60 f   DrawLine.obj
 0001:000055d0       ?SetTitle@@YA_NHH@Z        100065d0 f   DrawLine.obj
 0001:00005710       _GetGlobalInfoW@4          10006710 f   DrawLine.obj
 0001:000057a0       _GetPluginInfoW@4          100067a0 f   DrawLine.obj
 0001:000057f0       _OpenW@4                   100067f0 f   DrawLine.obj
 0001:00005b10       _SetStartupInfoW@4         10006b10 f   DrawLine.obj
 0001:00005ef0       _DecodePointerWrapper@4    10006ef0 f   vc_crt_fix_impl.obj
 0001:00005f40       _EncodePointerWrapper@4    10006f40 f   vc_crt_fix_impl.obj
 0001:00005f90       _GetLogicalProcessorInformationWrapper@8 10006f90 f   vc_crt_fix_impl.obj
 0001:00005fe0       _GetModuleHandleExWWrapper@12 10006fe0 f   vc_crt_fix_impl.obj
 0001:00006030       _GetNumaHighestNodeNumberWrapper@4 10007030 f   vc_crt_fix_impl.obj
 0001:00006080       _InitializeSListHeadWrapper@4 10007080 f   vc_crt_fix_impl.obj
 0001:000060d0       _InterlockedFlushSListWrapper@4 100070d0 f   vc_crt_fix_impl.obj
 0001:00006120       _InterlockedPopEntrySListWrapper@4 10007120 f   vc_crt_fix_impl.obj
 0001:00006170       _InterlockedPushEntrySListWrapper@8 10007170 f   vc_crt_fix_impl.obj
 0001:000061c0       _InterlockedPushListSListExWrapper@16 100071c0 f   vc_crt_fix_impl.obj
 0001:00006210       _QueryDepthSListWrapper@4  10007210 f   vc_crt_fix_impl.obj
 0001:00006260       _RtlFirstEntrySListWrapper@4 10007260 f   vc_crt_fix_impl.obj
 0001:000062a3       ??$__crt_fast_encode_pointer@PAP6AXXZ@@YAPAP6AXXZQAP6AXXZ@Z 100072a3 f i LIBCMT:utility.obj
 0001:000062a3       ??$__crt_fast_encode_pointer@PAX@@YAPAXQAX@Z 100072a3 f i libvcruntime:winapi_downlevel.obj
 0001:00006304       ___scrt_acquire_startup_lock 10007304 f   LIBCMT:utility.obj
 0001:00006336       ___scrt_dllmain_after_initialize_c 10007336 f   LIBCMT:utility.obj
 0001:00006361       ___scrt_dllmain_before_initialize_c 10007361 f   LIBCMT:utility.obj
 0001:0000636f       ___scrt_dllmain_crt_thread_attach 1000736f f   LIBCMT:utility.obj
 0001:0000638e       ___scrt_dllmain_crt_thread_detach 1000738e f   LIBCMT:utility.obj
 0001:0000639b       ___scrt_dllmain_exception_filter 1000739b f   LIBCMT:utility.obj
 0001:000063cf       ___scrt_dllmain_uninitialize_c 100073cf f   LIBCMT:utility.obj
 0001:000063f2       ___scrt_dllmain_uninitialize_critical 100073f2 f   LIBCMT:utility.obj
 0001:000063ff       ___scrt_initialize_crt     100073ff f   LIBCMT:utility.obj
 0001:00006438       ___scrt_initialize_onexit_tables 10007438 f   LIBCMT:utility.obj
 0001:000064dd       ___scrt_is_nonwritable_in_current_image 100074dd f   LIBCMT:utility.obj
 0001:00006571       ___scrt_release_startup_lock 10007571 f   LIBCMT:utility.obj
 0001:0000658e       ___scrt_uninitialize_crt   1000758e f   LIBCMT:utility.obj
 0001:000065b6       __onexit                   100075b6 f   LIBCMT:utility.obj
 0001:000065f1       _atexit                    100075f1 f   LIBCMT:utility.obj
 0001:00006926       __DllMainCRTStartup@12     10007926 f   LIBCMT:dll_dllmain.obj
 0001:00006949       ___isa_available_init      10007949 f   LIBCMT:cpu_disp.obj
 0001:00006ae0       __get_startup_argv_mode    10007ae0 f   LIBCMT:argv_mode.obj
 0001:00006ae4       ___scrt_is_ucrt_dll_in_use 10007ae4 f   LIBCMT:ucrt_detection.obj
 0001:00006af0       ___scrt_fastfail           10007af0 f   LIBCMT:utility_desktop.obj
 0001:00006c0a       __crt_debugger_hook        10007c0a f   LIBCMT:utility_desktop.obj
 0001:00006c20       __SEH_prolog4              10007c20 f   LIBCMT:sehprolg4.obj
 0001:00006c66       __SEH_epilog4              10007c66 f   LIBCMT:sehprolg4.obj
 0001:00006c7b       @_guard_check_icall_nop@4  10007c7b f i LIBCMT:guard_support.obj
 0001:00006cc9       ___security_init_cookie    10007cc9 f   LIBCMT:gs_support.obj
 0001:00006d14       _DllMain@12                10007d14 f   LIBCMT:dll_dllmain_stub.obj
 0001:00006d1a       ?__scrt_initialize_type_info@@YAXXZ 10007d1a f   LIBCMT:tncleanup.obj
 0001:00006d26       ?__scrt_uninitialize_type_info@@YAXXZ 10007d26 f   LIBCMT:tncleanup.obj
 0001:00006d32       ___local_stdio_printf_options 10007d32 f i LIBCMT:default_local_stdio_options.obj
 0001:00006d38       ___local_stdio_scanf_options 10007d38 f i LIBCMT:default_local_stdio_options.obj
 0001:00006d3e       ___scrt_initialize_default_local_stdio_options 10007d3e f   LIBCMT:default_local_stdio_options.obj
 0001:00006d5b       ___scrt_get_dyn_tls_init_callback 10007d5b f   LIBCMT:dyn_tls_init.obj
 0001:00006d61       __RTC_Initialize           10007d61 f   LIBCMT:initsect.obj
 0001:00006d8d       __RTC_Terminate            10007d8d f   LIBCMT:initsect.obj
 0001:00006db9       @__security_check_cookie@4 10007db9 f   LIBCMT:secchk.obj
 0001:00006dca       ___raise_securityfailure   10007dca f   LIBCMT:gs_report.obj
 0001:00006df2       ___report_gsfailure        10007df2 f   LIBCMT:gs_report.obj
 0001:00006ef0       _memcpy                    10007ef0 f   libvcruntime:memcpy.obj
 0001:00007470       _memset                    10008470 f   libvcruntime:memset.obj
 0001:000075ca       ___vcrt_initialize         100085ca f   libvcruntime:initialization.obj
 0001:000075f3       ___vcrt_thread_attach      100085f3 f   libvcruntime:initialization.obj
 0001:000075fe       ___vcrt_thread_detach      100085fe f   libvcruntime:initialization.obj
 0001:00007609       ___vcrt_uninitialize       10008609 f   libvcruntime:initialization.obj
 0001:00007628       ___vcrt_uninitialize_critical 10008628 f   libvcruntime:initialization.obj
 0001:00007670       __except_handler4          10008670 f   libvcruntime:chandler4.obj
 0001:000077c7       ___std_type_info_destroy_list 100087c7 f   libvcruntime:std_type_info.obj
 0001:000077ea       ___vcrt_freefls@4          100087ea f   libvcruntime:per_thread_data.obj
 0001:00007806       ___vcrt_freeptd            10008806 f   libvcruntime:per_thread_data.obj
 0001:0000783c       ___vcrt_getptd_noexit      1000883c f   libvcruntime:per_thread_data.obj
 0001:000078ce       ___vcrt_initialize_ptd     100088ce f   libvcruntime:per_thread_data.obj
 0001:00007901       ___vcrt_uninitialize_ptd   10008901 f   libvcruntime:per_thread_data.obj
 0001:0000791c       ___vcrt_initialize_locks   1000891c f   libvcruntime:locks.obj
 0001:00007958       ___vcrt_uninitialize_locks 10008958 f   libvcruntime:locks.obj
 0001:00007aba       ___vcrt_FlsAlloc           10008aba f   libvcruntime:winapi_downlevel.obj
 0001:00007af5       ___vcrt_FlsFree            10008af5 f   libvcruntime:winapi_downlevel.obj
 0001:00007b30       ___vcrt_FlsGetValue        10008b30 f   libvcruntime:winapi_downlevel.obj
 0001:00007b6b       ___vcrt_FlsSetValue        10008b6b f   libvcruntime:winapi_downlevel.obj
 0001:00007ba9       ___vcrt_InitializeCriticalSectionEx 10008ba9 f   libvcruntime:winapi_downlevel.obj
 0001:00007bf0       ___vcrt_initialize_winapi_thunks 10008bf0 f   libvcruntime:winapi_downlevel.obj
 0001:00007c19       ___vcrt_uninitialize_winapi_thunks 10008c19 f   libvcruntime:winapi_downlevel.obj
 0001:00007c4b       ___vcrt_initialize_pure_virtual_call_handler 10008c4b f   libvcruntime:purevirt_data.obj
 0001:00007c60       __local_unwind4            10008c60 f   libvcruntime:exsup4.obj
 0001:00007d38       __seh_longjmp_unwind4@4    10008d38 f   libvcruntime:exsup4.obj
 0001:00007d60       @_EH4_CallFilterFunc@8     10008d60 f   libvcruntime:exsup4.obj
 0001:00007d78       @_EH4_TransferToHandler@8  10008d78 f   libvcruntime:exsup4.obj
 0001:00007d94       @_EH4_GlobalUnwind2@8      10008d94 f   libvcruntime:exsup4.obj
 0001:00007db0       @_EH4_LocalUnwind@16       10008db0 f   libvcruntime:exsup4.obj
 0001:00007dc7       ___except_validate_context_record 10008dc7 f   libvcruntime:jbcxrval.obj
 0001:00007df7       ___except_validate_jump_buffer 10008df7 f   libvcruntime:jbcxrval.obj
 0001:00007e30       __global_unwind2           10008e30 f   libvcruntime:exsup.obj
 0001:00007e96       __local_unwind2            10008e96 f   libvcruntime:exsup.obj
 0001:00007f1a       __abnormal_termination     10008f1a f   libvcruntime:exsup.obj
 0001:00007f40       __NLG_Notify1              10008f40 f   libvcruntime:exsup.obj
 0001:00007f4c       __NLG_Notify               10008f4c f   libvcruntime:exsup.obj
 0001:00007f63       __NLG_Dispatch             10008f63     libvcruntime:exsup.obj
 0001:00007f63       __NLG_Dispatch2            10008f63     libvcruntime:exsup.obj
 0001:00007f6b       __NLG_Call                 10008f6b f   libvcruntime:exsup.obj
 0001:00007f6d       __NLG_Return2              10008f6d     libvcruntime:exsup.obj
 0001:00007f70       __CallSettingFrame@12      10008f70 f   libvcruntime:lowhelpr.obj
 0001:00007f97       __NLG_Return               10008f97     libvcruntime:lowhelpr.obj
 0001:00007fbc       ___DestructExceptionObject 10008fbc f   libvcruntime:ehhelpers.obj
 0001:0000805c       ?_CallMemberFunction0@@YGXQAX0@Z 1000905c f i libvcruntime:ehhelpers.obj
 0001:00008070       _memmove                   10009070 f   libvcruntime:memmove.obj
 0001:000085e4       _free                      100095e4 f   libucrt:free.obj
 0001:00008601       _malloc                    10009601 f   libucrt:malloc.obj
 0001:0000860c       __seh_filter_dll           1000960c f   libucrt:exception_filter.obj
 0001:0000862c       __seh_filter_exe           1000962c f   libucrt:exception_filter.obj
 0001:000089ec       ___acrt_initialize_thread_local_exit_callback 100099ec f   libucrt:exit.obj
 0001:000089fb       __cexit                    100099fb f   libucrt:exit.obj
 0001:00008a0a       __exit                     10009a0a f   libucrt:exit.obj
 0001:00008a20       __is_c_termination_complete 10009a20 f   libucrt:exit.obj
 0001:00008cd8       ___acrt_allocate_buffer_for_argv 10009cd8 f   libucrt:argv_parsing.obj
 0001:00008d27       __configure_narrow_argv    10009d27 f   libucrt:argv_parsing.obj
 0001:00008e86       ??$uninitialize@A6AXAAPAPA_W@Z@?$dual_state_global@PAPA_W@__crt_state_management@@QAEXA6AXAAPAPA_W@Z@Z 10009e86 f i libucrt:environment_initialization.obj
 0001:00008e86       ??$uninitialize@A6AXAAPAPAD@Z@?$dual_state_global@PAPAD@__crt_state_management@@QAEXA6AXAAPAPAD@Z@Z 10009e86 f i libucrt:environment_initialization.obj
 0001:00008ee5       ___dcrt_uninitialize_environments_nolock 10009ee5 f   libucrt:environment_initialization.obj
 0001:00008f1c       __initialize_narrow_environment 10009f1c f   libucrt:environment_initialization.obj
 0001:00008fc3       ??$__crt_fast_encode_pointer@P6AHXZ@@YAP6AHXZQ6AHXZ@Z 10009fc3 f i libucrt:onexit.obj
 0001:000091ea       __crt_atexit               1000a1ea f   libucrt:onexit.obj
 0001:00009200       __execute_onexit_table     1000a200 f   libucrt:onexit.obj
 0001:0000922f       __initialize_onexit_table  1000a22f f   libucrt:onexit.obj
 0001:00009258       __register_onexit_function 1000a258 f   libucrt:onexit.obj
 0001:000092b4       ___acrt_uninitialize_command_line 1000a2b4 f   libucrt:argv_data.obj
 0001:0000938d       ___acrt_initialize         1000a38d f   libucrt:initialization.obj
 0001:0000939f       ___acrt_thread_attach      1000a39f f   libucrt:initialization.obj
 0001:000093aa       ___acrt_thread_detach      1000a3aa f   libucrt:initialization.obj
 0001:000093b2       ___acrt_uninitialize       1000a3b2 f   libucrt:initialization.obj
 0001:000093e2       ___acrt_uninitialize_critical 1000a3e2 f   libucrt:initialization.obj
 0001:000093f4       __initterm                 1000a3f4 f   libucrt:initterm.obj
 0001:0000943b       __initterm_e               1000a43b f   libucrt:initterm.obj
 0001:00009469       _terminate                 1000a469 f   libucrt:terminate.obj
 0001:000094a5       _strcpy_s                  1000a4a5 f   libucrt:strcpy_s.obj
 0001:000094ff       _abort                     1000a4ff f   libucrt:abort.obj
 0001:00009543       _calloc                    1000a543 f   libucrt:calloc.obj
 0001:0000954e       _wcsncmp                   1000a54e f   libucrt:wcsncmp.obj
 0001:00009588       ??0_LocaleUpdate@@QAE@QAU__crt_locale_pointers@@@Z 1000a588 f i libucrt:output.obj
 0001:0000960b       ___acrt_locale_get_ctype_array_value 1000a60b f i libucrt:output.obj
 0001:00009630       _strncmp                   1000a630 f   libucrt:strncmp.obj
 0001:000096a8       __free_base                1000a6a8 f   libucrt:free_base.obj
 0001:000096e2       __malloc_base              1000a6e2 f   libucrt:malloc_base.obj
 0001:00009a4a       ___acrt_freeptd            1000aa4a f   libucrt:per_thread_data.obj
 0001:00009a76       ___acrt_getptd             1000aa76 f   libucrt:per_thread_data.obj
 0001:00009b33       ___acrt_getptd_head        1000ab33 f   libucrt:per_thread_data.obj
 0001:00009bcd       ___acrt_getptd_noexit      1000abcd f   libucrt:per_thread_data.obj
 0001:00009c82       ___acrt_initialize_ptd     1000ac82 f   libucrt:per_thread_data.obj
 0001:00009cae       ___acrt_uninitialize_ptd   1000acae f   libucrt:per_thread_data.obj
 0001:00009cc8       ___acrt_initialize_locks   1000acc8 f   libucrt:locks.obj
 0001:00009d09       ___acrt_lock               1000ad09 f   libucrt:locks.obj
 0001:00009d20       ___acrt_uninitialize_locks 1000ad20 f   libucrt:locks.obj
 0001:00009d51       ___acrt_unlock             1000ad51 f   libucrt:locks.obj
 0001:00009d68       ___acrt_get_process_end_policy 1000ad68 f   libucrt:win_policies.obj
 0001:00009d9b       ___acrt_call_reportfault   1000ad9b f   libucrt:invalid_parameter.obj
 0001:00009ed6       ___acrt_initialize_invalid_parameter_handler 1000aed6 f   libucrt:invalid_parameter.obj
 0001:00009ee5       __invalid_parameter        1000aee5 f   libucrt:invalid_parameter.obj
 0001:00009f49       __invalid_parameter_noinfo 1000af49 f   libucrt:invalid_parameter.obj
 0001:00009f59       __invoke_watson            1000af59 f   libucrt:invalid_parameter.obj
 0001:00009f8d       ___acrt_errno_from_os_error 1000af8d f   libucrt:errno.obj
 0001:00009fd0       ___acrt_errno_map_os_error 1000afd0 f   libucrt:errno.obj
 0001:00009ff6       ___doserrno                1000aff6 f   libucrt:errno.obj
 0001:0000a009       __errno                    1000b009 f   libucrt:errno.obj
 0001:0000a01c       __calloc_base              1000b01c f   libucrt:calloc_base.obj
 0001:0000a212       ??$__acrt_mbs_to_wcs_cp@U__crt_win32_buffer_internal_dynamic_resizing@@@@YAHQBDAAV?$__crt_win32_buffer@_WU__crt_win32_buffer_internal_dynamic_resizing@@@@I@Z 1000b212 f i libucrt:argv_wildcards.obj
 0001:0000a72e       ?__acrt_get_utf8_acp_compatibility_codepage@@YAIXZ 1000b72e f i libucrt:argv_wildcards.obj
 0001:0000a76f       ?_deallocate@?$__crt_win32_buffer@_WU__crt_win32_buffer_internal_dynamic_resizing@@@@AAEXXZ 1000b76f f i libucrt:argv_wildcards.obj
 0001:0000a76f       ?_deallocate@?$__crt_win32_buffer@DU__crt_win32_buffer_internal_dynamic_resizing@@@@AAEXXZ 1000b76f f i libucrt:argv_wildcards.obj
 0001:0000a789       ?allocate@?$__crt_win32_buffer@DU__crt_win32_buffer_internal_dynamic_resizing@@@@QAEHI@Z 1000b789 f i libucrt:argv_wildcards.obj
 0001:0000a7c5       ?allocate@?$__crt_win32_buffer@_WU__crt_win32_buffer_internal_dynamic_resizing@@@@QAEHI@Z 1000b7c5 f i libucrt:argv_wildcards.obj
 0001:0000a804       ?allocate@__crt_win32_buffer_internal_dynamic_resizing@@SAHQAPAXIABV__crt_win32_buffer_empty_debug_info@@@Z 1000b804 f i libucrt:argv_wildcards.obj
 0001:0000a8aa       ___acrt_expand_narrow_argv_wildcards 1000b8aa f   libucrt:argv_wildcards.obj
 0001:0000a97c       ?allocate@?$__crt_win32_buffer@DU__crt_win32_buffer_no_resizing@@@@QAEHI@Z 1000b97c f i libucrt:getmodulefilenamea.obj
 0001:0000a9a3       ?set_to_nullptr@?$__crt_win32_buffer@DU__crt_win32_buffer_no_resizing@@@@QAEXXZ 1000b9a3 f i libucrt:getmodulefilenamea.obj
 0001:0000a9b7       ___acrt_GetModuleFileNameA 1000b9b7 f   libucrt:getmodulefilenamea.obj
 0001:0000af6a       ___acrt_initialize_multibyte 1000bf6a f   libucrt:mbctype.obj
 0001:0000afb2       ___acrt_update_thread_multibyte_data 1000bfb2 f   libucrt:mbctype.obj
 0001:0000afc5       __setmbcp_nolock           1000bfc5 f   libucrt:mbctype.obj
 0001:0000b294       __ismbblead                1000c294 f   libucrt:ismbbyte.obj
 0001:0000b2ac       ___acrt_initialize_command_line 1000c2ac f   libucrt:argv_data.obj
 0001:0000b2c5       ___acrt_MultiByteToWideChar 1000c2c5 f   libucrt:multibytetowidechar.obj
 0001:0000b341       ___acrt_WideCharToMultiByte 1000c341 f   libucrt:widechartomultibyte.obj
 0001:0000b425       ___dcrt_get_narrow_environment_from_os 1000c425 f   libucrt:get_environment_from_os.obj
 0001:0000b4ab       __recalloc_base            1000c4ab f   libucrt:recalloc.obj
 0001:0000b684       ___acrt_initialize_lowio   1000c684 f   libucrt:ioinit.obj
 0001:0000b6da       ___acrt_uninitialize_lowio 1000c6da f   libucrt:ioinit.obj
 0001:0000b8a0       ___acrt_AppPolicyGetProcessTerminationMethodInternal@4 1000c8a0 f   libucrt:winapi_thunks.obj
 0001:0000b8e0       ___acrt_AreFileApisANSI@0  1000c8e0 f   libucrt:winapi_thunks.obj
 0001:0000b8ff       ___acrt_FlsAlloc@4         1000c8ff f   libucrt:winapi_thunks.obj
 0001:0000b93e       ___acrt_FlsFree@4          1000c93e f   libucrt:winapi_thunks.obj
 0001:0000b97d       ___acrt_FlsGetValue@4      1000c97d f   libucrt:winapi_thunks.obj
 0001:0000b9bc       ___acrt_FlsSetValue@8      1000c9bc f   libucrt:winapi_thunks.obj
 0001:0000b9fe       ___acrt_InitializeCriticalSectionEx@12 1000c9fe f   libucrt:winapi_thunks.obj
 0001:0000ba49       ___acrt_LCMapStringEx@36   1000ca49 f   libucrt:winapi_thunks.obj
 0001:0000baa6       ___acrt_LocaleNameToLCID@8 1000caa6 f   libucrt:winapi_thunks.obj
 0001:0000bad7       ___acrt_initialize_winapi_thunks 1000cad7 f   libucrt:winapi_thunks.obj
 0001:0000bb02       ___acrt_uninitialize_winapi_thunks 1000cb02 f   libucrt:winapi_thunks.obj
 0001:0000bb38       ___acrt_initialize_heap    1000cb38 f   libucrt:heap_handle.obj
 0001:0000bb49       ___acrt_uninitialize_heap  1000cb49 f   libucrt:heap_handle.obj
 0001:0000bb53       ___acrt_execute_initializers 1000cb53 f   libucrt:shared_initialization.obj
 0001:0000bbbb       ___acrt_execute_uninitializers 1000cbbb f   libucrt:shared_initialization.obj
 0001:0000bbec       ___acrt_initialize_new_handler 1000cbec f   libucrt:new_handler.obj
 0001:0000bbfb       __callnewh                 1000cbfb f   libucrt:new_handler.obj
 0001:0000bc28       __query_new_handler        1000cc28 f   libucrt:new_handler.obj
 0001:0000bd3e       ___acrt_get_sigabrt_handler 1000cd3e f   libucrt:signal.obj
 0001:0000bd67       ___acrt_initialize_signal_handlers 1000cd67 f   libucrt:signal.obj
 0001:0000bd85       ___fpecode                 1000cd85 f   libucrt:signal.obj
 0001:0000bd8e       _raise                     1000cd8e f   libucrt:signal.obj
 0001:0000bf75       ___acrt_has_user_matherr   1000cf75 f   libucrt:matherr.obj
 0001:0000bf8d       ___acrt_initialize_user_matherr 1000cf8d f   libucrt:matherr.obj
 0001:0000bf9c       ___acrt_invoke_user_matherr 1000cf9c f   libucrt:matherr.obj
 0001:0000c199       ___acrt_stdio_flush_nolock 1000d199 f   libucrt:fflush.obj
 0001:0000c1fe       __fflush_nolock            1000d1fe f   libucrt:fflush.obj
 0001:0000c246       __flushall                 1000d246 f   libucrt:fflush.obj
 0001:0000c24f       ___acrt_initialize_stdio   1000d24f f   libucrt:_file.obj
 0001:0000c317       ___acrt_uninitialize_stdio 1000d317 f   libucrt:_file.obj
 0001:0000c363       __lock_file                1000d363 f   libucrt:_file.obj
 0001:0000c377       __unlock_file              1000d377 f   libucrt:_file.obj
 0001:0000c38b       __mbtowc_l                 1000d38b f   libucrt:mbtowc.obj
 0001:0000c4cf       _mbtowc                    1000d4cf f   libucrt:mbtowc.obj
 0001:0000c4e9       ___acrt_update_locale_info 1000d4e9 f   libucrt:locale_update.obj
 0001:0000c516       ___acrt_update_multibyte_info 1000d516 f   libucrt:locale_update.obj
 0001:0000c543       __fileno                   1000d543 f   libucrt:fileno.obj
 0001:0000c5ce       ___acrt_set_locale_changed 1000d5ce f   libucrt:wsetlocale.obj
 0001:0000c5d9       ___acrt_uninitialize_locale 1000d5d9 f   libucrt:wsetlocale.obj
 0001:0000c602       ___pctype_func             1000d602 f   libucrt:ctype.obj
 0001:0000c628       __query_new_mode           1000d628 f   libucrt:new_mode.obj
 0001:0000c62f       ___acrt_add_locale_ref     1000d62f f   libucrt:locale_refcounting.obj
 0001:0000c6ac       ___acrt_free_locale        1000d6ac f   libucrt:locale_refcounting.obj
 0001:0000c7f6       ___acrt_locale_add_lc_time_reference 1000d7f6 f   libucrt:locale_refcounting.obj
 0001:0000c81f       ___acrt_locale_free_lc_time_if_unreferenced 1000d81f f   libucrt:locale_refcounting.obj
 0001:0000c850       ___acrt_locale_release_lc_time_reference 1000d850 f   libucrt:locale_refcounting.obj
 0001:0000c879       ___acrt_release_locale_ref 1000d879 f   libucrt:locale_refcounting.obj
 0001:0000c8fa       ___acrt_update_thread_locale_data 1000d8fa f   libucrt:locale_refcounting.obj
 0001:0000c971       __updatetlocinfoEx_nolock  1000d971 f   libucrt:locale_refcounting.obj
 0001:0000ca10       _qsort                     1000da10 f   libucrt:qsort.obj
 0001:0000cf07       _strncpy_s                 1000df07 f   libucrt:strncpy_s.obj
 0001:0000cf20       _strpbrk                   1000df20 f   libucrt:strpbrk.obj
 0001:0000cf60       __mbsdec                   1000df60 f   libucrt:mbsdec.obj
 0001:0000cf77       __mbsdec_l                 1000df77 f   libucrt:mbsdec.obj
 0001:0000d006       ___acrt_GetStringTypeA     1000e006 f   libucrt:getstringtypea.obj
 0001:0000d10b       __freea_crt                1000e10b f i libucrt:getstringtypea.obj
 0001:0000d317       ___acrt_LCMapStringA       1000e317 f   libucrt:lcmapstringa.obj
 0001:0000d371       __msize_base               1000e371 f   libucrt:msize.obj
 0001:0000d3a4       __realloc_base             1000e3a4 f   libucrt:realloc_base.obj
 0001:0000d40d       ___acrt_lowio_create_handle_array 1000e40d f   libucrt:osfinfo.obj
 0001:0000d48a       ___acrt_lowio_destroy_handle_array 1000e48a f   libucrt:osfinfo.obj
 0001:0000d4bf       ___acrt_lowio_ensure_fh_exists 1000e4bf f   libucrt:osfinfo.obj
 0001:0000d553       ___acrt_lowio_lock_fh      1000e553 f   libucrt:osfinfo.obj
 0001:0000d576       ___acrt_lowio_unlock_fh    1000e576 f   libucrt:osfinfo.obj
 0001:0000d599       __free_osfhnd              1000e599 f   libucrt:osfinfo.obj
 0001:0000d62a       __get_osfhandle            1000e62a f   libucrt:osfinfo.obj
 0001:0000d748       ___acrt_DownlevelLocaleNameToLCID 1000e748 f   libucrt:lcidtoname_downlevel.obj
 0001:0000d80c       __commit                   1000e80c f   libucrt:commit.obj
 0001:0000e010       __write                    1000f010 f   libucrt:write.obj
 0001:0000e0f8       __write_nolock             1000f0f8 f   libucrt:write.obj
 0001:0000e2dc       __fcloseall                1000f2dc f   libucrt:closeall.obj
 0001:0000e37d       ___acrt_stdio_free_buffer_nolock 1000f37d f   libucrt:_freebuf.obj
 0001:0000e3bd       __isatty                   1000f3bd f   libucrt:isatty.obj
 0001:0000e413       __isleadbyte_l             1000f413 f i libucrt:_wctype.obj
 0001:0000e47b       ?__mbrtowc_utf8@__crt_mbstring@@YAIPA_WPBDIPAU_Mbstatet@@@Z 1000f47b f   libucrt:mbrtowc.obj
 0001:0000e4bd       ?__mbsrtowcs_utf8@__crt_mbstring@@YAIPA_WPAPBDIPAU_Mbstatet@@@Z 1000f4bd f   libucrt:mbrtowc.obj
 0001:0000e5ba       ?return_illegal_sequence@__crt_mbstring@@YAIPAU_Mbstatet@@@Z 1000f5ba f i libucrt:c32rtomb.obj
 0001:0000e5d9       ___acrt_locale_free_monetary 1000f5d9 f   libucrt:initmon.obj
 0001:0000e6d7       ___acrt_locale_free_numeric 1000f6d7 f   libucrt:initnum.obj
 0001:0000e778       ___acrt_locale_free_time   1000f778 f   libucrt:inittime.obj
 0001:0000e85c       ___strncnt                 1000f85c f   libucrt:strncnt.obj
 0001:0000e878       __query_app_type           1000f878 f   libucrt:report_runtime_error.obj
 0001:0000e8fc       __lseeki64_nolock          1000f8fc f   libucrt:lseek.obj
 0001:0000e917       __putwch_nolock            1000f917 f   libucrt:putwch.obj
 0001:0000e94b       __fclose_nolock            1000f94b f   libucrt:fclose.obj
 0001:0000e9c2       _fclose                    1000f9c2 f   libucrt:fclose.obj
 0001:0000ea3c       ?__mbrtoc32_utf8@__crt_mbstring@@YAIPA_UPBDIPAU_Mbstatet@@@Z 1000fa3c f   libucrt:mbrtoc32.obj
 0001:0000ebf0       __CIlog10                  1000fbf0 f   libucrt:log10_impl.obj
 0001:0000ec2b       __CIlog10_default          1000fc2b f   libucrt:log10_impl.obj
 0001:0000ec3f       __log10_default            1000fc3f     libucrt:log10_impl.obj
 0001:0000ed00       _ceil                      1000fd00 f   libucrt:ceil_pentium4.obj
 0001:0000ed40       __ceil_pentium4            1000fd40 f   libucrt:ceil_pentium4.obj
 0001:0000ee20       ___ascii_strnicmp          1000fe20 f   libucrt:_strnicm.obj
 0001:0000eea0       ___dcrt_lowio_ensure_console_output_initialized 1000fea0 f   libucrt:initcon.obj
 0001:0000eebf       ___dcrt_terminate_console_output 1000febf f   libucrt:initcon.obj
 0001:0000eed6       ___dcrt_write_console      1000fed6 f   libucrt:initcon.obj
 0001:0000efad       __close                    1000ffad f   libucrt:close.obj
 0001:0000f03c       __close_nolock             1001003c f   libucrt:close.obj
 0001:0000f0d8       ?__acrt_stdio_free_stream@@YAXV__crt_stdio_stream@@@Z 100100d8 f   libucrt:stream.obj
 0001:0000f113       ___acrt_initialize_sse2    10010113 f   libucrt:mathfcns.obj
 0001:0000f130       __CIlog10_pentium4         10010130 f   libucrt:log10_pentium4.obj
 0001:0000f148       __log10_pentium4           10010148     libucrt:log10_pentium4.obj
 0001:0000f3e0       __fFEXP                    100103e0 f   libucrt:87tran.obj
 0001:0000f437       __rtinfpopse               10010437     libucrt:87tran.obj
 0001:0000f439       __rtinfnpopse              10010439     libucrt:87tran.obj
 0001:0000f449       __fFLN                     10010449     libucrt:87tran.obj
 0001:0000f4fe       __rtinfpop                 100104fe     libucrt:87tran.obj
 0001:0000f500       __rtinfnpop                10010500     libucrt:87tran.obj
 0001:0000f510       __rtforexpinf              10010510 f   libucrt:87tran.obj
 0001:0000f51d       __ffexpm1                  1001051d     libucrt:87tran.obj
 0001:0000f5d0       __trandisp1                100105d0 f   libucrt:87disp.obj
 0001:0000f645       __trandisp2                10010645 f   libucrt:87disp.obj
 0001:0000f6df       __rttospopde               100106df     libucrt:87disp.obj
 0001:0000f6e4       __rttospop                 100106e4     libucrt:87disp.obj
 0001:0000f6f0       __rtnospop                 100106f0 f   libucrt:87disp.obj
 0001:0000f700       __rttosnpop                10010700 f   libucrt:87disp.obj
 0001:0000f701       __rtnospopde               10010701     libucrt:87disp.obj
 0001:0000f708       __rtzeropop                10010708     libucrt:87disp.obj
 0001:0000f70a       __rtzeronpop               1001070a     libucrt:87disp.obj
 0001:0000f710       __rtzerospop               10010710 f   libucrt:87disp.obj
 0001:0000f71d       __rtonepop                 1001071d     libucrt:87disp.obj
 0001:0000f720       __rtonenpop                10010720 f   libucrt:87disp.obj
 0001:0000f730       __tosnan1                  10010730 f   libucrt:87disp.obj
 0001:0000f760       __nosnan2                  10010760 f   libucrt:87disp.obj
 0001:0000f770       __tosnan2                  10010770 f   libucrt:87disp.obj
 0001:0000f7a0       __nan2                     100107a0 f   libucrt:87disp.obj
 0001:0000f7e0       __rtindfpop                100107e0 f   libucrt:87disp.obj
 0001:0000f7e2       __rtindfnpop               100107e2     libucrt:87disp.obj
 0001:0000f7f3       __rttosnpopde              100107f3     libucrt:87disp.obj
 0001:0000f800       __rtatan2inf               10010800 f   libucrt:87disp.obj
 0001:0000f81d       __rtchsifneg               1001081d     libucrt:87disp.obj
 0001:0000f830       __twoToTOS                 10010830 f   libucrt:common.obj
 0001:0000f845       __load_CW                  10010845 f   libucrt:common.obj
 0001:0000f85c       __convertTOStoQNaN         1001085c f   libucrt:common.obj
 0001:0000f875       __fload_withFB             10010875 f   libucrt:common.obj
 0001:0000f8b8       __checkTOS_withFB          100108b8 f   libucrt:common.obj
 0001:0000f8ce       __fast_exit                100108ce f   libucrt:common.obj
 0001:0000f8db       __math_exit                100108db f   libucrt:common.obj
 0001:0000f905       __check_overflow_exit      10010905 f   libucrt:common.obj
 0001:0000f919       __check_range_exit         10010919 f   libucrt:common.obj
 0001:0000f9c0       __startTwoArgErrorHandling 100109c0 f   libucrt:genexcep.obj
 0001:0000f9d7       __startOneArgErrorHandling 100109d7 f   libucrt:genexcep.obj
 0001:0000fa13       ___libm_error_support      10010a13 f   libucrt:libm_error.obj
 0001:0000fc09       __ceil_default             10010c09 f   libucrt:ceil.obj
 0001:0000fcc0       __clrfp                    10010cc0 f   libucrt:fpctrl.obj
 0001:0000fcd3       __ctrlfp                   10010cd3 f   libucrt:fpctrl.obj
 0001:0000fcff       __set_statfp               10010cff f   libucrt:fpctrl.obj
 0001:0000fd5a       __statfp                   10010d5a f   libucrt:fpctrl.obj
 0001:0000fd6c       __d_inttype                10010d6c f   libucrt:powhlp.obj
 0001:0000fdd6       __powhlp                   10010dd6 f   libucrt:powhlp.obj
 0001:0000ff01       __87except                 10010f01 f   libucrt:87except.obj
 0001:0001000b       __frnd                     1001100b f   libucrt:frnd.obj
 0001:00010021       __errcode                  10011021 f   libucrt:fpexcept.obj
 0001:00010055       __except1                  10011055 f   libucrt:fpexcept.obj
 0001:00010123       __handle_exc               10011123 f   libucrt:fpexcept.obj
 0001:00010310       __raise_exc                10011310 f   libucrt:fpexcept.obj
 0001:00010333       __raise_exc_ex             10011333 f   libucrt:fpexcept.obj
 0001:00010629       __set_errno_from_matherr   10011629 f   libucrt:fpexcept.obj
 0001:00010658       __umatherr                 10011658 f   libucrt:fpexcept.obj
 0001:000106fa       __decomp                   100116fa f   libucrt:util.obj
 0001:000107d8       __set_exp                  100117d8 f   libucrt:util.obj
 0001:00010807       __sptype                   10011807 f   libucrt:util.obj
 0001:00010865       __fpclass                  10011865 f   libucrt:ieeemisc.obj
 0001:00010909       _IsProcessorFeaturePresent@4 10011909 f   kernel32:KERNEL32.dll
 0001:00010910       __FindPESection            10011910 f   LIBCMT:pesect.obj
 0001:00010960       __IsNonwritableInCurrentImage 10011960 f   LIBCMT:pesect.obj
 0001:00010a20       __ValidateImageBase        10011a20 f   LIBCMT:pesect.obj
 0001:00010a60       __aulldvrm                 10011a60 f   LIBCMT:ulldvrm.obj
 0001:00010b00       __allmul                   10011b00 f   LIBCMT:llmul.obj
 0001:00010b40       __alldvrm                  10011b40 f   LIBCMT:lldvrm.obj
 0001:00010c20       __aullshr                  10011c20 f   LIBCMT:ullshr.obj
 0001:00010c40       __alloca_probe_16          10011c40 f   LIBCMT:alloca16.obj
 0001:00010c56       __alloca_probe_8           10011c56     LIBCMT:alloca16.obj
 0001:00010c70       __allshl                   10011c70 f   LIBCMT:llshl.obj
 0001:00010c90       __ftol2_sse                10011c90 f   LIBCMT:ftol2.obj
 0001:00010c99       __ftol2_pentium4           10011c99 f   LIBCMT:ftol2.obj
 0001:00010cac       __ftol2_sse_excpt          10011cac f   LIBCMT:ftol2.obj
 0001:00010cd0       __ftol2                    10011cd0 f   LIBCMT:ftol2.obj
 0001:00010d50       _strchr                    10011d50 f   libvcruntime:strchr.obj
 0001:00010dbe       ___from_strstr_to_strchr   10011dbe     libvcruntime:strchr.obj
 0001:00010e80       _strrchr                   10011e80 f   libvcruntime:strrchr.obj
 0002:00000190       ___scrt_native_dllmain_reason 10013190     LIBCMT:utility.obj
 0002:00000194       ___isa_enabled             10013194     LIBCMT:cpu_disp.obj
 0002:000001a0       ___security_cookie_complement 100131a0     LIBCMT:gs_cookie.obj
 0002:000001a4       ___security_cookie         100131a4     LIBCMT:gs_cookie.obj
 0002:000001c0       __NLG_Destination          100131c0     libvcruntime:exsup.obj
 0002:000001d0       ___abort_behavior          100131d0     libucrt:abort.obj
 0002:000001f0       ___acrt_initial_multibyte_data 100131f0     libucrt:mbctype.obj
 0002:00000710       ___acrt_initial_locale_data 10013710     libucrt:nlsdata.obj
 0002:000007c8       ___acrt_initial_locale_pointers 100137c8     libucrt:nlsdata.obj
 0002:000007d0       ___acrt_wide_c_locale_string 100137d0     libucrt:nlsdata.obj
 0002:000007d8       __iob                      100137d8     libucrt:_file.obj
 0002:00000880       ___globallocalestatus      10013880     libucrt:glstatus.obj
 0002:00000888       ___acrt_lconv_c            10013888     libucrt:localeconv.obj
 0002:000008d8       ___acrt_lconv_static_decimal 100138d8     libucrt:localeconv.obj
 0002:000008dc       ___acrt_lconv_static_W_decimal 100138dc     libucrt:localeconv.obj
 0002:000008e0       __lookuptrailbytes         100138e0     libucrt:read.obj
 0002:000009f0       __fltused                  100139f0     LIBCMT:fltused.obj
 0002:00000a94       ?Ptr@?1???R<lambda_1af49d8e19f959e583a46d83b89ae789>@@QBE@XZ@4PAXA 10013a94     vc_crt_fix_impl.obj
 0002:00000b24       ___scrt_current_native_startup_state 10013b24     LIBCMT:utility.obj
 0002:00000b28       ___scrt_native_startup_lock 10013b28     LIBCMT:utility.obj
 0002:00000b4c       ___isa_available           10013b4c     LIBCMT:cpu_disp.obj
 0002:00000b50       ___favor                   10013b50     LIBCMT:cpu_disp.obj
 0002:00000b54       ___scrt_debugger_hook_flag 10013b54     LIBCMT:utility_desktop.obj
 0002:00000b58       ?__type_info_root_node@@3U__type_info_node@@A 10013b58     LIBCMT:tncleanup.obj
 0002:00000b60       ?_OptionsStorage@?1??__local_stdio_printf_options@@9@4_KA 10013b60     LIBCMT:default_local_stdio_options.obj
 0002:00000b68       ?_OptionsStorage@?1??__local_stdio_scanf_options@@9@4_KA 10013b68     LIBCMT:default_local_stdio_options.obj
 0002:00000ef0       ___pPurecall               10013ef0     libvcruntime:purevirt_data.obj
 0002:00000ef4       ?pArgList@UnDecorator@@0PAVReplicator@@A 10013ef4     libvcruntime:undname.obj
 0002:00000ef8       ?pZNameList@UnDecorator@@0PAVReplicator@@A 10013ef8     libvcruntime:undname.obj
 0002:00000efc       ?pTemplateArgList@UnDecorator@@0PAVReplicator@@A 10013efc     libvcruntime:undname.obj
 0002:00000f00       ?gName@UnDecorator@@0PBDB  10013f00     libvcruntime:undname.obj
 0002:00000f04       ?name@UnDecorator@@0PBDB   10013f04     libvcruntime:undname.obj
 0002:00000f08       ?disableFlags@UnDecorator@@0KA 10013f08     libvcruntime:undname.obj
 0002:00000f0c       ?fExplicitTemplateParams@UnDecorator@@0_NA 10013f0c     libvcruntime:undname.obj
 0002:00000f0d       ?fGetTemplateArgumentList@UnDecorator@@0_NA 10013f0d     libvcruntime:undname.obj
 0002:00000f10       ?m_pGetParameter@UnDecorator@@0P6APADJ@ZA 10013f10     libvcruntime:undname.obj
 0002:00000f14       ?m_CHPENameOffset@UnDecorator@@0KA 10013f14     libvcruntime:undname.obj
 0002:00000f18       ?m_recursionLevel@UnDecorator@@0KA 10013f18     libvcruntime:undname.obj
 0002:00000f30       ?__WinRTOutOfMemoryExceptionCallback@@3P6GPAXXZA 10013f30     libvcruntime:ehhelpers.obj
 0002:00000f3c       ?c_exit_complete@?1???R<lambda_6e4b09c48022b2350581041d5f6b0c4c>@@QBE@XZ@4_NA 10013f3c     libucrt:exit.obj
 0002:00001048       __environ_table            10014048     libucrt:environment_initialization.obj
 0002:0000104c       __wenviron_table           1001404c     libucrt:environment_initialization.obj
 0002:00001050       ___dcrt_initial_wide_environment 10014050     libucrt:environment_initialization.obj
 0002:00001054       ___dcrt_initial_narrow_environment 10014054     libucrt:environment_initialization.obj
 0002:00001058       ___acrt_atexit_table       10014058     libucrt:onexit.obj
 0002:00001064       ___acrt_at_quick_exit_table 10014064     libucrt:onexit.obj
 0002:000011c8       ___acrt_current_multibyte_data 100141c8     libucrt:mbctype.obj
 0002:000011cc       __mbctype                  100141cc     libucrt:mbctype.obj
 0002:000011d0       __mbcasemap                100141d0     libucrt:mbctype.obj
 0002:000011dc       __pgmptr                   100141dc     libucrt:argv_data.obj
 0002:000011e0       ___argc                    100141e0     libucrt:argv_data.obj
 0002:000011e4       ___argv                    100141e4     libucrt:argv_data.obj
 0002:000011e8       ___wargv                   100141e8     libucrt:argv_data.obj
 0002:000011ec       __acmdln                   100141ec     libucrt:argv_data.obj
 0002:000011f0       __wcmdln                   100141f0     libucrt:argv_data.obj
 0002:000011f8       ___pioinfo                 100141f8     libucrt:ioinit.obj
 0002:000013f8       __nhandle                  100143f8     libucrt:ioinit.obj
 0002:000014d8       ___acrt_heap               100144d8     libucrt:heap_handle.obj
 0002:000014f4       ___acrt_current_locale_data 100144f4     libucrt:nlsdata.obj
 0002:000014f8       __nstream                  100144f8     libucrt:_file.obj
 0002:000014fc       ___piob                    100144fc     libucrt:_file.obj
 0002:00001500       ___acrt_stdout_buffer      10014500     libucrt:_sftbuf.obj
 0002:00001504       ___acrt_stderr_buffer      10014504     libucrt:_sftbuf.obj
 0002:00001510       ___acrt_locale_changed_data 10014510     libucrt:wsetlocale.obj
 0002:00001518       ___acrt_lconv_static_null  10014518     libucrt:localeconv.obj
 0002:0000151c       ___acrt_lconv_static_W_null 1001451c     libucrt:localeconv.obj
 0002:0000152c       ___fastflag                1001452c     libucrt:fp_flags.obj
 0002:00001534       ___dyn_tls_init_callback   10014534     <common>
 0002:00001538       ___scrt_ucrt_dll_is_in_use 10014538     <common>
 0002:0000153c       __pmatherr                 1001453c     <common>
 0002:00001540       ___use_sse2_mathfcns       10014540     <common>
 0003:00000000       __imp__SetLastError@4      10015000     kernel32:KERNEL32.dll
 0003:00000004       __imp__InitializeCriticalSection@4 10015004     kernel32:KERNEL32.dll
 0003:00000008       __imp__EnterCriticalSection@4 10015008     kernel32:KERNEL32.dll
 0003:0000000c       __imp__LeaveCriticalSection@4 1001500c     kernel32:KERNEL32.dll
 0003:00000010       __imp__DeleteCriticalSection@4 10015010     kernel32:KERNEL32.dll
 0003:00000014       __imp__GetCurrentThread@0  10015014     kernel32:KERNEL32.dll
 0003:00000018       __imp__GetThreadTimes@20   10015018     kernel32:KERNEL32.dll
 0003:0000001c       __imp__VirtualQuery@12     1001501c     kernel32:KERNEL32.dll
 0003:00000020       __imp__GetModuleFileNameW@12 10015020     kernel32:KERNEL32.dll
 0003:00000024       __imp__GetModuleHandleW@4  10015024     kernel32:KERNEL32.dll
 0003:00000028       __imp__GetProcAddress@8    10015028     kernel32:KERNEL32.dll
 0003:0000002c       __imp__LoadLibraryW@4      1001502c     kernel32:KERNEL32.dll
 0003:00000030       __imp__CloseHandle@4       10015030     kernel32:KERNEL32.dll
 0003:00000034       __imp__IsProcessorFeaturePresent@4 10015034     kernel32:KERNEL32.dll
 0003:00000038       __imp__IsDebuggerPresent@0 10015038     kernel32:KERNEL32.dll
 0003:0000003c       __imp__UnhandledExceptionFilter@4 1001503c     kernel32:KERNEL32.dll
 0003:00000040       __imp__SetUnhandledExceptionFilter@4 10015040     kernel32:KERNEL32.dll
 0003:00000044       __imp__GetStartupInfoW@4   10015044     kernel32:KERNEL32.dll
 0003:00000048       __imp__QueryPerformanceCounter@4 10015048     kernel32:KERNEL32.dll
 0003:0000004c       __imp__GetCurrentProcessId@0 1001504c     kernel32:KERNEL32.dll
 0003:00000050       __imp__GetCurrentThreadId@0 10015050     kernel32:KERNEL32.dll
 0003:00000054       __imp__GetSystemTimeAsFileTime@4 10015054     kernel32:KERNEL32.dll
 0003:00000058       __imp__GetCurrentProcess@0 10015058     kernel32:KERNEL32.dll
 0003:0000005c       __imp__TerminateProcess@8  1001505c     kernel32:KERNEL32.dll
 0003:00000060       __imp__GetLastError@0      10015060     kernel32:KERNEL32.dll
 0003:00000064       __imp__InitializeCriticalSectionAndSpinCount@8 10015064     kernel32:KERNEL32.dll
 0003:00000068       __imp__TlsAlloc@0          10015068     kernel32:KERNEL32.dll
 0003:0000006c       __imp__TlsGetValue@4       1001506c     kernel32:KERNEL32.dll
 0003:00000070       __imp__TlsSetValue@8       10015070     kernel32:KERNEL32.dll
 0003:00000074       __imp__TlsFree@4           10015074     kernel32:KERNEL32.dll
 0003:00000078       __imp__FreeLibrary@4       10015078     kernel32:KERNEL32.dll
 0003:0000007c       __imp__LoadLibraryExW@12   1001507c     kernel32:KERNEL32.dll
 0003:00000080       __imp__RtlUnwind@16        10015080     kernel32:KERNEL32.dll
 0003:00000084       __imp__RaiseException@16   10015084     kernel32:KERNEL32.dll
 0003:00000088       __imp__ExitProcess@4       10015088     kernel32:KERNEL32.dll
 0003:0000008c       __imp__HeapFree@12         1001508c     kernel32:KERNEL32.dll
 0003:00000090       __imp__HeapAlloc@12        10015090     kernel32:KERNEL32.dll
 0003:00000094       __imp__FindClose@4         10015094     kernel32:KERNEL32.dll
 0003:00000098       __imp__FindFirstFileExW@24 10015098     kernel32:KERNEL32.dll
 0003:0000009c       __imp__FindNextFileW@8     1001509c     kernel32:KERNEL32.dll
 0003:000000a0       __imp__IsValidCodePage@4   100150a0     kernel32:KERNEL32.dll
 0003:000000a4       __imp__GetACP@0            100150a4     kernel32:KERNEL32.dll
 0003:000000a8       __imp__GetOEMCP@0          100150a8     kernel32:KERNEL32.dll
 0003:000000ac       __imp__GetCPInfo@8         100150ac     kernel32:KERNEL32.dll
 0003:000000b0       __imp__GetCommandLineA@0   100150b0     kernel32:KERNEL32.dll
 0003:000000b4       __imp__GetCommandLineW@0   100150b4     kernel32:KERNEL32.dll
 0003:000000b8       __imp__MultiByteToWideChar@24 100150b8     kernel32:KERNEL32.dll
 0003:000000bc       __imp__WideCharToMultiByte@32 100150bc     kernel32:KERNEL32.dll
 0003:000000c0       __imp__GetEnvironmentStringsW@0 100150c0     kernel32:KERNEL32.dll
 0003:000000c4       __imp__FreeEnvironmentStringsW@4 100150c4     kernel32:KERNEL32.dll
 0003:000000c8       __imp__GetStdHandle@4      100150c8     kernel32:KERNEL32.dll
 0003:000000cc       __imp__GetFileType@4       100150cc     kernel32:KERNEL32.dll
 0003:000000d0       __imp__LCMapStringW@24     100150d0     kernel32:KERNEL32.dll
 0003:000000d4       __imp__GetProcessHeap@0    100150d4     kernel32:KERNEL32.dll
 0003:000000d8       __imp__GetStringTypeW@16   100150d8     kernel32:KERNEL32.dll
 0003:000000dc       __imp__HeapSize@12         100150dc     kernel32:KERNEL32.dll
 0003:000000e0       __imp__HeapReAlloc@16      100150e0     kernel32:KERNEL32.dll
 0003:000000e4       __imp__SetStdHandle@8      100150e4     kernel32:KERNEL32.dll
 0003:000000e8       __imp__FlushFileBuffers@4  100150e8     kernel32:KERNEL32.dll
 0003:000000ec       __imp__WriteFile@20        100150ec     kernel32:KERNEL32.dll
 0003:000000f0       __imp__GetConsoleCP@0      100150f0     kernel32:KERNEL32.dll
 0003:000000f4       __imp__GetConsoleMode@8    100150f4     kernel32:KERNEL32.dll
 0003:000000f8       __imp__SetFilePointerEx@20 100150f8     kernel32:KERNEL32.dll
 0003:000000fc       __imp__CreateFileW@28      100150fc     kernel32:KERNEL32.dll
 0003:00000100       __imp__WriteConsoleW@20    10015100     kernel32:KERNEL32.dll
 0003:00000104       \177KERNEL32_NULL_THUNK_DATA 10015104     kernel32:KERNEL32.dll
 0003:00000108       ___guard_check_icall_fptr  10015108     LIBCMT:guard_support.obj
 0003:0000010c       __IMPORT_DESCRIPTOR_KERNEL32 1001510c     kernel32:KERNEL32.dll
 0003:00000120       __NULL_IMPORT_DESCRIPTOR   10015120     kernel32:KERNEL32.dll

 entry point at        0001:00006926

 Static symbols

 0001:00000120       ?kernel32@modules@@3QB_WB  10001120     vc_crt_fix_impl.obj
 0001:00000134       ?ntdll@modules@@3QB_WB     10001134     vc_crt_fix_impl.obj
 0001:00000258       _GS_ExceptionPointers      10001258     LIBCMT:gs_report.obj
 0001:00000260       ?module_names@?A0x5c520fe1@@3QBQB_WB 10001260     libvcruntime:winapi_downlevel.obj
 0001:00000318       ?candidate_modules@?1??try_get_FlsAlloc@@YAP6GKP6GXPAX@Z@ZXZ@4QBW4module_id@?A0x5c520fe1@@B 10001318     libvcruntime:winapi_downlevel.obj
 0001:0000032c       ?candidate_modules@?1??try_get_FlsFree@@YAP6GHK@ZXZ@4QBW4module_id@?A0x5c520fe1@@B 1000132c     libvcruntime:winapi_downlevel.obj
 0001:0000033c       ?candidate_modules@?1??try_get_FlsGetValue@@YAP6GPAXK@ZXZ@4QBW4module_id@?A0x5c520fe1@@B 1000133c     libvcruntime:winapi_downlevel.obj
 0001:00000350       ?candidate_modules@?1??try_get_FlsSetValue@@YAP6GHKPAX@ZXZ@4QBW4module_id@?A0x5c520fe1@@B 10001350     libvcruntime:winapi_downlevel.obj
 0001:00000364       ?candidate_modules@?1??try_get_InitializeCriticalSectionEx@@YAP6GHPAU_RTL_CRITICAL_SECTION@@KK@ZXZ@4QBW4module_id@?A0x5c520fe1@@B 10001364     libvcruntime:winapi_downlevel.obj
 0001:00000388       ?tokenTable@@3QBQBDB       10001388     libvcruntime:undname.obj
 0001:000003c8       ?nameTable@@3QBQBDB        100013c8     libvcruntime:undname.obj
 0001:00000510       ?rttiTable@@3QBQBDB        10001510     libvcruntime:undname.obj
 0001:00000bf0       ___acrt_initializers       10001bf0     libucrt:initialization.obj
 0001:00000c70       ?errtable@@3QBUerrentry@?A0x31fdb9ec@@B 10001c70     libucrt:errno.obj
 0001:00000dd8       ?_mb_locale_names@@3QBQB_WB 10001dd8     libucrt:mbctype.obj
 0001:00000e18       ?module_names@?A0x391cf84c@@3QBQB_WB 10001e18     libucrt:winapi_thunks.obj
 0001:00001338       ?candidate_modules@?1??try_get_AreFileApisANSI@@YAP6GHXZXZ@4QBW4module_id@?A0x391cf84c@@B 10002338     libucrt:winapi_thunks.obj
 0001:0000134c       ?candidate_modules@?1??try_get_FlsAlloc@@YAP6GKP6GXPAX@Z@ZXZ@4QBW4module_id@?A0x391cf84c@@B 1000234c     libucrt:winapi_thunks.obj
 0001:00001360       ?candidate_modules@?1??try_get_FlsFree@@YAP6GHK@ZXZ@4QBW4module_id@?A0x391cf84c@@B 10002360     libucrt:winapi_thunks.obj
 0001:00001370       ?candidate_modules@?1??try_get_FlsGetValue@@YAP6GPAXK@ZXZ@4QBW4module_id@?A0x391cf84c@@B 10002370     libucrt:winapi_thunks.obj
 0001:00001384       ?candidate_modules@?1??try_get_FlsSetValue@@YAP6GHKPAX@ZXZ@4QBW4module_id@?A0x391cf84c@@B 10002384     libucrt:winapi_thunks.obj
 0001:00001398       ?candidate_modules@?1??try_get_InitializeCriticalSectionEx@@YAP6GHPAU_RTL_CRITICAL_SECTION@@KK@ZXZ@4QBW4module_id@?A0x391cf84c@@B 10002398     libucrt:winapi_thunks.obj
 0001:000013bc       ?candidate_modules@?1??try_get_LCMapStringEx@@YAP6GHPB_WK0HPA_WHPAU_nlsversioninfo@@PAXJ@ZXZ@4QBW4module_id@?A0x391cf84c@@B 100023bc     libucrt:winapi_thunks.obj
 0001:000013d4       ?candidate_modules@?1??try_get_LocaleNameToLCID@@YAP6GKPB_WK@ZXZ@4QBW4module_id@?A0x391cf84c@@B 100023d4     libucrt:winapi_thunks.obj
 0001:000013f0       ?candidate_modules@?1??try_get_AppPolicyGetProcessTerminationMethod@@YAP6GJPAXPAW4AppPolicyProcessTerminationMethod@@@ZXZ@4QBW4module_id@?A0x391cf84c@@B 100023f0     libucrt:winapi_thunks.obj
 0001:00001ee0       ?LcidToLocaleNameTable@?A0x881e4c05@@3QBULcidToLocaleName@1@B 10002ee0     libucrt:lcidtoname_downlevel.obj
 0001:00003008       ?LocaleNameToIndexTable@?A0x881e4c05@@3QBULocaleNameIndex@1@B 10004008     libucrt:lcidtoname_downlevel.obj
 0001:00003f60       LOG_name                   10004f60     libucrt:log10_impl.obj
 0001:00003f70       _One                       10004f70     libucrt:ceil_pentium4.obj
 0001:00003f80       _Bns                       10004f80     libucrt:ceil_pentium4.obj
 0001:00003f90       _Zero                      10004f90     libucrt:ceil_pentium4.obj
 0001:00003fa0       _S                         10004fa0     libucrt:ceil_pentium4.obj
 0001:00003fb0       _NegZero                   10004fb0     libucrt:ceil_pentium4.obj
 0001:00003fd0       emask                      10004fd0     libucrt:log10_pentium4.obj
 0001:00003fe0       CC                         10004fe0     libucrt:log10_pentium4.obj
 0001:00003ff0       Magic                      10004ff0     libucrt:log10_pentium4.obj
 0001:00004000       hi_mask                    10005000     libucrt:log10_pentium4.obj
 0001:00004010       LOG10_2                    10005010     libucrt:log10_pentium4.obj
 0001:00004020       place_L                    10005020     libucrt:log10_pentium4.obj
 0001:00004040       One                        10005040     libucrt:log10_pentium4.obj
 0001:00004050       Zero                       10005050     libucrt:log10_pentium4.obj
 0001:00004060       Two52                      10005060     libucrt:log10_pentium4.obj
 0001:00004070       Infs                       10005070     libucrt:log10_pentium4.obj
 0001:00004080       NaN                        10005080     libucrt:log10_pentium4.obj
 0001:00004090       coeff                      10005090     libucrt:log10_pentium4.obj
 0001:000040ee       _log2max                   100050ee     libucrt:87tran.obj
 0001:000040f8       _smallarg                  100050f8     libucrt:87tran.obj
 0001:00004102       _half                      10005102     libucrt:87tran.obj
 0001:0000414e       One                        1000514e     libucrt:87disp.obj
 0001:00004156       Three                      10005156     libucrt:87disp.obj
 0001:0000415e       XAMtoTagTab                1000515e     libucrt:87disp.obj
 0001:00004170       One                        10005170     libucrt:common.obj
 0001:00004184       DblMax                     10005184     libucrt:common.obj
 0001:0000418c       DblMin                     1000518c     libucrt:common.obj
 0001:00004194       IeeeAdjO                   10005194     libucrt:common.obj
 0001:0000419c       IeeeAdjU                   1000519c     libucrt:common.obj
 0001:000041a4       _infinity                  100051a4     libucrt:common.obj
 0001:000041ac       _zero                      100051ac     libucrt:common.obj
 0001:000041e8       _over                      100051e8     libucrt:fpctrl.obj
 0001:000041f4       _under                     100051f4     libucrt:fpctrl.obj
 0001:00004a28       ?_names@?1??_get_fname@@9@9 10005a28     libucrt:fpexcept.obj
 0001:00004f30       $$000000                   10005f30     chkstk.obj
 0001:00005518       $LN81                      10006518     DrawLine.obj
 0001:0000552c       $LN76                      1000652c     DrawLine.obj
 0001:00005570       $LN82                      10006570     DrawLine.obj
 0001:00005584       $LN77                      10006584     DrawLine.obj
 0001:00005a98       $LN51                      10006a98     DrawLine.obj
 0001:00005aa8       $LN46                      10006aa8     DrawLine.obj
 0001:00005b30       ?DecodePointer@implementation@?1??DecodePointerWrapper@@YGPAXPAX@Z@SGPAX0@Z 10006b30 f   vc_crt_fix_impl.obj
 0001:00005b30       ?EncodePointer@implementation@?1??EncodePointerWrapper@@YGPAXPAX@Z@SGPAX0@Z 10006b30 f   vc_crt_fix_impl.obj
 0001:00005b40       ?GetLogicalProcessorInformation@implementation@?1??GetLogicalProcessorInformationWrapper@@YGHPAU_SYSTEM_LOGICAL_PROCESSOR_INFORMATION@@PAK@Z@SGH01@Z 10006b40 f   vc_crt_fix_impl.obj
 0001:00005b50       ?GetModuleHandleExW@implementation@?1??GetModuleHandleExWWrapper@@YGHKPB_WPAPAUHINSTANCE__@@@Z@SGHK01@Z 10006b50 f   vc_crt_fix_impl.obj
 0001:00005c20       ?GetNumaHighestNodeNumber@implementation@?1??GetNumaHighestNodeNumberWrapper@@YGHPAK@Z@SGH0@Z 10006c20 f   vc_crt_fix_impl.obj
 0001:00005c40       ?InitializeSListHead@implementation@slist@@YGXPAT_SLIST_HEADER@@@Z 10006c40 f   vc_crt_fix_impl.obj
 0001:00005d20       ?InterlockedFlushSList@implementation@slist@@YGPAU_SINGLE_LIST_ENTRY@@PAT_SLIST_HEADER@@@Z 10006d20 f   vc_crt_fix_impl.obj
 0001:00005d50       ?InterlockedPopEntrySList@implementation@slist@@YGPAU_SINGLE_LIST_ENTRY@@PAT_SLIST_HEADER@@@Z 10006d50 f   vc_crt_fix_impl.obj
 0001:00005da0       ?InterlockedPushEntrySList@implementation@slist@@YGPAU_SINGLE_LIST_ENTRY@@PAT_SLIST_HEADER@@PAU3@@Z 10006da0 f   vc_crt_fix_impl.obj
 0001:00005de0       ?InterlockedPushListSListEx@implementation@slist@@YGPAU_SINGLE_LIST_ENTRY@@PAT_SLIST_HEADER@@PAU3@1K@Z 10006de0 f   vc_crt_fix_impl.obj
 0001:00005e20       ?QueryDepthSList@implementation@slist@@YGGPAT_SLIST_HEADER@@@Z 10006e20 f   vc_crt_fix_impl.obj
 0001:00005e50       ?RtlFirstEntrySList@implementation@slist@@YGPAU_SINGLE_LIST_ENTRY@@PAT_SLIST_HEADER@@@Z 10006e50 f   vc_crt_fix_impl.obj
 0001:00005e80       ?XorPointer@@YAPAXPAX@Z    10006e80 f   vc_crt_fix_impl.obj
 0001:000062c0       ?find_pe_section@@YAPAU_IMAGE_SECTION_HEADER@@QAEI@Z 100072c0 f   LIBCMT:utility.obj
 0001:00006606       ?dllmain_crt_dispatch@@YGHQAUHINSTANCE__@@KQAX@Z 10007606 f   LIBCMT:dll_dllmain.obj
 0001:00006659       ?dllmain_crt_process_attach@@YAHQAUHINSTANCE__@@QAX@Z 10007659 f   LIBCMT:dll_dllmain.obj
 0001:00006763       ?dllmain_crt_process_detach@@YAH_N@Z 10007763 f   LIBCMT:dll_dllmain.obj
 0001:000067f5       ?dllmain_dispatch@@YAHQAUHINSTANCE__@@KQAX@Z 100077f5 f   LIBCMT:dll_dllmain.obj
 0001:000068fb       ?dllmain_raw@@YGHQAUHINSTANCE__@@KQAX@Z 100078fb f   LIBCMT:dll_dllmain.obj
 0001:00006c20       $$000000                   10007c20     LIBCMT:sehprolg4.obj
 0001:00006c7c       ___get_entropy             10007c7c f   LIBCMT:gs_support.obj
 0001:00006ef0       $$000000                   10007ef0     libvcruntime:memcpy.obj
 0001:00007154       TrailingUpVec              10008154     libvcruntime:memcpy.obj
 0001:00007200       TrailingDownVec            10008200     libvcruntime:memcpy.obj
 0001:00007470       $$000000                   10008470     libvcruntime:memset.obj
 0001:00007630       _ValidateLocalCookies      10008630 f   libvcruntime:chandler4.obj
 0001:00007987       ?try_get_first_available_module@@YAPAUHINSTANCE__@@QBW4module_id@?A0x5c520fe1@@0@Z 10008987 f   libvcruntime:winapi_downlevel.obj
 0001:00007a4b       ?try_get_function@@YAPAXW4function_id@?A0x5c520fe1@@QBDQBW4module_id@2@2@Z 10008a4b f   libvcruntime:winapi_downlevel.obj
 0001:00007c60       $$000000                   10008c60     libvcruntime:exsup4.obj
 0001:00007cf0       __unwind_handler4          10008cf0 f   libvcruntime:exsup4.obj
 0001:00007e30       $$000000                   10008e30     libvcruntime:exsup.obj
 0001:00007e51       __unwind_handler           10008e51 f   libvcruntime:exsup.obj
 0001:00007f70       $$000000                   10008f70     libvcruntime:lowhelpr.obj
 0001:00008070       $$000000                   10009070     libvcruntime:memmove.obj
 0001:000082d4       TrailingUpVec              100092d4     libvcruntime:memmove.obj
 0001:00008380       TrailingDownVec            10009380     libvcruntime:memmove.obj
 0001:00008786       ??$?RV<lambda_03b1d95aef87969028cfba75ccab2455>@@AAV<lambda_6e4b09c48022b2350581041d5f6b0c4c>@@V<lambda_22bdf7517842c4b3e53723af5aa32b9e>@@@?$__crt_seh_guarded_call@X@@QAEX$$QAV<lambda_03b1d95aef87969028cfba75ccab2455>@@AAV<lambda_6e4b09c48022b2350581041d5f6b0c4c>@@$$QAV<lambda_22bdf7517842c4b3e53723af5aa32b9e>@@@Z 10009786 f   libucrt:exit.obj
 0001:000087c9       ??R<lambda_6e4b09c48022b2350581041d5f6b0c4c>@@QBE@XZ 100097c9 f   libucrt:exit.obj
 0001:00008899       ?atexit_exception_filter@@YAHK@Z 10009899 f   libucrt:exit.obj
 0001:000088ac       ?common_exit@@YAXHW4_crt_exit_cleanup_mode@@W4_crt_exit_return_mode@@@Z 100098ac f   libucrt:exit.obj
 0001:00008912       ?exit_or_terminate_process@@YAXI@Z 10009912 f   libucrt:exit.obj
 0001:00008954       ?is_managed_app@@YA_NXZ    10009954 f   libucrt:exit.obj
 0001:00008997       ?try_cor_exit_process@@YAXI@Z 10009997 f   libucrt:exit.obj
 0001:00008a27       ??$common_configure_argv@D@@YAHW4_crt_argv_mode@@@Z 10009a27 f   libucrt:argv_parsing.obj
 0001:00008b5f       ??$parse_command_line@D@@YAXPADPAPAD0PAI2@Z 10009b5f f   libucrt:argv_parsing.obj
 0001:00008d32       ??$common_initialize_environment_nolock@D@@YAHXZ 10009d32 f   libucrt:environment_initialization.obj
 0001:00008d85       ??$create_environment@D@@YAQAPADQAD@Z 10009d85 f   libucrt:environment_initialization.obj
 0001:00008e57       ??$free_environment@_W@@YAXQAPA_W@Z 10009e57 f   libucrt:environment_initialization.obj
 0001:00008e57       ??$free_environment@D@@YAXQAPAD@Z 10009e57 f   libucrt:environment_initialization.obj
 0001:00008eaf       ??$uninitialize_environment_internal@D@@YAXAAPAPAD@Z 10009eaf f   libucrt:environment_initialization.obj
 0001:00008eca       ??$uninitialize_environment_internal@_W@@YAXAAPAPA_W@Z 10009eca f   libucrt:environment_initialization.obj
 0001:00008f21       ??$?RV<lambda_69a2805e680e0e292e8ba93315fe43a8>@@AAV<lambda_f03950bc5685219e0bcd2087efbe011e>@@V<lambda_03fcd07e894ec930e3f35da366ca99d6>@@@?$__crt_seh_guarded_call@H@@QAEH$$QAV<lambda_69a2805e680e0e292e8ba93315fe43a8>@@AAV<lambda_f03950bc5685219e0bcd2087efbe011e>@@$$QAV<lambda_03fcd07e894ec930e3f35da366ca99d6>@@@Z 10009f21 f   libucrt:onexit.obj
 0001:00008f72       ??$?RV<lambda_8e746cf0007f6ed984d6f78af1fec997>@@AAV<lambda_22ebabd17bc4fa466a2aca6d8deb888d>@@V<lambda_18ed0c0b38a6dc0daf1e7ac6d6adf05e>@@@?$__crt_seh_guarded_call@H@@QAEH$$QAV<lambda_8e746cf0007f6ed984d6f78af1fec997>@@AAV<lambda_22ebabd17bc4fa466a2aca6d8deb888d>@@$$QAV<lambda_18ed0c0b38a6dc0daf1e7ac6d6adf05e>@@@Z 10009f72 f   libucrt:onexit.obj
 0001:00008fe3       ??R<lambda_22ebabd17bc4fa466a2aca6d8deb888d>@@QBEHXZ 10009fe3 f   libucrt:onexit.obj
 0001:0000910e       ??R<lambda_f03950bc5685219e0bcd2087efbe011e>@@QBEHXZ 1000a10e f   libucrt:onexit.obj
 0001:0000928d       _initialize_global_variables 1000a28d f   libucrt:initialization.obj
 0001:0000929a       _initialize_c              1000a29a f   libucrt:initialization.obj
 0001:000092b4       _uninitialize_c            1000a2b4 f   libucrt:initialization.obj
 0001:000092b4       _initialize_environment    1000a2b4 f   libucrt:initialization.obj
 0001:000092b4       _report_memory_leaks       1000a2b4 f   libucrt:initialization.obj
 0001:000092b4       _initialize_global_state_isolation 1000a2b4 f   libucrt:initialization.obj
 0001:000092b4       _uninitialize_global_state_isolation 1000a2b4 f   libucrt:initialization.obj
 0001:000092b7       _uninitialize_environment  1000a2b7 f   libucrt:initialization.obj
 0001:000092bf       _initialize_pointers       1000a2bf f   libucrt:initialization.obj
 0001:000092ed       _uninitialize_vcruntime    1000a2ed f   libucrt:initialization.obj
 0001:000092f6       _uninitialize_allocated_memory 1000a2f6 f   libucrt:initialization.obj
 0001:0000930f       _uninitialize_allocated_io_buffers 1000a30f f   libucrt:initialization.obj
 0001:0000935f       ??R<lambda_af42a3ee9806e9a7305d451646e05244>@@QBEXAAPAU__crt_multibyte_data@@@Z 1000a35f f   libucrt:initialization.obj
 0001:00009630       $$000000                   1000a630     libucrt:strncmp.obj
 0001:00009730       ??$?RV<lambda_15ade71b0218206bbe3333a0c9b79046>@@AAV<lambda_da44e0f8b0f19ba52fefafb335991732>@@V<lambda_207f2d024fc103971653565357d6cd41>@@@?$__crt_seh_guarded_call@X@@QAEX$$QAV<lambda_15ade71b0218206bbe3333a0c9b79046>@@AAV<lambda_da44e0f8b0f19ba52fefafb335991732>@@$$QAV<lambda_207f2d024fc103971653565357d6cd41>@@@Z 1000a730 f   libucrt:per_thread_data.obj
 0001:00009778       ??$?RV<lambda_38edbb1296d33220d7e4dd0ed76b244a>@@AAV<lambda_5ce1d447e08cb34b2473517608e21441>@@V<lambda_fb385d3da700c9147fc39e65dd577a8c>@@@?$__crt_seh_guarded_call@X@@QAEX$$QAV<lambda_38edbb1296d33220d7e4dd0ed76b244a>@@AAV<lambda_5ce1d447e08cb34b2473517608e21441>@@$$QAV<lambda_fb385d3da700c9147fc39e65dd577a8c>@@@Z 1000a778 f   libucrt:per_thread_data.obj
 0001:000097d9       ??$?RV<lambda_6affb1475c98b40b75cdec977db92e3c>@@AAV<lambda_b8d4b9c228a6ecc3f80208dbb4b4a104>@@V<lambda_608742c3c92a14382c1684fc64f96c88>@@@?$__crt_seh_guarded_call@X@@QAEX$$QAV<lambda_6affb1475c98b40b75cdec977db92e3c>@@AAV<lambda_b8d4b9c228a6ecc3f80208dbb4b4a104>@@$$QAV<lambda_608742c3c92a14382c1684fc64f96c88>@@@Z 1000a7d9 f   libucrt:per_thread_data.obj
 0001:00009824       ??$?RV<lambda_a7e850c220f1c8d1e6efeecdedd162c6>@@AAV<lambda_46720907175c18b6c9d2717bc0d2d362>@@V<lambda_9048902d66e8d99359bc9897bbb930a8>@@@?$__crt_seh_guarded_call@X@@QAEX$$QAV<lambda_a7e850c220f1c8d1e6efeecdedd162c6>@@AAV<lambda_46720907175c18b6c9d2717bc0d2d362>@@$$QAV<lambda_9048902d66e8d99359bc9897bbb930a8>@@@Z 1000a824 f   libucrt:per_thread_data.obj
 0001:00009874       ?construct_ptd@@YAXQAU__acrt_ptd@@QAPAU__crt_locale_data@@@Z 1000a874 f   libucrt:per_thread_data.obj
 0001:0000990f       ?destroy_fls@@YGXPAX@Z     1000a90f f   libucrt:per_thread_data.obj
 0001:00009930       ?destroy_ptd@@YAXQAU__acrt_ptd@@@Z 1000a930 f   libucrt:per_thread_data.obj
 0001:000099ff       ?replace_current_thread_locale_nolock@@YAXQAU__acrt_ptd@@QAU__crt_locale_data@@@Z 1000a9ff f   libucrt:per_thread_data.obj
 0001:0000a079       ?<lambda_invoker_cdecl>@<lambda_86056e3c024bff449830248dc1621ed2>@@CAHPBX0@Z 1000b079 f   libucrt:argv_wildcards.obj
 0001:0000a091       ??$__acrt_convert_wcs_mbs_cp@D_WV<lambda_62f6974d9771e494a5ea317cc32e971c>@@U__crt_win32_buffer_internal_dynamic_resizing@@@@YAHQBDAAV?$__crt_win32_buffer@_WU__crt_win32_buffer_internal_dynamic_resizing@@@@ABV<lambda_62f6974d9771e494a5ea317cc32e971c>@@I@Z 1000b091 f   libucrt:argv_wildcards.obj
 0001:0000a143       ??$__acrt_convert_wcs_mbs_cp@_WDV<lambda_28bda7af82a03b66c1cb3803a755f95d>@@U__crt_win32_buffer_internal_dynamic_resizing@@@@YAHQB_WAAV?$__crt_win32_buffer@DU__crt_win32_buffer_internal_dynamic_resizing@@@@ABV<lambda_28bda7af82a03b66c1cb3803a755f95d>@@I@Z 1000b143 f   libucrt:argv_wildcards.obj
 0001:0000a231       ??$common_expand_argv_wildcards@D@@YAHQAPADQAPAPAD@Z 1000b231 f   libucrt:argv_wildcards.obj
 0001:0000a422       ??$copy_and_add_argument_to_buffer@D@@YAHQBD0IAAV?$argument_list@D@?A0x5f5c8891@@@Z 1000b422 f   libucrt:argv_wildcards.obj
 0001:0000a4d5       ??$expand_argument_wildcards@D@@YAHQAD0AAV?$argument_list@D@?A0x5f5c8891@@@Z 1000b4d5 f   libucrt:argv_wildcards.obj
 0001:0000a823       ?expand_if_necessary@?$argument_list@D@?A0x5f5c8891@@AAEHXZ 1000b823 f   libucrt:argv_wildcards.obj
 0001:0000a8b5       ??$__acrt_convert_wcs_mbs_cp@_WDV<lambda_0fec1a7b3f42a53036604e18c2d5e07e>@@U__crt_win32_buffer_no_resizing@@@@YAHQB_WAAV?$__crt_win32_buffer@DU__crt_win32_buffer_no_resizing@@@@ABV<lambda_0fec1a7b3f42a53036604e18c2d5e07e>@@I@Z 1000b8b5 f   libucrt:getmodulefilenamea.obj
 0001:0000aa5a       ??$?RV<lambda_ceb1ee4838e85a9d631eb091e2fbe199>@@AAV<lambda_ae742caa10f662c28703da3d2ea5e57e>@@V<lambda_cd08b5d6af4937fe54fc07d0c9bf6b37>@@@?$__crt_seh_guarded_call@X@@QAEX$$QAV<lambda_ceb1ee4838e85a9d631eb091e2fbe199>@@AAV<lambda_ae742caa10f662c28703da3d2ea5e57e>@@$$QAV<lambda_cd08b5d6af4937fe54fc07d0c9bf6b37>@@@Z 1000ba5a f   libucrt:mbctype.obj
 0001:0000aa9d       ??R<lambda_ae742caa10f662c28703da3d2ea5e57e>@@QBEXXZ 1000ba9d f   libucrt:mbctype.obj
 0001:0000ab20       ?CPtoLocaleName@@YAPB_WH@Z 1000bb20 f   libucrt:mbctype.obj
 0001:0000ab5e       ?getSystemCP@@YAHH@Z       1000bb5e f   libucrt:mbctype.obj
 0001:0000abd1       ?setSBCS@@YAXPAU__crt_multibyte_data@@@Z 1000bbd1 f   libucrt:mbctype.obj
 0001:0000ac36       ?setSBUpLow@@YAXPAU__crt_multibyte_data@@@Z 1000bc36 f   libucrt:mbctype.obj
 0001:0000adb9       ?setmbcp_internal@@YAHH_NQAU__acrt_ptd@@QAPAU__crt_multibyte_data@@@Z 1000bdb9 f   libucrt:mbctype.obj
 0001:0000aed4       ?update_thread_multibyte_data_internal@@YAPAU__crt_multibyte_data@@QAU__acrt_ptd@@QAPAU1@@Z 1000bed4 f   libucrt:mbctype.obj
 0001:0000b1ba       _memcpy_s                  1000c1ba f   libucrt:mbctype.obj
 0001:0000b23b       ?x_ismbbtype_l@@YAHPAU__crt_locale_pointers@@IHH@Z 1000c23b f   libucrt:ismbbyte.obj
 0001:0000b3ee       ?find_end_of_double_null_terminated_sequence@@YAPB_WQB_W@Z 1000c3ee f   libucrt:get_environment_from_os.obj
 0001:0000b518       ?initialize_inherited_file_handles_nolock@@YAXXZ 1000c518 f   libucrt:ioinit.obj
 0001:0000b5d0       ?initialize_stdio_handles_nolock@@YAXXZ 1000c5d0 f   libucrt:ioinit.obj
 0001:0000b706       ?try_get_AreFileApisANSI@@YAP6GHXZXZ 1000c706 f   libucrt:winapi_thunks.obj
 0001:0000b720       ?try_get_LCMapStringEx@@YAP6GHPB_WK0HPA_WHPAU_nlsversioninfo@@PAXJ@ZXZ 1000c720 f   libucrt:winapi_thunks.obj
 0001:0000b73a       ?try_get_LocaleNameToLCID@@YAP6GKPB_WK@ZXZ 1000c73a f   libucrt:winapi_thunks.obj
 0001:0000b754       ?try_get_first_available_module@@YAPAUHINSTANCE__@@QBW4module_id@?A0x391cf84c@@0@Z 1000c754 f   libucrt:winapi_thunks.obj
 0001:0000b81d       ?try_get_function@@YAPAXW4function_id@?A0x391cf84c@@QBDQBW4module_id@2@2@Z 1000c81d f   libucrt:winapi_thunks.obj
 0001:0000bc7a       ??$?RV<lambda_cbab9ec6f41b0180b23cc171c22676b0>@@AAV<lambda_44731a7d0e6d81c3e6aa82d741081786>@@V<lambda_4b292cb8dd18144e164572427af410ab>@@@?$__crt_seh_guarded_call@P6AXH@Z@@QAEP6AXH@Z$$QAV<lambda_cbab9ec6f41b0180b23cc171c22676b0>@@AAV<lambda_44731a7d0e6d81c3e6aa82d741081786>@@$$QAV<lambda_4b292cb8dd18144e164572427af410ab>@@@Z 1000cc7a f   libucrt:signal.obj
 0001:0000bcd4       ?get_global_action_nolock@@YAPAP6AXH@ZH@Z 1000ccd4 f   libucrt:signal.obj
 0001:0000bd16       ?siglookup@@YAPAU__crt_signal_action_t@@HQAU1@@Z 1000cd16 f   libucrt:signal.obj
 0001:0000bfce       ??$?RV<lambda_2866be3712abc81a800a822484c830d8>@@AAV<lambda_39ca0ed439415581b5b15c265174cece>@@V<lambda_2b24c74d71094a6cd0cb82e44167d71b>@@@?$__crt_seh_guarded_call@X@@QAEX$$QAV<lambda_2866be3712abc81a800a822484c830d8>@@AAV<lambda_39ca0ed439415581b5b15c265174cece>@@$$QAV<lambda_2b24c74d71094a6cd0cb82e44167d71b>@@@Z 1000cfce f   libucrt:fflush.obj
 0001:0000c050       ??$?RV<lambda_2cc53f568c5a2bb6f192f930a45d44ea>@@AAV<lambda_ab61a845afdef5b7c387490eaf3616ee>@@V<lambda_c2ffc0b7726aa6be21d5f0026187e748>@@@?$__crt_seh_guarded_call@X@@QAEX$$QAV<lambda_2cc53f568c5a2bb6f192f930a45d44ea>@@AAV<lambda_ab61a845afdef5b7c387490eaf3616ee>@@$$QAV<lambda_c2ffc0b7726aa6be21d5f0026187e748>@@@Z 1000d050 f   libucrt:fflush.obj
 0001:0000c0f2       ?common_flush_all@@YAH_N@Z 1000d0f2 f   libucrt:fflush.obj
 0001:0000c141       ?common_flush_all_should_try_to_flush_stream@@YA_NV__crt_stdio_stream@@QAH@Z 1000d141 f   libucrt:fflush.obj
 0001:0000c174       ?is_stream_flushable_or_commitable@@YA_NJ@Z 1000d174 f   libucrt:fflush.obj
 0001:0000c56a       ??$?RV<lambda_e5124f882df8998aaf41531e079ba474>@@AAV<lambda_3e16ef9562a7dcce91392c22ab16ea36>@@V<lambda_e25ca0880e6ef98be67edffd8c599615>@@@?$__crt_seh_guarded_call@X@@QAEX$$QAV<lambda_e5124f882df8998aaf41531e079ba474>@@AAV<lambda_3e16ef9562a7dcce91392c22ab16ea36>@@$$QAV<lambda_e25ca0880e6ef98be67edffd8c599615>@@@Z 1000d56a f   libucrt:wsetlocale.obj
 0001:0000c9d0       ?swap@@YAXPAD0I@Z          1000d9d0 f   libucrt:qsort.obj
 0001:0000ce54       ??$common_tcsncpy_s@D@@YAHQADIQBDI@Z 1000de54 f   libucrt:strncpy_s.obj
 0001:0000cf20       $$000000                   1000df20     libucrt:strpbrk.obj
 0001:0000d12b       ?__acrt_LCMapStringA_stat@@YAHPAU__crt_locale_pointers@@PB_WKPBDHPADHHH@Z 1000e12b f   libucrt:lcmapstringa.obj
 0001:0000d362       ?initialize_multibyte@@YAHXZ 1000e362 f   libucrt:multibyte_initializer.obj
 0001:0000d694       ?GetTableIndexFromLocaleName@@YAHPB_W@Z 1000e694 f   libucrt:lcidtoname_downlevel.obj
 0001:0000d774       ??$?RV<lambda_9e9de3de5fa147e2223d7db92bc10aa6>@@AAV<lambda_38ce7e780aa69e748d6df282ebc68efe>@@V<lambda_8ca6da459f0f6780f1cff60fdc3d00e5>@@@?$__crt_seh_guarded_call@H@@QAEH$$QAV<lambda_9e9de3de5fa147e2223d7db92bc10aa6>@@AAV<lambda_38ce7e780aa69e748d6df282ebc68efe>@@$$QAV<lambda_8ca6da459f0f6780f1cff60fdc3d00e5>@@@Z 1000e774 f   libucrt:commit.obj
 0001:0000d88b       ?write_double_translated_ansi_nolock@@YA?AUwrite_result@?A0x17268360@@HQBDI@Z 1000e88b f   libucrt:write.obj
 0001:0000dc37       ?write_double_translated_unicode_nolock@@YA?AUwrite_result@?A0x17268360@@QBDI@Z 1000ec37 f   libucrt:write.obj
 0001:0000dca1       ?write_requires_double_translation_nolock@@YA_NH@Z 1000eca1 f   libucrt:write.obj
 0001:0000dd14       ?write_text_ansi_nolock@@YA?AUwrite_result@?A0x17268360@@HQBDI@Z 1000ed14 f   libucrt:write.obj
 0001:0000ddf1       ?write_text_utf16le_nolock@@YA?AUwrite_result@?A0x17268360@@HQBDI@Z 1000edf1 f   libucrt:write.obj
 0001:0000dedc       ?write_text_utf8_nolock@@YA?AUwrite_result@?A0x17268360@@HQBDI@Z 1000eedc f   libucrt:write.obj
 0001:0000e44f       ??R<lambda_0f007d4f94c691a9a85cf1869a09f0c3>@@QBEIPBD@Z 1000f44f f   libucrt:mbrtowc.obj
 0001:0000e740       ?free_crt_array_internal@@YAXQAPBXI@Z 1000f740 f   libucrt:inittime.obj
 0001:0000e87e       ??$common_lseek_nolock@_J@@YA_JH_JH@Z 1000f87e f   libucrt:lseek.obj
 0001:0000ebf0       $$000000                   1000fbf0     libucrt:log10_impl.obj
 0001:0000ed00       $$000000                   1000fd00     libucrt:ceil_pentium4.obj
 0001:0000ee20       $$000000                   1000fe20     libucrt:_strnicm.obj
 0001:0000ee81       ?__dcrt_lowio_initialize_console_output@@YAXXZ 1000fe81 f   libucrt:initcon.obj
 0001:0000ef2b       ??$?RV<lambda_218ce3db14220d0be481dae8ef3383b6>@@AAV<lambda_628dfdc04ba53c8bfc02c9951375f3f5>@@V<lambda_57dc472bd5c9d5f3b2cbca59b8a843ae>@@@?$__crt_seh_guarded_call@H@@QAEH$$QAV<lambda_218ce3db14220d0be481dae8ef3383b6>@@AAV<lambda_628dfdc04ba53c8bfc02c9951375f3f5>@@$$QAV<lambda_57dc472bd5c9d5f3b2cbca59b8a843ae>@@@Z 1000ff2b f   libucrt:close.obj
 0001:0000f130       $$000000                   10010130     libucrt:log10_pentium4.obj
 0001:0000f3c0       $$000000                   100103c0     libucrt:87tran.obj
 0001:0000f5d0       $$000000                   100105d0     libucrt:87disp.obj
 0001:0000f830       $$000000                   10010830     libucrt:common.obj
 0001:0000f9c0       $$000000                   100109c0     libucrt:genexcep.obj
 0001:00010a60       $$000000                   10011a60     LIBCMT:ulldvrm.obj
 0001:00010b00       $$000000                   10011b00     LIBCMT:llmul.obj
 0001:00010b40       $$000000                   10011b40     LIBCMT:lldvrm.obj
 0001:00010c20       $$000000                   10011c20     LIBCMT:ullshr.obj
 0001:00010c40       $$000000                   10011c40     LIBCMT:alloca16.obj
 0001:00010c70       $$000000                   10011c70     LIBCMT:llshl.obj
 0001:00010c90       $$000000                   10011c90     LIBCMT:ftol2.obj
 0001:00010d50       $$000000                   10011d50     libvcruntime:strchr.obj
 0001:00010e80       $$000000                   10011e80     libvcruntime:strrchr.obj
 0001:00010fc0       ??__FDeleter@?1??InitializeSListHead@implementation@slist@@YGXPAT_SLIST_HEADER@@@Z@YAXXZ 10011fc0 f   vc_crt_fix_impl.obj
 0001:00011000       __sehtable$___scrt_is_nonwritable_in_current_image 10012000     LIBCMT:utility.obj
 0001:00011020       __sehtable$?dllmain_crt_process_attach@@YAHQAUHINSTANCE__@@QAX@Z 10012020     LIBCMT:dll_dllmain.obj
 0001:00011040       __sehtable$?dllmain_crt_process_detach@@YAH_N@Z 10012040     LIBCMT:dll_dllmain.obj
 0001:00011060       __sehtable$?dllmain_dispatch@@YAHQAUHINSTANCE__@@KQAX@Z 10012060     LIBCMT:dll_dllmain.obj
 0001:00011080       __sehtable$___DestructExceptionObject 10012080     libvcruntime:ehhelpers.obj
 0001:000110a0       __sehtable$??R<lambda_6e4b09c48022b2350581041d5f6b0c4c>@@QBE@XZ 100120a0     libucrt:exit.obj
 0001:000110c0       __sehtable$??$?RV<lambda_03b1d95aef87969028cfba75ccab2455>@@AAV<lambda_6e4b09c48022b2350581041d5f6b0c4c>@@V<lambda_22bdf7517842c4b3e53723af5aa32b9e>@@@?$__crt_seh_guarded_call@X@@QAEX$$QAV<lambda_03b1d95aef87969028cfba75ccab2455>@@AAV<lambda_6e4b09c48022b2350581041d5f6b0c4c>@@$$QAV<lambda_22bdf7517842c4b3e53723af5aa32b9e>@@@Z 100120c0     libucrt:exit.obj
 0001:000110e0       __sehtable$??$?RV<lambda_8e746cf0007f6ed984d6f78af1fec997>@@AAV<lambda_22ebabd17bc4fa466a2aca6d8deb888d>@@V<lambda_18ed0c0b38a6dc0daf1e7ac6d6adf05e>@@@?$__crt_seh_guarded_call@H@@QAEH$$QAV<lambda_8e746cf0007f6ed984d6f78af1fec997>@@AAV<lambda_22ebabd17bc4fa466a2aca6d8deb888d>@@$$QAV<lambda_18ed0c0b38a6dc0daf1e7ac6d6adf05e>@@@Z 100120e0     libucrt:onexit.obj
 0001:00011100       __sehtable$??$?RV<lambda_69a2805e680e0e292e8ba93315fe43a8>@@AAV<lambda_f03950bc5685219e0bcd2087efbe011e>@@V<lambda_03fcd07e894ec930e3f35da366ca99d6>@@@?$__crt_seh_guarded_call@H@@QAEH$$QAV<lambda_69a2805e680e0e292e8ba93315fe43a8>@@AAV<lambda_f03950bc5685219e0bcd2087efbe011e>@@$$QAV<lambda_03fcd07e894ec930e3f35da366ca99d6>@@@Z 10012100     libucrt:onexit.obj
 0001:00011120       __sehtable$_terminate      10012120     libucrt:terminate.obj
 0001:00011140       __sehtable$??$?RV<lambda_15ade71b0218206bbe3333a0c9b79046>@@AAV<lambda_da44e0f8b0f19ba52fefafb335991732>@@V<lambda_207f2d024fc103971653565357d6cd41>@@@?$__crt_seh_guarded_call@X@@QAEX$$QAV<lambda_15ade71b0218206bbe3333a0c9b79046>@@AAV<lambda_da44e0f8b0f19ba52fefafb335991732>@@$$QAV<lambda_207f2d024fc103971653565357d6cd41>@@@Z 10012140     libucrt:per_thread_data.obj
 0001:00011160       __sehtable$??$?RV<lambda_a7e850c220f1c8d1e6efeecdedd162c6>@@AAV<lambda_46720907175c18b6c9d2717bc0d2d362>@@V<lambda_9048902d66e8d99359bc9897bbb930a8>@@@?$__crt_seh_guarded_call@X@@QAEX$$QAV<lambda_a7e850c220f1c8d1e6efeecdedd162c6>@@AAV<lambda_46720907175c18b6c9d2717bc0d2d362>@@$$QAV<lambda_9048902d66e8d99359bc9897bbb930a8>@@@Z 10012160     libucrt:per_thread_data.obj
 0001:00011180       __sehtable$??$?RV<lambda_38edbb1296d33220d7e4dd0ed76b244a>@@AAV<lambda_5ce1d447e08cb34b2473517608e21441>@@V<lambda_fb385d3da700c9147fc39e65dd577a8c>@@@?$__crt_seh_guarded_call@X@@QAEX$$QAV<lambda_38edbb1296d33220d7e4dd0ed76b244a>@@AAV<lambda_5ce1d447e08cb34b2473517608e21441>@@$$QAV<lambda_fb385d3da700c9147fc39e65dd577a8c>@@@Z 10012180     libucrt:per_thread_data.obj
 0001:000111a0       __sehtable$??$?RV<lambda_6affb1475c98b40b75cdec977db92e3c>@@AAV<lambda_b8d4b9c228a6ecc3f80208dbb4b4a104>@@V<lambda_608742c3c92a14382c1684fc64f96c88>@@@?$__crt_seh_guarded_call@X@@QAEX$$QAV<lambda_6affb1475c98b40b75cdec977db92e3c>@@AAV<lambda_b8d4b9c228a6ecc3f80208dbb4b4a104>@@$$QAV<lambda_608742c3c92a14382c1684fc64f96c88>@@@Z 100121a0     libucrt:per_thread_data.obj
 0001:000111c0       __sehtable$?update_thread_multibyte_data_internal@@YAPAU__crt_multibyte_data@@QAU__acrt_ptd@@QAPAU1@@Z 100121c0     libucrt:mbctype.obj
 0001:000111e0       __sehtable$??$?RV<lambda_ceb1ee4838e85a9d631eb091e2fbe199>@@AAV<lambda_ae742caa10f662c28703da3d2ea5e57e>@@V<lambda_cd08b5d6af4937fe54fc07d0c9bf6b37>@@@?$__crt_seh_guarded_call@X@@QAEX$$QAV<lambda_ceb1ee4838e85a9d631eb091e2fbe199>@@AAV<lambda_ae742caa10f662c28703da3d2ea5e57e>@@$$QAV<lambda_cd08b5d6af4937fe54fc07d0c9bf6b37>@@@Z 100121e0     libucrt:mbctype.obj
 0001:00011200       __sehtable$___acrt_initialize_lowio 10012200     libucrt:ioinit.obj
 0001:00011220       __sehtable$__query_new_handler 10012220     libucrt:new_handler.obj
 0001:00011240       __sehtable$_raise          10012240     libucrt:signal.obj
 0001:00011260       __sehtable$??$?RV<lambda_cbab9ec6f41b0180b23cc171c22676b0>@@AAV<lambda_44731a7d0e6d81c3e6aa82d741081786>@@V<lambda_4b292cb8dd18144e164572427af410ab>@@@?$__crt_seh_guarded_call@P6AXH@Z@@QAEP6AXH@Z$$QAV<lambda_cbab9ec6f41b0180b23cc171c22676b0>@@AAV<lambda_44731a7d0e6d81c3e6aa82d741081786>@@$$QAV<lambda_4b292cb8dd18144e164572427af410ab>@@@Z 10012260     libucrt:signal.obj
 0001:00011280       __sehtable$??$?RV<lambda_2866be3712abc81a800a822484c830d8>@@AAV<lambda_39ca0ed439415581b5b15c265174cece>@@V<lambda_2b24c74d71094a6cd0cb82e44167d71b>@@@?$__crt_seh_guarded_call@X@@QAEX$$QAV<lambda_2866be3712abc81a800a822484c830d8>@@AAV<lambda_39ca0ed439415581b5b15c265174cece>@@$$QAV<lambda_2b24c74d71094a6cd0cb82e44167d71b>@@@Z 10012280     libucrt:fflush.obj
 0001:000112a0       __sehtable$??$?RV<lambda_2cc53f568c5a2bb6f192f930a45d44ea>@@AAV<lambda_ab61a845afdef5b7c387490eaf3616ee>@@V<lambda_c2ffc0b7726aa6be21d5f0026187e748>@@@?$__crt_seh_guarded_call@X@@QAEX$$QAV<lambda_2cc53f568c5a2bb6f192f930a45d44ea>@@AAV<lambda_ab61a845afdef5b7c387490eaf3616ee>@@$$QAV<lambda_c2ffc0b7726aa6be21d5f0026187e748>@@@Z 100122a0     libucrt:fflush.obj
 0001:000112c0       __sehtable$??$?RV<lambda_e5124f882df8998aaf41531e079ba474>@@AAV<lambda_3e16ef9562a7dcce91392c22ab16ea36>@@V<lambda_e25ca0880e6ef98be67edffd8c599615>@@@?$__crt_seh_guarded_call@X@@QAEX$$QAV<lambda_e5124f882df8998aaf41531e079ba474>@@AAV<lambda_3e16ef9562a7dcce91392c22ab16ea36>@@$$QAV<lambda_e25ca0880e6ef98be67edffd8c599615>@@@Z 100122c0     libucrt:wsetlocale.obj
 0001:000112e0       __sehtable$___acrt_update_thread_locale_data 100122e0     libucrt:locale_refcounting.obj
 0001:00011300       __sehtable$___acrt_lowio_ensure_fh_exists 10012300     libucrt:osfinfo.obj
 0001:00011320       __sehtable$??$?RV<lambda_9e9de3de5fa147e2223d7db92bc10aa6>@@AAV<lambda_38ce7e780aa69e748d6df282ebc68efe>@@V<lambda_8ca6da459f0f6780f1cff60fdc3d00e5>@@@?$__crt_seh_guarded_call@H@@QAEH$$QAV<lambda_9e9de3de5fa147e2223d7db92bc10aa6>@@AAV<lambda_38ce7e780aa69e748d6df282ebc68efe>@@$$QAV<lambda_8ca6da459f0f6780f1cff60fdc3d00e5>@@@Z 10012320     libucrt:commit.obj
 0001:00011340       __sehtable$__write         10012340     libucrt:write.obj
 0001:00011360       __sehtable$__fcloseall     10012360     libucrt:closeall.obj
 0001:00011380       __sehtable$_fclose         10012380     libucrt:fclose.obj
 0001:000113a0       __sehtable$??$?RV<lambda_218ce3db14220d0be481dae8ef3383b6>@@AAV<lambda_628dfdc04ba53c8bfc02c9951375f3f5>@@V<lambda_57dc472bd5c9d5f3b2cbca59b8a843ae>@@@?$__crt_seh_guarded_call@H@@QAEH$$QAV<lambda_218ce3db14220d0be481dae8ef3383b6>@@AAV<lambda_628dfdc04ba53c8bfc02c9951375f3f5>@@$$QAV<lambda_57dc472bd5c9d5f3b2cbca59b8a843ae>@@@Z 100123a0     libucrt:close.obj
 0001:000113c0       __sehtable$__IsNonwritableInCurrentImage 100123c0     LIBCMT:pesect.obj
 0001:000113e0       .edata                     100123e0     DrawLine.exp
 0001:00011408       rgpv                       10012408     DrawLine.exp
 0001:00011418       rgszName                   10012418     DrawLine.exp
 0001:00011428       rgwOrd                     10012428     DrawLine.exp
 0001:00011430       szName                     10012430     DrawLine.exp
 0001:0001143d       $N00001                    1001243d     DrawLine.exp
 0001:0001144c       $N00002                    1001244c     DrawLine.exp
 0001:0001145b       $N00003                    1001245b     DrawLine.exp
 0001:00011461       $N00004                    10012461     DrawLine.exp
 0002:00000000       ?BoxChar@@3PA_WA           10013000     DrawLine.obj
 0002:00000050       ?BoxLeft@@3PAFA            10013050     DrawLine.obj
 0002:000000a0       ?BoxUp@@3PAFA              100130a0     DrawLine.obj
 0002:000000f0       ?BoxRight@@3PAFA           100130f0     DrawLine.obj
 0002:00000140       ?BoxDown@@3PAFA            10013140     DrawLine.obj
 0002:000001b0       ?__vcrt_flsindex@@3KA      100131b0     libvcruntime:per_thread_data.obj
 0002:000001e0       ?__acrt_flsindex@@3KA      100131e0     libucrt:per_thread_data.obj
 0002:000001e4       ?errno_no_memory@@3HA      100131e4     libucrt:errno.obj
 0002:000001e8       ?doserrno_no_memory@@3KA   100131e8     libucrt:errno.obj
 0002:00000410       __mbctypes                 10013410     libucrt:mbctype.obj
 0002:00000518       __mbcasemaps               10013518     libucrt:mbctype.obj
 0002:00000618       ?__rgctypeflag@@3PADA      10013618     libucrt:mbctype.obj
 0002:00000620       ?__rgcode_page_info@@3PAUcode_page_info@@A 10013620     libucrt:mbctype.obj
 0002:000009e0       ?__dcrt_lowio_console_output_handle@@3PAXA 100139e0     libucrt:initcon.obj
 0002:00000a00       ?Info@@3UPluginStartupInfo@@A 10013a00     DrawLine.obj
 0002:00000a88       ?Present_Direction@@3W4DirectionType@@A 10013a88     DrawLine.obj
 0002:00000a8c       ?Reenter@?1??OpenW@@9@4@4_NA 10013a8c     DrawLine.obj
 0002:00000a90       ?PluginMenuStrings@?1??GetPluginInfoW@@9@4@4PAPB_WA 10013a90     DrawLine.obj
 0002:00000a98       ?Cookie@?1??XorPointer@@YAPAXPAX@Z@4IB 10013a98     vc_crt_fix_impl.obj
 0002:00000a9c       ?$S1@?1??XorPointer@@YAPAXPAX@Z@4IA 10013a9c     vc_crt_fix_impl.obj
 0002:00000aa0       ?Function@?1??EncodePointerWrapper@@9@4@4Q6GPAXPAX@ZA 10013aa0     vc_crt_fix_impl.obj
 0002:00000aa4       ?$S2@?1??EncodePointerWrapper@@9@4@4IA 10013aa4     vc_crt_fix_impl.obj
 0002:00000aa8       ?Function@?1??DecodePointerWrapper@@9@4@4Q6GPAXPAX@ZA 10013aa8     vc_crt_fix_impl.obj
 0002:00000aac       ?$S3@?1??DecodePointerWrapper@@9@4@4IA 10013aac     vc_crt_fix_impl.obj
 0002:00000ab0       ?Function@?1??GetModuleHandleExWWrapper@@9@12@4Q6GHKPB_WPAPAUHINSTANCE__@@@ZA 10013ab0     vc_crt_fix_impl.obj
 0002:00000ab4       ?$S4@?1??GetModuleHandleExWWrapper@@9@12@4IA 10013ab4     vc_crt_fix_impl.obj
 0002:00000ab8       ?Deleter@?1??InitializeSListHead@implementation@slist@@YGXPAT_SLIST_HEADER@@@Z@4Vservice_deleter@23@A 10013ab8     vc_crt_fix_impl.obj
 0002:00000ad8       ?$S5@?1??InitializeSListHead@implementation@slist@@YGXPAT_SLIST_HEADER@@@Z@4IA 10013ad8     vc_crt_fix_impl.obj
 0002:00000adc       ?Function@?1??InitializeSListHeadWrapper@@9@4@4Q6GXPAT_SLIST_HEADER@@@ZA 10013adc     vc_crt_fix_impl.obj
 0002:00000ae0       ?$S6@?1??InitializeSListHeadWrapper@@9@4@4IA 10013ae0     vc_crt_fix_impl.obj
 0002:00000ae4       ?Function@?1??InterlockedFlushSListWrapper@@9@4@4Q6GPAU_SINGLE_LIST_ENTRY@@PAT_SLIST_HEADER@@@ZA 10013ae4     vc_crt_fix_impl.obj
 0002:00000ae8       ?$S7@?1??InterlockedFlushSListWrapper@@9@4@4IA 10013ae8     vc_crt_fix_impl.obj
 0002:00000aec       ?Function@?1??InterlockedPopEntrySListWrapper@@9@4@4Q6GPAU_SINGLE_LIST_ENTRY@@PAT_SLIST_HEADER@@@ZA 10013aec     vc_crt_fix_impl.obj
 0002:00000af0       ?$S8@?1??InterlockedPopEntrySListWrapper@@9@4@4IA 10013af0     vc_crt_fix_impl.obj
 0002:00000af4       ?Function@?1??InterlockedPushEntrySListWrapper@@9@8@4Q6GPAU_SINGLE_LIST_ENTRY@@PAT_SLIST_HEADER@@PAU2@@ZA 10013af4     vc_crt_fix_impl.obj
 0002:00000af8       ?$S9@?1??InterlockedPushEntrySListWrapper@@9@8@4IA 10013af8     vc_crt_fix_impl.obj
 0002:00000afc       ?Function@?1??InterlockedPushListSListExWrapper@@9@16@4Q6GPAU_SINGLE_LIST_ENTRY@@PAT_SLIST_HEADER@@PAU2@1K@ZA 10013afc     vc_crt_fix_impl.obj
 0002:00000b00       ?$S10@?1??InterlockedPushListSListExWrapper@@9@16@4IA 10013b00     vc_crt_fix_impl.obj
 0002:00000b04       ?Function@?1??RtlFirstEntrySListWrapper@@9@4@4Q6GPAU_SINGLE_LIST_ENTRY@@PAT_SLIST_HEADER@@@ZA 10013b04     vc_crt_fix_impl.obj
 0002:00000b08       ?$S11@?1??RtlFirstEntrySListWrapper@@9@4@4IA 10013b08     vc_crt_fix_impl.obj
 0002:00000b0c       ?Function@?1??QueryDepthSListWrapper@@9@4@4Q6GGPAT_SLIST_HEADER@@@ZA 10013b0c     vc_crt_fix_impl.obj
 0002:00000b10       ?$S12@?1??QueryDepthSListWrapper@@9@4@4IA 10013b10     vc_crt_fix_impl.obj
 0002:00000b14       ?Function@?1??GetNumaHighestNodeNumberWrapper@@9@4@4Q6GHPAK@ZA 10013b14     vc_crt_fix_impl.obj
 0002:00000b18       ?$S13@?1??GetNumaHighestNodeNumberWrapper@@9@4@4IA 10013b18     vc_crt_fix_impl.obj
 0002:00000b1c       ?Function@?1??GetLogicalProcessorInformationWrapper@@9@8@4Q6GHPAU_SYSTEM_LOGICAL_PROCESSOR_INFORMATION@@PAK@ZA 10013b1c     vc_crt_fix_impl.obj
 0002:00000b20       ?$S14@?1??GetLogicalProcessorInformationWrapper@@9@8@4IA 10013b20     vc_crt_fix_impl.obj
 0002:00000b2c       ?is_initialized_as_dll@@3_NA 10013b2c     LIBCMT:utility.obj
 0002:00000b2d       ?module_local_atexit_table_initialized@@3_NA 10013b2d     LIBCMT:utility.obj
 0002:00000b30       ?module_local_atexit_table@@3U_onexit_table_t@@A 10013b30     LIBCMT:utility.obj
 0002:00000b3c       ?module_local_at_quick_exit_table@@3U_onexit_table_t@@A 10013b3c     LIBCMT:utility.obj
 0002:00000b48       ?__proc_attached@@3HA      10013b48     LIBCMT:dll_dllmain.obj
 0002:00000b70       _GS_ExceptionRecord        10013b70     LIBCMT:gs_report.obj
 0002:00000bc0       _GS_ContextRecord          10013bc0     LIBCMT:gs_report.obj
 0002:00000e8c       ?__vcrt_startup_thread_ptd@@3U__vcrt_ptd@@A 10013e8c     libvcruntime:per_thread_data.obj
 0002:00000eb4       ___vcrt_lock_table         10013eb4     libvcruntime:locks.obj
 0002:00000ecc       ___vcrt_locks_initialized  10013ecc     libvcruntime:locks.obj
 0002:00000ed0       ?module_handles@@3PAPAUHINSTANCE__@@A 10013ed0     libvcruntime:winapi_downlevel.obj
 0002:00000edc       ?encoded_function_pointers@@3PAPAXA 10013edc     libvcruntime:winapi_downlevel.obj
 0002:00000f1c       ?heap@@3V_HeapManager@@A   10013f1c     libvcruntime:undname.obj
 0002:00000f34       ?c_termination_complete@@3JA 10013f34     libucrt:exit.obj
 0002:00000f38       ?thread_local_exit_callback_func@@3P6GXPAXK0@ZA 10013f38     libucrt:exit.obj
 0002:00000f40       ?program_name@?1???$common_configure_argv@D@@YAHW4_crt_argv_mode@@@Z@4PADA 10013f40     libucrt:argv_parsing.obj
 0002:00001070       ?__acrt_lock_table@@3PAU_RTL_CRITICAL_SECTION@@A 10014070     libucrt:locks.obj
 0002:000011c0       ?__acrt_locks_initialized@@3IA 100141c0     libucrt:locks.obj
 0002:000011c4       ?__acrt_invalid_parameter_handler@@3V?$dual_state_global@P6AXPB_W00II@Z@__crt_state_management@@A 100141c4     libucrt:invalid_parameter.obj
 0002:000011d4       ?fSystemSet@@3HA           100141d4     libucrt:mbctype.obj
 0002:000011d8       ?initialized@?1??__acrt_initialize_multibyte@@9@4_NA 100141d8     libucrt:mbctype.obj
 0002:00001400       ?module_handles@@3PAPAUHINSTANCE__@@A 10014400     libucrt:winapi_thunks.obj
 0002:00001450       ?encoded_function_pointers@@3PAPAXA 10014450     libucrt:winapi_thunks.obj
 0002:000014dc       ?__acrt_new_handler@@3V?$dual_state_global@P6AHI@Z@__crt_state_management@@A 100144dc     libucrt:new_handler.obj
 0002:000014e0       ?ctrlc_action@@3V?$dual_state_global@P6AXH@Z@__crt_state_management@@A 100144e0     libucrt:signal.obj
 0002:000014e4       ?ctrlbreak_action@@3V?$dual_state_global@P6AXH@Z@__crt_state_management@@A 100144e4     libucrt:signal.obj
 0002:000014e8       ?abort_action@@3V?$dual_state_global@P6AXH@Z@__crt_state_management@@A 100144e8     libucrt:signal.obj
 0002:000014ec       ?term_action@@3V?$dual_state_global@P6AXH@Z@__crt_state_management@@A 100144ec     libucrt:signal.obj
 0002:000014f0       ?user_matherr@@3V?$dual_state_global@P6AHPAU_exception@@@Z@__crt_state_management@@A 100144f0     libucrt:matherr.obj
 0002:00001508       ?internal_state@?1??_mbtowc_l@@9@4U_Mbstatet@@A 10014508     libucrt:mbtowc.obj
 0002:00001514       ?__acrt_global_new_mode@@3V?$dual_state_global@J@__crt_state_management@@A 10014514     libucrt:new_mode.obj
 0002:00001520       ?__acrt_app_type@@3W4_crt_app_type@@A 10014520     libucrt:report_runtime_error.obj
 0002:00001524       ?internal_pst@?1??__mbrtoc32_utf8@__crt_mbstring@@YAIPA_UPBDIPAU_Mbstatet@@@Z@4U3@A 10014524     libucrt:mbrtoc32.obj
 0002:00001530       __pmatherr_set             10014530     libucrt:libm_error.obj
 0003:00000332       .idata$6                   10015332     kernel32:KERNEL32.dll
 0004:00000060       $R000000                   10016060     DrawLine.res
